 vJoyInterface

 Timestamp is 63bd7cb3 (Tue Jan 10 08:56:51 2023)

 Preferred load address is 10000000

 Start         Length     Name                   Class
 0001:00000000 00010000H .textbss                DATA
 0002:00000000 00002ea0H .text$di                CODE
 0002:00002ea0 0001cab0H .text$mn                CODE
 0002:0001f950 00001840H .text$x                 CODE
 0002:00021190 00001096H .text$yd                CODE
 0003:00000000 00000104H .CRT$XCA                DATA
 0003:00000104 0000010cH .CRT$XCU                DATA
 0003:00000210 00000104H .CRT$XCZ                DATA
 0003:00000314 00000104H .CRT$XIA                DATA
 0003:00000418 00000104H .CRT$XIZ                DATA
 0003:0000051c 00000104H .CRT$XPA                DATA
 0003:00000620 00000104H .CRT$XPZ                DATA
 0003:00000724 00000104H .CRT$XTA                DATA
 0003:00000828 00000108H .CRT$XTZ                DATA
 0003:00000930 00002f90H .rdata                  DATA
 0003:000038c0 00000180H .rdata$CastGuardVftablesA DATA
 0003:00003a40 0000014cH .rdata$CastGuardVftablesC DATA
 0003:00003b8c 00000274H .rdata$r                DATA
 0003:00003e00 00000184H .rdata$zzzdbg           DATA
 0003:00003f84 00000104H .rtc$IAA                DATA
 0003:00004088 00000104H .rtc$IMZ                DATA
 0003:0000418c 00000104H .rtc$IZZ                DATA
 0003:00004290 00000104H .rtc$TAA                DATA
 0003:00004394 00000104H .rtc$TMZ                DATA
 0003:00004498 00000108H .rtc$TZZ                DATA
 0003:000045a0 000008d0H .xdata$x                DATA
 0003:00004e70 0000070aH .edata                  DATA
 0004:00000000 00000194H .data                   DATA
 0004:00000194 00000178H .data$r                 DATA
 0004:0000030c 0000011cH .data$rs                DATA
 0004:00000428 000004f4H .bss                    DATA
 0005:00000000 000003c0H .idata$5                DATA
 0005:000003c0 000000a0H .idata$2                DATA
 0005:00000460 00000014H .idata$3                DATA
 0005:00000474 000003c0H .idata$4                DATA
 0005:00000834 00000c58H .idata$6                DATA
 0006:00000000 0000031cH .msvcjmc                DATA
 0007:00000000 0000010eH .00cfg                  DATA
 0008:00000000 00000270H .rsrc$01                DATA
 0008:00000270 0000071cH .rsrc$02                DATA

  Address         Publics by Value              Rva+Base       Lib:Object

 0000:00000000       ___AbsoluteZero            00000000     <absolute>
 0000:00000000       ___arm64x_extra_rfe_table  00000000     <absolute>
 0000:00000000       ___arm64x_extra_rfe_table_size 00000000     <absolute>
 0000:00000000       ___arm64x_native_entrypoint 00000000     <absolute>
 0000:00000000       ___arm64x_redirection_metadata 00000000     <absolute>
 0000:00000000       ___arm64x_redirection_metadata_count 00000000     <absolute>
 0000:00000000       ___dynamic_value_reloc_table 00000000     <absolute>
 0000:00000000       ___enclave_config          00000000     <absolute>
 0000:00000000       ___guard_check_icall_a64n_fptr 00000000     <absolute>
 0000:00000000       ___guard_eh_cont_count     00000000     <absolute>
 0000:00000000       ___guard_eh_cont_table     00000000     <absolute>
 0000:00000000       ___guard_fids_count        00000000     <absolute>
 0000:00000000       ___guard_fids_table        00000000     <absolute>
 0000:00000000       ___guard_iat_count         00000000     <absolute>
 0000:00000000       ___guard_iat_table         00000000     <absolute>
 0000:00000000       ___guard_longjmp_count     00000000     <absolute>
 0000:00000000       ___guard_longjmp_table     00000000     <absolute>
 0000:00000000       ___hybrid_auxiliary_iat    00000000     <absolute>
 0000:00000000       ___hybrid_auxiliary_iat_copy 00000000     <absolute>
 0000:00000000       ___hybrid_code_map         00000000     <absolute>
 0000:00000000       ___hybrid_code_map_count   00000000     <absolute>
 0000:00000000       ___safe_se_handler_count   00000000     <absolute>
 0000:00000000       ___safe_se_handler_table   00000000     <absolute>
 0000:00000000       ___volatile_metadata       00000000     <absolute>
 0000:00000000       ___x64_code_ranges_to_entry_points 00000000     <absolute>
 0000:00000000       ___x64_code_ranges_to_entry_points_count 00000000     <absolute>
 0000:00000100       ___guard_flags             00000100     <absolute>
 0000:00000000       ___ImageBase               10000000     <linker-defined>
 0001:00000000       __enc$textbss$begin        10001000     <linker-defined>
 0001:00010000       __enc$textbss$end          10011000     <linker-defined>
 0002:00002ea0       __JustMyCode_Default       10013ea0 f i stdafx.obj
 0002:00002eb0       ??$?0$$QAH$$Z$$V@?$pair@$$CBHUDeviceStat@@@std@@QAE@Upiecewise_construct_t@1@V?$tuple@$$QAH@1@V?$tuple@$$V@1@@Z 10013eb0 f i vJoyInterface.obj
 0002:00002f40       ??$?0$$V@?$_Compressed_pair@V?$allocator@U?$_Tree_node@U?$pair@$$CBHUDeviceStat@@@std@@PAX@std@@@std@@V?$_Tree_val@U?$_Tree_simple_types@U?$pair@$$CBHUDeviceStat@@@std@@@std@@@2@$00@std@@QAE@U_Zero_then_variadic_args_t@1@@Z 10013f40 f i vJoyInterface.obj
 0002:00002fb0       ??$?0$$V@?$_Compressed_pair@V?$allocator@U?$_Tree_node@U?$pair@$$CBHW4FFB_EFFECTS@@@std@@PAX@std@@@std@@V?$_Tree_val@U?$_Tree_simple_types@U?$pair@$$CBHW4FFB_EFFECTS@@@std@@@std@@@2@$00@std@@QAE@U_Zero_then_variadic_args_t@1@@Z 10013fb0 f i vJoyInterface.obj
 0002:00003020       ??$?0AAHUDeviceStat@@$0A@@?$pair@$$CBHUDeviceStat@@@std@@QAE@AAH$$QAUDeviceStat@@@Z 10014020 f i vJoyInterface.obj
 0002:000030b0       ??$?0AAHUDeviceStat@@@?$_Tree_temp_node@V?$allocator@U?$_Tree_node@U?$pair@$$CBHUDeviceStat@@@std@@PAX@std@@@std@@@std@@QAE@AAV?$allocator@U?$_Tree_node@U?$pair@$$CBHUDeviceStat@@@std@@PAX@std@@@1@PAU?$_Tree_node@U?$pair@$$CBHUDeviceStat@@@std@@PAX@1@AAH$$QAUDeviceStat@@@Z 100140b0 f i vJoyInterface.obj
 0002:00003210       ??$?0AAPAU?$_Tree_node@U?$pair@$$CBHUDeviceStat@@@std@@PAX@std@@AAPAU01@$0A@@?$pair@PAU?$_Tree_node@U?$pair@$$CBHUDeviceStat@@@std@@PAX@std@@PAU12@@std@@QAE@AAPAU?$_Tree_node@U?$pair@$$CBHUDeviceStat@@@std@@PAX@1@0@Z 10014210 f i vJoyInterface.obj
 0002:000032a0       ??$?0AAPAU?$_Tree_node@U?$pair@$$CBHUDeviceStat@@@std@@PAX@std@@_N$0A@@?$pair@PAU?$_Tree_node@U?$pair@$$CBHUDeviceStat@@@std@@PAX@std@@_N@std@@QAE@AAPAU?$_Tree_node@U?$pair@$$CBHUDeviceStat@@@std@@PAX@1@$$QA_N@Z 100142a0 f i vJoyInterface.obj
 0002:00003330       ??$?0ABH$$Z$$V@?$pair@$$CBHUDeviceStat@@@std@@QAE@Upiecewise_construct_t@1@V?$tuple@ABH@1@V?$tuple@$$V@1@@Z 10014330 f i vJoyInterface.obj
 0002:000033c0       ??$?0ABH$0A@@?$tuple@ABH@std@@QAE@ABH@Z 100143c0 f i vJoyInterface.obj
 0002:00003470       ??$?0ABH@?$_Tuple_val@ABH@std@@QAE@ABH@Z 10014470 f i vJoyInterface.obj
 0002:000034e0       ??$?0ABQAU?$_Tree_node@U?$pair@$$CBHUDeviceStat@@@std@@PAX@std@@_N$0A@@?$pair@PAU?$_Tree_node@U?$pair@$$CBHUDeviceStat@@@std@@PAX@std@@_N@std@@QAE@ABQAU?$_Tree_node@U?$pair@$$CBHUDeviceStat@@@std@@PAX@1@$$QA_N@Z 100144e0 f i vJoyInterface.obj
 0002:00003570       ??$?0ABU?$less@H@std@@U_Zero_then_variadic_args_t@1@@?$_Compressed_pair@U?$less@H@std@@V?$_Compressed_pair@V?$allocator@U?$_Tree_node@U?$pair@$$CBHUDeviceStat@@@std@@PAX@std@@@std@@V?$_Tree_val@U?$_Tree_simple_types@U?$pair@$$CBHUDeviceStat@@@std@@@std@@@2@$00@2@$00@std@@QAE@U_One_then_variadic_args_t@1@ABU?$less@H@1@$$QAU_Zero_then_variadic_args_t@1@@Z 10014570 f i vJoyInterface.obj
 0002:00003600       ??$?0ABU?$less@H@std@@U_Zero_then_variadic_args_t@1@@?$_Compressed_pair@U?$less@H@std@@V?$_Compressed_pair@V?$allocator@U?$_Tree_node@U?$pair@$$CBHW4FFB_EFFECTS@@@std@@PAX@std@@@std@@V?$_Tree_val@U?$_Tree_simple_types@U?$pair@$$CBHW4FFB_EFFECTS@@@std@@@std@@@2@$00@2@$00@std@@QAE@U_One_then_variadic_args_t@1@ABU?$less@H@1@$$QAU_Zero_then_variadic_args_t@1@@Z 10014600 f i vJoyInterface.obj
 0002:00003690       ??$?0ABUpiecewise_construct_t@std@@V?$tuple@$$QAH@1@V?$tuple@$$V@1@@?$_Tree_temp_node@V?$allocator@U?$_Tree_node@U?$pair@$$CBHUDeviceStat@@@std@@PAX@std@@@std@@@std@@QAE@AAV?$allocator@U?$_Tree_node@U?$pair@$$CBHUDeviceStat@@@std@@PAX@std@@@1@PAU?$_Tree_node@U?$pair@$$CBHUDeviceStat@@@std@@PAX@1@ABUpiecewise_construct_t@1@$$QAV?$tuple@$$QAH@1@$$QAV?$tuple@$$V@1@@Z 10014690 f i vJoyInterface.obj
 0002:00003800       ??$?0ABUpiecewise_construct_t@std@@V?$tuple@ABH@1@V?$tuple@$$V@1@@?$_Tree_temp_node@V?$allocator@U?$_Tree_node@U?$pair@$$CBHUDeviceStat@@@std@@PAX@std@@@std@@@std@@QAE@AAV?$allocator@U?$_Tree_node@U?$pair@$$CBHUDeviceStat@@@std@@PAX@std@@@1@PAU?$_Tree_node@U?$pair@$$CBHUDeviceStat@@@std@@PAX@1@ABUpiecewise_construct_t@1@$$QAV?$tuple@ABH@1@$$QAV?$tuple@$$V@1@@Z 10014800 f i vJoyInterface.obj
 0002:00003970       ??$?0H$$V$0A@@?$tuple@$$QAH@std@@QAE@$$QAH@Z 10014970 f i vJoyInterface.obj
 0002:00003a30       ??$?0H@?$_Tuple_val@$$QAH@std@@QAE@$$QAH@Z 10014a30 f i vJoyInterface.obj
 0002:00003aa0       ??$?0PAU?$_Tree_node@U?$pair@$$CBHUDeviceStat@@@std@@PAX@std@@_N$0A@@?$pair@PAU?$_Tree_node@U?$pair@$$CBHUDeviceStat@@@std@@PAX@std@@_N@std@@QAE@$$QAPAU?$_Tree_node@U?$pair@$$CBHUDeviceStat@@@std@@PAX@1@$$QA_N@Z 10014aa0 f i vJoyInterface.obj
 0002:00003b30       ??$?0U?$_Tree_node@U?$pair@$$CBHUDeviceStat@@@std@@PAX@std@@@?$allocator@U_Container_proxy@std@@@std@@QAE@ABV?$allocator@U?$_Tree_node@U?$pair@$$CBHUDeviceStat@@@std@@PAX@std@@@1@@Z 10014b30 f i vJoyInterface.obj
 0002:00003b90       ??$?0U?$_Tree_node@U?$pair@$$CBHW4FFB_EFFECTS@@@std@@PAX@std@@@?$allocator@U_Container_proxy@std@@@std@@QAE@ABV?$allocator@U?$_Tree_node@U?$pair@$$CBHW4FFB_EFFECTS@@@std@@PAX@std@@@1@@Z 10014b90 f i vJoyInterface.obj
 0002:00003bf0       ??$?0U_Exact_args_t@std@@$0A@@?$tuple@$$V@std@@QAE@U_Exact_args_t@1@@Z 10014bf0 f i vJoyInterface.obj
 0002:00003c50       ??$?0U_Exact_args_t@std@@ABH$$V$0A@@?$tuple@ABH@std@@QAE@U_Exact_args_t@1@ABH@Z 10014c50 f i vJoyInterface.obj
 0002:00003ce0       ??$?0U_Exact_args_t@std@@H$$V$0A@@?$tuple@$$QAH@std@@QAE@U_Exact_args_t@1@$$QAH@Z 10014ce0 f i vJoyInterface.obj
 0002:00003d70       ??$?0V?$_Tree_iterator@V?$_Tree_val@U?$_Tree_simple_types@U?$pair@$$CBHUDeviceStat@@@std@@@std@@@std@@@std@@AB_N$0A@@?$pair@V?$_Tree_iterator@V?$_Tree_val@U?$_Tree_simple_types@U?$pair@$$CBHUDeviceStat@@@std@@@std@@@std@@@std@@_N@std@@QAE@$$QAV?$_Tree_iterator@V?$_Tree_val@U?$_Tree_simple_types@U?$pair@$$CBHUDeviceStat@@@std@@@std@@@std@@@1@AB_N@Z 10014d70 f i vJoyInterface.obj
 0002:00003e00       ??$?0V?$tuple@$$QAH@std@@V?$tuple@$$V@1@$0A@$$Z$S@?$pair@$$CBHUDeviceStat@@@std@@QAE@AAV?$tuple@$$QAH@1@AAV?$tuple@$$V@1@U?$integer_sequence@I$0A@@1@U?$integer_sequence@I$S@1@@Z 10014e00 f i vJoyInterface.obj
 0002:00003ea0       ??$?0V?$tuple@ABH@std@@V?$tuple@$$V@1@$0A@$$Z$S@?$pair@$$CBHUDeviceStat@@@std@@QAE@AAV?$tuple@ABH@1@AAV?$tuple@$$V@1@U?$integer_sequence@I$0A@@1@U?$integer_sequence@I$S@1@@Z 10014ea0 f i vJoyInterface.obj
 0002:00003f40       ??$_Adl_verify_range@V?$_Tree_unchecked_const_iterator@V?$_Tree_val@U?$_Tree_simple_types@U?$pair@$$CBHUDeviceStat@@@std@@@std@@@std@@U_Iterator_base0@2@@std@@V12@@std@@YAXABV?$_Tree_unchecked_const_iterator@V?$_Tree_val@U?$_Tree_simple_types@U?$pair@$$CBHUDeviceStat@@@std@@@std@@@std@@U_Iterator_base0@2@@0@0@Z 10014f40 f i vJoyInterface.obj
 0002:00003f90       ??$_Allocate@$07U_Default_allocate_traits@std@@$0A@@std@@YAPAXI@Z 10014f90 f i vJoyInterface.obj
 0002:00004010       ??$_Allocate_manually_vector_aligned@U_Default_allocate_traits@std@@@std@@YAPAXI@Z 10015010 f i vJoyInterface.obj
 0002:00004150       ??$_Buyheadnode@V?$allocator@U?$_Tree_node@U?$pair@$$CBHUDeviceStat@@@std@@PAX@std@@@std@@@?$_Tree_node@U?$pair@$$CBHUDeviceStat@@@std@@PAX@std@@SAPAU01@AAV?$allocator@U?$_Tree_node@U?$pair@$$CBHUDeviceStat@@@std@@PAX@std@@@1@@Z 10015150 f i vJoyInterface.obj
 0002:00004240       ??$_Buyheadnode@V?$allocator@U?$_Tree_node@U?$pair@$$CBHW4FFB_EFFECTS@@@std@@PAX@std@@@std@@@?$_Tree_node@U?$pair@$$CBHW4FFB_EFFECTS@@@std@@PAX@std@@SAPAU01@AAV?$allocator@U?$_Tree_node@U?$pair@$$CBHW4FFB_EFFECTS@@@std@@PAX@std@@@1@@Z 10015240 f i vJoyInterface.obj
 0002:00004330       ??$_Construct_in_place@PAU?$_Tree_node@U?$pair@$$CBHUDeviceStat@@@std@@PAX@std@@AAPAU12@@std@@YAXAAPAU?$_Tree_node@U?$pair@$$CBHUDeviceStat@@@std@@PAX@0@0@Z 10015330 f i vJoyInterface.obj
 0002:000043d0       ??$_Construct_in_place@PAU?$_Tree_node@U?$pair@$$CBHUDeviceStat@@@std@@PAX@std@@ABQAU12@@std@@YAXAAPAU?$_Tree_node@U?$pair@$$CBHUDeviceStat@@@std@@PAX@0@ABQAU10@@Z 100153d0 f i vJoyInterface.obj
 0002:00004470       ??$_Construct_in_place@PAU?$_Tree_node@U?$pair@$$CBHW4FFB_EFFECTS@@@std@@PAX@std@@ABQAU12@@std@@YAXAAPAU?$_Tree_node@U?$pair@$$CBHW4FFB_EFFECTS@@@std@@PAX@0@ABQAU10@@Z 10015470 f i vJoyInterface.obj
 0002:00004510       ??$_Construct_in_place@U_Container_proxy@std@@PAU_Container_base12@2@@std@@YAXAAU_Container_proxy@0@$$QAPAU_Container_base12@0@@Z 10015510 f i vJoyInterface.obj
 0002:000045b0       ??$_Deallocate@$07$0A@@std@@YAXPAXI@Z 100155b0 f i vJoyInterface.obj
 0002:00004670       ??$_Deallocate_plain@V?$allocator@U_Container_proxy@std@@@std@@@std@@YAXAAV?$allocator@U_Container_proxy@std@@@0@QAU_Container_proxy@0@@Z 10015670 f i vJoyInterface.obj
 0002:00004710       ??$_Debug_lt_pred@ABU?$less@H@std@@ABHABH$0A@@std@@YA_NABU?$less@H@0@ABH1@Z 10015710 f i vJoyInterface.obj
 0002:00004820       ??$_Delete_plain_internal@V?$allocator@U_Container_proxy@std@@@std@@@std@@YAXAAV?$allocator@U_Container_proxy@std@@@0@QAU_Container_proxy@0@@Z 10015820 f i vJoyInterface.obj
 0002:00004880       ??$_Destroy_in_place@PAU?$_Tree_node@U?$pair@$$CBHUDeviceStat@@@std@@PAX@std@@@std@@YAXAAPAU?$_Tree_node@U?$pair@$$CBHUDeviceStat@@@std@@PAX@0@@Z 10015880 f i vJoyInterface.obj
 0002:000048d0       ??$_Destroy_in_place@PAU?$_Tree_node@U?$pair@$$CBHW4FFB_EFFECTS@@@std@@PAX@std@@@std@@YAXAAPAU?$_Tree_node@U?$pair@$$CBHW4FFB_EFFECTS@@@std@@PAX@0@@Z 100158d0 f i vJoyInterface.obj
 0002:00004920       ??$_Emplace@AAHUDeviceStat@@@?$_Tree@V?$_Tmap_traits@HUDeviceStat@@U?$less@H@std@@V?$allocator@U?$pair@$$CBHUDeviceStat@@@std@@@3@$0A@@std@@@std@@IAE?AU?$pair@PAU?$_Tree_node@U?$pair@$$CBHUDeviceStat@@@std@@PAX@std@@_N@1@AAH$$QAUDeviceStat@@@Z 10015920 f i vJoyInterface.obj
 0002:00004b10       ??$_Eqrange@H@?$_Tree@V?$_Tmap_traits@HUDeviceStat@@U?$less@H@std@@V?$allocator@U?$pair@$$CBHUDeviceStat@@@std@@@3@$0A@@std@@@std@@IBE?AU?$pair@PAU?$_Tree_node@U?$pair@$$CBHUDeviceStat@@@std@@PAX@std@@PAU12@@1@ABH@Z 10015b10 f i vJoyInterface.obj
 0002:00004d90       ??$_Erase_head@V?$allocator@U?$_Tree_node@U?$pair@$$CBHUDeviceStat@@@std@@PAX@std@@@std@@@?$_Tree_val@U?$_Tree_simple_types@U?$pair@$$CBHUDeviceStat@@@std@@@std@@@std@@QAEXAAV?$allocator@U?$_Tree_node@U?$pair@$$CBHUDeviceStat@@@std@@PAX@std@@@1@@Z 10015d90 f i vJoyInterface.obj
 0002:00004e20       ??$_Erase_head@V?$allocator@U?$_Tree_node@U?$pair@$$CBHW4FFB_EFFECTS@@@std@@PAX@std@@@std@@@?$_Tree_val@U?$_Tree_simple_types@U?$pair@$$CBHW4FFB_EFFECTS@@@std@@@std@@@std@@QAEXAAV?$allocator@U?$_Tree_node@U?$pair@$$CBHW4FFB_EFFECTS@@@std@@PAX@std@@@1@@Z 10015e20 f i vJoyInterface.obj
 0002:00004eb0       ??$_Erase_tree@V?$allocator@U?$_Tree_node@U?$pair@$$CBHUDeviceStat@@@std@@PAX@std@@@std@@@?$_Tree_val@U?$_Tree_simple_types@U?$pair@$$CBHUDeviceStat@@@std@@@std@@@std@@QAEXAAV?$allocator@U?$_Tree_node@U?$pair@$$CBHUDeviceStat@@@std@@PAX@std@@@1@PAU?$_Tree_node@U?$pair@$$CBHUDeviceStat@@@std@@PAX@1@@Z 10015eb0 f i vJoyInterface.obj
 0002:00004f50       ??$_Erase_tree@V?$allocator@U?$_Tree_node@U?$pair@$$CBHW4FFB_EFFECTS@@@std@@PAX@std@@@std@@@?$_Tree_val@U?$_Tree_simple_types@U?$pair@$$CBHW4FFB_EFFECTS@@@std@@@std@@@std@@QAEXAAV?$allocator@U?$_Tree_node@U?$pair@$$CBHW4FFB_EFFECTS@@@std@@PAX@std@@@1@PAU?$_Tree_node@U?$pair@$$CBHW4FFB_EFFECTS@@@std@@PAX@1@@Z 10015f50 f i vJoyInterface.obj
 0002:00004ff0       ??$_Find@H@?$_Tree@V?$_Tmap_traits@HUDeviceStat@@U?$less@H@std@@V?$allocator@U?$pair@$$CBHUDeviceStat@@@std@@@3@$0A@@std@@@std@@ABEPAU?$_Tree_node@U?$pair@$$CBHUDeviceStat@@@std@@PAX@1@ABH@Z 10015ff0 f i vJoyInterface.obj
 0002:000050c0       ??$_Find_lower_bound@H@?$_Tree@V?$_Tmap_traits@HUDeviceStat@@U?$less@H@std@@V?$allocator@U?$pair@$$CBHUDeviceStat@@@std@@@3@$0A@@std@@@std@@IBE?AU?$_Tree_find_result@PAU?$_Tree_node@U?$pair@$$CBHUDeviceStat@@@std@@PAX@std@@@1@ABH@Z 100160c0 f i vJoyInterface.obj
 0002:00005220       ??$_Freenode0@V?$allocator@U?$_Tree_node@U?$pair@$$CBHUDeviceStat@@@std@@PAX@std@@@std@@@?$_Tree_node@U?$pair@$$CBHUDeviceStat@@@std@@PAX@std@@SAXAAV?$allocator@U?$_Tree_node@U?$pair@$$CBHUDeviceStat@@@std@@PAX@std@@@1@PAU01@@Z 10016220 f i vJoyInterface.obj
 0002:000052f0       ??$_Freenode0@V?$allocator@U?$_Tree_node@U?$pair@$$CBHW4FFB_EFFECTS@@@std@@PAX@std@@@std@@@?$_Tree_node@U?$pair@$$CBHW4FFB_EFFECTS@@@std@@PAX@std@@SAXAAV?$allocator@U?$_Tree_node@U?$pair@$$CBHW4FFB_EFFECTS@@@std@@PAX@std@@@1@PAU01@@Z 100162f0 f i vJoyInterface.obj
 0002:000053c0       ??$_Freenode@V?$allocator@U?$_Tree_node@U?$pair@$$CBHUDeviceStat@@@std@@PAX@std@@@std@@@?$_Tree_node@U?$pair@$$CBHUDeviceStat@@@std@@PAX@std@@SAXAAV?$allocator@U?$_Tree_node@U?$pair@$$CBHUDeviceStat@@@std@@PAX@std@@@1@PAU01@@Z 100163c0 f i vJoyInterface.obj
 0002:00005480       ??$_Freenode@V?$allocator@U?$_Tree_node@U?$pair@$$CBHW4FFB_EFFECTS@@@std@@PAX@std@@@std@@@?$_Tree_node@U?$pair@$$CBHW4FFB_EFFECTS@@@std@@PAX@std@@SAXAAV?$allocator@U?$_Tree_node@U?$pair@$$CBHW4FFB_EFFECTS@@@std@@PAX@std@@@1@PAU01@@Z 10016480 f i vJoyInterface.obj
 0002:00005540       ??$_Get_size_of_n@$07@std@@YAII@Z 10016540 f i vJoyInterface.obj
 0002:000055b0       ??$_Get_size_of_n@$0BI@@std@@YAII@Z 100165b0 f i vJoyInterface.obj
 0002:00005620       ??$_Get_size_of_n@$0OE@@std@@YAII@Z 10016620 f i vJoyInterface.obj
 0002:00005690       ??$_Get_unwrapped@AAV?$_Tree_unchecked_const_iterator@V?$_Tree_val@U?$_Tree_simple_types@U?$pair@$$CBHUDeviceStat@@@std@@@std@@@std@@U_Iterator_base0@2@@std@@@std@@YA?A_TAAV?$_Tree_unchecked_const_iterator@V?$_Tree_val@U?$_Tree_simple_types@U?$pair@$$CBHUDeviceStat@@@std@@@std@@@std@@U_Iterator_base0@2@@0@@Z 10016690 f i vJoyInterface.obj
 0002:000056e0       ??$_Kfn@$$CBHUDeviceStat@@@?$_Tmap_traits@HUDeviceStat@@U?$less@H@std@@V?$allocator@U?$pair@$$CBHUDeviceStat@@@std@@@3@$0A@@std@@SAABHABU?$pair@$$CBHUDeviceStat@@@1@@Z 100166e0 f i vJoyInterface.obj
 0002:00005730       ??$_Lower_bound_duplicate@H@?$_Tree@V?$_Tmap_traits@HUDeviceStat@@U?$less@H@std@@V?$allocator@U?$pair@$$CBHUDeviceStat@@@std@@@3@$0A@@std@@@std@@IBE_NQAU?$_Tree_node@U?$pair@$$CBHUDeviceStat@@@std@@PAX@1@ABH@Z 10016730 f i vJoyInterface.obj
 0002:000057f0       ??$_Try_emplace@ABH$$V@?$map@HUDeviceStat@@U?$less@H@std@@V?$allocator@U?$pair@$$CBHUDeviceStat@@@std@@@3@@std@@AAE?AU?$pair@PAU?$_Tree_node@U?$pair@$$CBHUDeviceStat@@@std@@PAX@std@@_N@1@ABH@Z 100167f0 f i vJoyInterface.obj
 0002:000059c0       ??$_Try_emplace@H$$V@?$map@HUDeviceStat@@U?$less@H@std@@V?$allocator@U?$pair@$$CBHUDeviceStat@@@std@@@3@@std@@AAE?AU?$pair@PAU?$_Tree_node@U?$pair@$$CBHUDeviceStat@@@std@@PAX@std@@_N@1@$$QAH@Z 100169c0 f i vJoyInterface.obj
 0002:00005b90       ??$_Tuple_get@$0A@$$QAH@std@@YA$$QA_P$$QAV?$tuple@$$QAH@0@@Z 10016b90 f i vJoyInterface.obj
 0002:00005be0       ??$_Tuple_get@$0A@ABH@std@@YA$$QA_P$$QAV?$tuple@ABH@0@@Z 10016be0 f i vJoyInterface.obj
 0002:00005c30       ??$_Unfancy@U_Container_proxy@std@@@std@@YAPAU_Container_proxy@0@PAU10@@Z 10016c30 f i vJoyInterface.obj
 0002:00005c80       ??$_Voidify_iter@PAPAU?$_Tree_node@U?$pair@$$CBHUDeviceStat@@@std@@PAX@std@@@std@@YAPAXPAPAU?$_Tree_node@U?$pair@$$CBHUDeviceStat@@@std@@PAX@0@@Z 10016c80 f i vJoyInterface.obj
 0002:00005cd0       ??$_Voidify_iter@PAPAU?$_Tree_node@U?$pair@$$CBHW4FFB_EFFECTS@@@std@@PAX@std@@@std@@YAPAXPAPAU?$_Tree_node@U?$pair@$$CBHW4FFB_EFFECTS@@@std@@PAX@0@@Z 10016cd0 f i vJoyInterface.obj
 0002:00005d20       ??$_Voidify_iter@PAU?$pair@$$CBHUDeviceStat@@@std@@@std@@YAPAXPAU?$pair@$$CBHUDeviceStat@@@0@@Z 10016d20 f i vJoyInterface.obj
 0002:00005d70       ??$_Voidify_iter@PAU_Container_proxy@std@@@std@@YAPAXPAU_Container_proxy@0@@Z 10016d70 f i vJoyInterface.obj
 0002:00005dc0       ??$addressof@$$CBV?$_Tree_val@U?$_Tree_simple_types@U?$pair@$$CBHUDeviceStat@@@std@@@std@@@std@@@std@@YAPBV?$_Tree_val@U?$_Tree_simple_types@U?$pair@$$CBHUDeviceStat@@@std@@@std@@@0@ABV10@@Z 10016dc0 f i vJoyInterface.obj
 0002:00005e10       ??$addressof@PAU?$_Tree_node@U?$pair@$$CBHUDeviceStat@@@std@@PAX@std@@@std@@YAPAPAU?$_Tree_node@U?$pair@$$CBHUDeviceStat@@@std@@PAX@0@AAPAU10@@Z 10016e10 f i vJoyInterface.obj
 0002:00005e60       ??$addressof@PAU?$_Tree_node@U?$pair@$$CBHW4FFB_EFFECTS@@@std@@PAX@std@@@std@@YAPAPAU?$_Tree_node@U?$pair@$$CBHW4FFB_EFFECTS@@@std@@PAX@0@AAPAU10@@Z 10016e60 f i vJoyInterface.obj
 0002:00005eb0       ??$addressof@U?$pair@$$CBHUDeviceStat@@@std@@@std@@YAPAU?$pair@$$CBHUDeviceStat@@@0@AAU10@@Z 10016eb0 f i vJoyInterface.obj
 0002:00005f00       ??$addressof@U?$pair@$$CBHW4FFB_EFFECTS@@@std@@@std@@YAPAU?$pair@$$CBHW4FFB_EFFECTS@@@0@AAU10@@Z 10016f00 f i vJoyInterface.obj
 0002:00005f50       ??$addressof@U_Container_base12@std@@@std@@YAPAU_Container_base12@0@AAU10@@Z 10016f50 f i vJoyInterface.obj
 0002:00005fa0       ??$addressof@U_Container_proxy@std@@@std@@YAPAU_Container_proxy@0@AAU10@@Z 10016fa0 f i vJoyInterface.obj
 0002:00005ff0       ??$addressof@V?$_Tree_val@U?$_Tree_simple_types@U?$pair@$$CBHUDeviceStat@@@std@@@std@@@std@@@std@@YAPAV?$_Tree_val@U?$_Tree_simple_types@U?$pair@$$CBHUDeviceStat@@@std@@@std@@@0@AAV10@@Z 10016ff0 f i vJoyInterface.obj
 0002:00006040       ??$addressof@V?$_Tree_val@U?$_Tree_simple_types@U?$pair@$$CBHW4FFB_EFFECTS@@@std@@@std@@@std@@@std@@YAPAV?$_Tree_val@U?$_Tree_simple_types@U?$pair@$$CBHW4FFB_EFFECTS@@@std@@@std@@@0@AAV10@@Z 10017040 f i vJoyInterface.obj
 0002:00006090       ??$construct@U?$pair@$$CBHUDeviceStat@@@std@@AAHUDeviceStat@@@?$_Default_allocator_traits@V?$allocator@U?$_Tree_node@U?$pair@$$CBHUDeviceStat@@@std@@PAX@std@@@std@@@std@@SAXAAV?$allocator@U?$_Tree_node@U?$pair@$$CBHUDeviceStat@@@std@@PAX@std@@@1@QAU?$pair@$$CBHUDeviceStat@@@1@AAH$$QAUDeviceStat@@@Z 10017090 f i vJoyInterface.obj
 0002:00006130       ??$construct@U?$pair@$$CBHUDeviceStat@@@std@@ABUpiecewise_construct_t@2@V?$tuple@$$QAH@2@V?$tuple@$$V@2@@?$_Default_allocator_traits@V?$allocator@U?$_Tree_node@U?$pair@$$CBHUDeviceStat@@@std@@PAX@std@@@std@@@std@@SAXAAV?$allocator@U?$_Tree_node@U?$pair@$$CBHUDeviceStat@@@std@@PAX@std@@@1@QAU?$pair@$$CBHUDeviceStat@@@1@ABUpiecewise_construct_t@1@$$QAV?$tuple@$$QAH@1@$$QAV?$tuple@$$V@1@@Z 10017130 f i vJoyInterface.obj
 0002:00006200       ??$construct@U?$pair@$$CBHUDeviceStat@@@std@@ABUpiecewise_construct_t@2@V?$tuple@ABH@2@V?$tuple@$$V@2@@?$_Default_allocator_traits@V?$allocator@U?$_Tree_node@U?$pair@$$CBHUDeviceStat@@@std@@PAX@std@@@std@@@std@@SAXAAV?$allocator@U?$_Tree_node@U?$pair@$$CBHUDeviceStat@@@std@@PAX@std@@@1@QAU?$pair@$$CBHUDeviceStat@@@1@ABUpiecewise_construct_t@1@$$QAV?$tuple@ABH@1@$$QAV?$tuple@$$V@1@@Z 10017200 f i vJoyInterface.obj
 0002:000062d0       ??$destroy@U?$pair@$$CBHUDeviceStat@@@std@@@?$_Default_allocator_traits@V?$allocator@U?$_Tree_node@U?$pair@$$CBHUDeviceStat@@@std@@PAX@std@@@std@@@std@@SAXAAV?$allocator@U?$_Tree_node@U?$pair@$$CBHUDeviceStat@@@std@@PAX@std@@@1@QAU?$pair@$$CBHUDeviceStat@@@1@@Z 100172d0 f i vJoyInterface.obj
 0002:00006320       ??$destroy@U?$pair@$$CBHW4FFB_EFFECTS@@@std@@@?$_Default_allocator_traits@V?$allocator@U?$_Tree_node@U?$pair@$$CBHW4FFB_EFFECTS@@@std@@PAX@std@@@std@@@std@@SAXAAV?$allocator@U?$_Tree_node@U?$pair@$$CBHW4FFB_EFFECTS@@@std@@PAX@std@@@1@QAU?$pair@$$CBHW4FFB_EFFECTS@@@1@@Z 10017320 f i vJoyInterface.obj
 0002:00006370       ??$distance@V?$_Tree_unchecked_const_iterator@V?$_Tree_val@U?$_Tree_simple_types@U?$pair@$$CBHUDeviceStat@@@std@@@std@@@std@@U_Iterator_base0@2@@std@@@std@@YAHV?$_Tree_unchecked_const_iterator@V?$_Tree_val@U?$_Tree_simple_types@U?$pair@$$CBHUDeviceStat@@@std@@@std@@@std@@U_Iterator_base0@2@@0@0@Z 10017370 f i vJoyInterface.obj
 0002:00006490       ??$emplace@AAHUDeviceStat@@@?$_Tree@V?$_Tmap_traits@HUDeviceStat@@U?$less@H@std@@V?$allocator@U?$pair@$$CBHUDeviceStat@@@std@@@3@$0A@@std@@@std@@QAE?AU?$pair@V?$_Tree_iterator@V?$_Tree_val@U?$_Tree_simple_types@U?$pair@$$CBHUDeviceStat@@@std@@@std@@@std@@@std@@_N@1@AAH$$QAUDeviceStat@@@Z 10017490 f i vJoyInterface.obj
 0002:000065c0       ??$exchange@PAU?$_Tree_node@U?$pair@$$CBHUDeviceStat@@@std@@PAX@std@@$$T@std@@YAPAU?$_Tree_node@U?$pair@$$CBHUDeviceStat@@@std@@PAX@0@AAPAU10@$$QA$$T@Z 100175c0 f i vJoyInterface.obj
 0002:00006630       ??$exchange@PAU?$_Tree_node@U?$pair@$$CBHUDeviceStat@@@std@@PAX@std@@AAPAU12@@std@@YAPAU?$_Tree_node@U?$pair@$$CBHUDeviceStat@@@std@@PAX@0@AAPAU10@0@Z 10017630 f i vJoyInterface.obj
 0002:000066a0       ??$exchange@PAU?$_Tree_node@U?$pair@$$CBHW4FFB_EFFECTS@@@std@@PAX@std@@AAPAU12@@std@@YAPAU?$_Tree_node@U?$pair@$$CBHW4FFB_EFFECTS@@@std@@PAX@0@AAPAU10@0@Z 100176a0 f i vJoyInterface.obj
 0002:00006710       ??$exchange@PAU_Iterator_base12@std@@$$T@std@@YAPAU_Iterator_base12@0@AAPAU10@$$QA$$T@Z 10017710 f i vJoyInterface.obj
 0002:00006780       ??$forward@AAH@std@@YAAAHAAH@Z 10017780 f i vJoyInterface.obj
 0002:000067d0       ??$forward@AAPAU?$_Tree_node@U?$pair@$$CBHUDeviceStat@@@std@@PAX@std@@@std@@YAAAPAU?$_Tree_node@U?$pair@$$CBHUDeviceStat@@@std@@PAX@0@AAPAU10@@Z 100177d0 f i vJoyInterface.obj
 0002:00006820       ??$forward@ABH@std@@YAABHABH@Z 10017820 f i vJoyInterface.obj
 0002:00006870       ??$forward@ABQAU?$_Tree_node@U?$pair@$$CBHUDeviceStat@@@std@@PAX@std@@@std@@YAABQAU?$_Tree_node@U?$pair@$$CBHUDeviceStat@@@std@@PAX@0@ABQAU10@@Z 10017870 f i vJoyInterface.obj
 0002:000068c0       ??$forward@ABQAU?$_Tree_node@U?$pair@$$CBHW4FFB_EFFECTS@@@std@@PAX@std@@@std@@YAABQAU?$_Tree_node@U?$pair@$$CBHW4FFB_EFFECTS@@@std@@PAX@0@ABQAU10@@Z 100178c0 f i vJoyInterface.obj
 0002:00006910       ??$forward@ABU?$less@H@std@@@std@@YAABU?$less@H@0@ABU10@@Z 10017910 f i vJoyInterface.obj
 0002:00006960       ??$forward@ABUpiecewise_construct_t@std@@@std@@YAABUpiecewise_construct_t@0@ABU10@@Z 10017960 f i vJoyInterface.obj
 0002:000069b0       ??$forward@AB_N@std@@YAAB_NAB_N@Z 100179b0 f i vJoyInterface.obj
 0002:00006a00       ??$forward@H@std@@YA$$QAHAAH@Z 10017a00 f i vJoyInterface.obj
 0002:00006a50       ??$forward@PAU?$_Tree_node@U?$pair@$$CBHUDeviceStat@@@std@@PAX@std@@@std@@YA$$QAPAU?$_Tree_node@U?$pair@$$CBHUDeviceStat@@@std@@PAX@0@AAPAU10@@Z 10017a50 f i vJoyInterface.obj
 0002:00006aa0       ??$forward@PAU_Container_base12@std@@@std@@YA$$QAPAU_Container_base12@0@AAPAU10@@Z 10017aa0 f i vJoyInterface.obj
 0002:00006af0       ??$forward@UDeviceStat@@@std@@YA$$QAUDeviceStat@@AAU1@@Z 10017af0 f i vJoyInterface.obj
 0002:00006b40       ??$forward@U_Zero_then_variadic_args_t@std@@@std@@YA$$QAU_Zero_then_variadic_args_t@0@AAU10@@Z 10017b40 f i vJoyInterface.obj
 0002:00006b90       ??$forward@V?$_Tree_iterator@V?$_Tree_val@U?$_Tree_simple_types@U?$pair@$$CBHUDeviceStat@@@std@@@std@@@std@@@std@@@std@@YA$$QAV?$_Tree_iterator@V?$_Tree_val@U?$_Tree_simple_types@U?$pair@$$CBHUDeviceStat@@@std@@@std@@@std@@@0@AAV10@@Z 10017b90 f i vJoyInterface.obj
 0002:00006be0       ??$forward@V?$tuple@$$QAH@std@@@std@@YA$$QAV?$tuple@$$QAH@0@AAV10@@Z 10017be0 f i vJoyInterface.obj
 0002:00006c30       ??$forward@V?$tuple@$$V@std@@@std@@YA$$QAV?$tuple@$$V@0@AAV10@@Z 10017c30 f i vJoyInterface.obj
 0002:00006c80       ??$forward@V?$tuple@ABH@std@@@std@@YA$$QAV?$tuple@ABH@0@AAV10@@Z 10017c80 f i vJoyInterface.obj
 0002:00006cd0       ??$forward@_N@std@@YA$$QA_NAA_N@Z 10017cd0 f i vJoyInterface.obj
 0002:00006d20       ??$forward_as_tuple@$$V@std@@YA?AV?$tuple@$$V@0@XZ 10017d20 f i vJoyInterface.obj
 0002:00006d70       ??$forward_as_tuple@ABH@std@@YA?AV?$tuple@ABH@0@ABH@Z 10017d70 f i vJoyInterface.obj
 0002:00006dd0       ??$forward_as_tuple@H@std@@YA?AV?$tuple@$$QAH@0@$$QAH@Z 10017dd0 f i vJoyInterface.obj
 0002:00006e30       ??$min@I@std@@YAABIABI0@Z  10017e30 f i vJoyInterface.obj
 0002:00006ec0       ??$move@AAD@std@@YA$$QADAAD@Z 10017ec0 f i vJoyInterface.obj
 0002:00006f10       ??$move@AAH@std@@YA$$QAHAAH@Z 10017f10 f i vJoyInterface.obj
 0002:00006f60       ??$move@AAV?$tuple@$$QAH@std@@@std@@YA$$QAV?$tuple@$$QAH@0@AAV10@@Z 10017f60 f i vJoyInterface.obj
 0002:00006fb0       ??$move@AAV?$tuple@ABH@std@@@std@@YA$$QAV?$tuple@ABH@0@AAV10@@Z 10017fb0 f i vJoyInterface.obj
 0002:00007000       ??$swap@D$0A@@std@@YAXAAD0@Z 10018000 f i vJoyInterface.obj
 0002:000070d0       ??0?$_Alloc_construct_ptr@V?$allocator@U?$_Tree_node@U?$pair@$$CBHUDeviceStat@@@std@@PAX@std@@@std@@@std@@QAE@AAV?$allocator@U?$_Tree_node@U?$pair@$$CBHUDeviceStat@@@std@@PAX@std@@@1@@Z 100180d0 f i vJoyInterface.obj
 0002:00007140       ??0?$_Container_proxy_ptr12@V?$allocator@U_Container_proxy@std@@@std@@@std@@QAE@AAV?$allocator@U_Container_proxy@std@@@1@AAU_Container_base12@1@@Z 10018140 f i vJoyInterface.obj
 0002:00007210       ??0?$_Tree@V?$_Tmap_traits@HUDeviceStat@@U?$less@H@std@@V?$allocator@U?$pair@$$CBHUDeviceStat@@@std@@@3@$0A@@std@@@std@@QAE@ABU?$less@H@1@@Z 10018210 f i vJoyInterface.obj
 0002:00007290       ??0?$_Tree@V?$_Tmap_traits@HW4FFB_EFFECTS@@U?$less@H@std@@V?$allocator@U?$pair@$$CBHW4FFB_EFFECTS@@@std@@@3@$0A@@std@@@std@@QAE@ABU?$less@H@1@@Z 10018290 f i vJoyInterface.obj
 0002:00007310       ??0?$_Tree_const_iterator@V?$_Tree_val@U?$_Tree_simple_types@U?$pair@$$CBHUDeviceStat@@@std@@@std@@@std@@@std@@QAE@$$QAV01@@Z 10018310 f i vJoyInterface.obj
 0002:00007370       ??0?$_Tree_const_iterator@V?$_Tree_val@U?$_Tree_simple_types@U?$pair@$$CBHUDeviceStat@@@std@@@std@@@std@@@std@@QAE@PAU?$_Tree_node@U?$pair@$$CBHUDeviceStat@@@std@@PAX@1@PBV?$_Tree_val@U?$_Tree_simple_types@U?$pair@$$CBHUDeviceStat@@@std@@@std@@@1@@Z 10018370 f i vJoyInterface.obj
 0002:000073d0       ??0?$_Tree_iterator@V?$_Tree_val@U?$_Tree_simple_types@U?$pair@$$CBHUDeviceStat@@@std@@@std@@@std@@@std@@QAE@$$QAV01@@Z 100183d0 f i vJoyInterface.obj
 0002:00007430       ??0?$_Tree_iterator@V?$_Tree_val@U?$_Tree_simple_types@U?$pair@$$CBHUDeviceStat@@@std@@@std@@@std@@@std@@QAE@PAU?$_Tree_node@U?$pair@$$CBHUDeviceStat@@@std@@PAX@1@PBV?$_Tree_val@U?$_Tree_simple_types@U?$pair@$$CBHUDeviceStat@@@std@@@std@@@1@@Z 10018430 f i vJoyInterface.obj
 0002:00007490       ??0?$_Tree_temp_node_alloc@V?$allocator@U?$_Tree_node@U?$pair@$$CBHUDeviceStat@@@std@@PAX@std@@@std@@@std@@QAE@AAV?$allocator@U?$_Tree_node@U?$pair@$$CBHUDeviceStat@@@std@@PAX@std@@@1@@Z 10018490 f i vJoyInterface.obj
 0002:00007550       ??0?$_Tree_unchecked_const_iterator@V?$_Tree_val@U?$_Tree_simple_types@U?$pair@$$CBHUDeviceStat@@@std@@@std@@@std@@U_Iterator_base0@2@@std@@QAE@PAU?$_Tree_node@U?$pair@$$CBHUDeviceStat@@@std@@PAX@1@PBV?$_Tree_val@U?$_Tree_simple_types@U?$pair@$$CBHUDeviceStat@@@std@@@std@@@1@@Z 10018550 f i vJoyInterface.obj
 0002:000075c0       ??0?$_Tree_unchecked_const_iterator@V?$_Tree_val@U?$_Tree_simple_types@U?$pair@$$CBHUDeviceStat@@@std@@@std@@@std@@U_Iterator_base12@2@@std@@QAE@$$QAV01@@Z 100185c0 f i vJoyInterface.obj
 0002:00007630       ??0?$_Tree_unchecked_const_iterator@V?$_Tree_val@U?$_Tree_simple_types@U?$pair@$$CBHUDeviceStat@@@std@@@std@@@std@@U_Iterator_base12@2@@std@@QAE@PAU?$_Tree_node@U?$pair@$$CBHUDeviceStat@@@std@@PAX@1@PBV?$_Tree_val@U?$_Tree_simple_types@U?$pair@$$CBHUDeviceStat@@@std@@@std@@@1@@Z 10018630 f i vJoyInterface.obj
 0002:000076b0       ??0?$_Tree_unchecked_iterator@V?$_Tree_val@U?$_Tree_simple_types@U?$pair@$$CBHUDeviceStat@@@std@@@std@@@std@@@std@@QAE@PAU?$_Tree_node@U?$pair@$$CBHUDeviceStat@@@std@@PAX@1@PBV?$_Tree_val@U?$_Tree_simple_types@U?$pair@$$CBHUDeviceStat@@@std@@@std@@@1@@Z 100186b0 f i vJoyInterface.obj
 0002:00007710       ??0?$_Tree_val@U?$_Tree_simple_types@U?$pair@$$CBHUDeviceStat@@@std@@@std@@@std@@QAE@XZ 10018710 f i vJoyInterface.obj
 0002:00007790       ??0?$_Tree_val@U?$_Tree_simple_types@U?$pair@$$CBHW4FFB_EFFECTS@@@std@@@std@@@std@@QAE@XZ 10018790 f i vJoyInterface.obj
 0002:00007810       ??0?$allocator@U?$_Tree_node@U?$pair@$$CBHUDeviceStat@@@std@@PAX@std@@@std@@QAE@XZ 10018810 f i vJoyInterface.obj
 0002:00007870       ??0?$allocator@U?$_Tree_node@U?$pair@$$CBHW4FFB_EFFECTS@@@std@@PAX@std@@@std@@QAE@XZ 10018870 f i vJoyInterface.obj
 0002:000078d0       ??0?$map@HUDeviceStat@@U?$less@H@std@@V?$allocator@U?$pair@$$CBHUDeviceStat@@@std@@@3@@std@@QAE@XZ 100188d0 f i vJoyInterface.obj
 0002:00007940       ??0?$map@HW4FFB_EFFECTS@@U?$less@H@std@@V?$allocator@U?$pair@$$CBHW4FFB_EFFECTS@@@std@@@3@@std@@QAE@XZ 10018940 f i vJoyInterface.obj
 0002:000079b0       ??0?$tuple@$$QAH@std@@QAE@$$QAV01@@Z 100189b0 f i vJoyInterface.obj
 0002:00007a20       ??0?$tuple@$$V@std@@QAE@ABV01@@Z 10018a20 f i vJoyInterface.obj
 0002:00007a80       ??0?$tuple@ABH@std@@QAE@$$QAV01@@Z 10018a80 f i vJoyInterface.obj
 0002:00007af0       ??0_Basic_container_proxy_ptr12@std@@IAE@XZ 10018af0 f i vJoyInterface.obj
 0002:00007b50       ??0_Container_base12@std@@QAE@XZ 10018b50 f i vJoyInterface.obj
 0002:00007bb0       ??0_Container_proxy@std@@QAE@PAU_Container_base12@1@@Z 10018bb0 f i vJoyInterface.obj
 0002:00007c20       ??0_Iterator_base12@std@@QAE@ABU01@@Z 10018c20 f i vJoyInterface.obj
 0002:00007ca0       ??0_Iterator_base12@std@@QAE@XZ 10018ca0 f i vJoyInterface.obj
 0002:00007d10       ??0bad_alloc@std@@AAE@QBD@Z 10018d10 f i vJoyInterface.obj
 0002:00007d80       ??0bad_alloc@std@@QAE@ABV01@@Z 10018d80 f i vJoyInterface.obj
 0002:00007df0       ??0bad_array_new_length@std@@QAE@ABV01@@Z 10018df0 f i vJoyInterface.obj
 0002:00007e60       ??0bad_array_new_length@std@@QAE@XZ 10018e60 f i vJoyInterface.obj
 0002:00007ed0       ??0exception@std@@QAE@ABV01@@Z 10018ed0 f i vJoyInterface.obj
 0002:00007f60       ??0exception@std@@QAE@QBDH@Z 10018f60 f i vJoyInterface.obj
 0002:00007fe0       ??1?$_Alloc_construct_ptr@V?$allocator@U?$_Tree_node@U?$pair@$$CBHUDeviceStat@@@std@@PAX@std@@@std@@@std@@QAE@XZ 10018fe0 f i vJoyInterface.obj
 0002:00008090       ??1?$_Container_proxy_ptr12@V?$allocator@U_Container_proxy@std@@@std@@@std@@QAE@XZ 10019090 f i vJoyInterface.obj
 0002:00008110       ??1?$_Tree@V?$_Tmap_traits@HUDeviceStat@@U?$less@H@std@@V?$allocator@U?$pair@$$CBHUDeviceStat@@@std@@@3@$0A@@std@@@std@@QAE@XZ 10019110 f i vJoyInterface.obj
 0002:000081f0       ??1?$_Tree@V?$_Tmap_traits@HW4FFB_EFFECTS@@U?$less@H@std@@V?$allocator@U?$pair@$$CBHW4FFB_EFFECTS@@@std@@@3@$0A@@std@@@std@@QAE@XZ 100191f0 f i vJoyInterface.obj
 0002:000082d0       ??1?$_Tree_const_iterator@V?$_Tree_val@U?$_Tree_simple_types@U?$pair@$$CBHUDeviceStat@@@std@@@std@@@std@@@std@@QAE@XZ 100192d0 f i vJoyInterface.obj
 0002:00008320       ??1?$_Tree_iterator@V?$_Tree_val@U?$_Tree_simple_types@U?$pair@$$CBHUDeviceStat@@@std@@@std@@@std@@@std@@QAE@XZ 10019320 f i vJoyInterface.obj
 0002:00008370       ??1?$_Tree_temp_node@V?$allocator@U?$_Tree_node@U?$pair@$$CBHUDeviceStat@@@std@@PAX@std@@@std@@@std@@QAE@XZ 10019370 f i vJoyInterface.obj
 0002:00008480       ??1?$_Tree_temp_node_alloc@V?$allocator@U?$_Tree_node@U?$pair@$$CBHUDeviceStat@@@std@@PAX@std@@@std@@@std@@QAE@XZ 10019480 f i vJoyInterface.obj
 0002:000084d0       ??1?$_Tree_unchecked_const_iterator@V?$_Tree_val@U?$_Tree_simple_types@U?$pair@$$CBHUDeviceStat@@@std@@@std@@@std@@U_Iterator_base12@2@@std@@QAE@XZ 100194d0 f i vJoyInterface.obj
 0002:00008520       ??1?$map@HUDeviceStat@@U?$less@H@std@@V?$allocator@U?$pair@$$CBHUDeviceStat@@@std@@@3@@std@@QAE@XZ 10019520 f i vJoyInterface.obj
 0002:00008570       ??1?$map@HW4FFB_EFFECTS@@U?$less@H@std@@V?$allocator@U?$pair@$$CBHW4FFB_EFFECTS@@@std@@@3@@std@@QAE@XZ 10019570 f i vJoyInterface.obj
 0002:000085c0       ??1?$pair@V?$_Tree_iterator@V?$_Tree_val@U?$_Tree_simple_types@U?$pair@$$CBHUDeviceStat@@@std@@@std@@@std@@@std@@_N@std@@QAE@XZ 100195c0 f i vJoyInterface.obj
 0002:00008610       ??1_Iterator_base12@std@@QAE@XZ 10019610 f i vJoyInterface.obj
 0002:00008670       ??1bad_alloc@std@@UAE@XZ   10019670 f i vJoyInterface.obj
 0002:000086c0       ??1bad_array_new_length@std@@UAE@XZ 100196c0 f i vJoyInterface.obj
 0002:00008710       ??1exception@std@@UAE@XZ   10019710 f i vJoyInterface.obj
 0002:00008780       ??2@YAPAXIPAX@Z            10019780 f i vJoyInterface.obj
 0002:000087d0       ??4_Iterator_base12@std@@QAEAAU01@ABU01@@Z 100197d0 f i vJoyInterface.obj
 0002:00008840       ??8?$_Tree_const_iterator@V?$_Tree_val@U?$_Tree_simple_types@U?$pair@$$CBHUDeviceStat@@@std@@@std@@@std@@@std@@QBE_NABV01@@Z 10019840 f i vJoyInterface.obj
 0002:00008960       ??8?$_Tree_unchecked_const_iterator@V?$_Tree_val@U?$_Tree_simple_types@U?$pair@$$CBHUDeviceStat@@@std@@@std@@@std@@U_Iterator_base0@2@@std@@QBE_NABV01@@Z 10019960 f i vJoyInterface.obj
 0002:000089f0       ??9?$_Tree_const_iterator@V?$_Tree_val@U?$_Tree_simple_types@U?$pair@$$CBHUDeviceStat@@@std@@@std@@@std@@@std@@QBE_NABV01@@Z 100199f0 f i vJoyInterface.obj
 0002:00008a80       ??9?$_Tree_unchecked_const_iterator@V?$_Tree_val@U?$_Tree_simple_types@U?$pair@$$CBHUDeviceStat@@@std@@@std@@@std@@U_Iterator_base0@2@@std@@QBE_NABV01@@Z 10019a80 f i vJoyInterface.obj
 0002:00008b10       ??A?$map@HUDeviceStat@@U?$less@H@std@@V?$allocator@U?$pair@$$CBHUDeviceStat@@@std@@@3@@std@@QAEAAUDeviceStat@@$$QAH@Z 10019b10 f i vJoyInterface.obj
 0002:00008b90       ??A?$map@HUDeviceStat@@U?$less@H@std@@V?$allocator@U?$pair@$$CBHUDeviceStat@@@std@@@3@@std@@QAEAAUDeviceStat@@ABH@Z 10019b90 f i vJoyInterface.obj
 0002:00008c00       ??E?$_Tree_unchecked_const_iterator@V?$_Tree_val@U?$_Tree_simple_types@U?$pair@$$CBHUDeviceStat@@@std@@@std@@@std@@U_Iterator_base0@2@@std@@QAE?AV01@H@Z 10019c00 f i vJoyInterface.obj
 0002:00008cb0       ??E?$_Tree_unchecked_const_iterator@V?$_Tree_val@U?$_Tree_simple_types@U?$pair@$$CBHUDeviceStat@@@std@@@std@@@std@@U_Iterator_base0@2@@std@@QAEAAV01@XZ 10019cb0 f i vJoyInterface.obj
 0002:00008d80       ??R?$less@H@std@@QBE_NABH0@Z 10019d80 f i vJoyInterface.obj
 0002:00008e10       ??_Ebad_alloc@std@@UAEPAXI@Z 10019e10 f i vJoyInterface.obj
 0002:00008e10       ??_Gbad_alloc@std@@UAEPAXI@Z 10019e10 f i vJoyInterface.obj
 0002:00008e80       ??_Ebad_array_new_length@std@@UAEPAXI@Z 10019e80 f i vJoyInterface.obj
 0002:00008e80       ??_Gbad_array_new_length@std@@UAEPAXI@Z 10019e80 f i vJoyInterface.obj
 0002:00008ef0       ??_Eexception@std@@UAEPAXI@Z 10019ef0 f i vJoyInterface.obj
 0002:00008ef0       ??_Gexception@std@@UAEPAXI@Z 10019ef0 f i vJoyInterface.obj
 0002:00008f60       ?AreControlsInit@@YAHI@Z   10019f60 f   vJoyInterface.obj
 0002:00009160       ?CalcInitValue@@YAXGPAUDEVICE_INIT_VALS@@@Z 1001a160 f   vJoyInterface.obj
 0002:00009540       ?CreateDevicePath@@YA_NPBDHPADH@Z 1001a540 f   vJoyInterface.obj
 0002:00009750       ?CreateDummyWindow@@YGHXZ  1001a750 f   vJoyInterface.obj
 0002:00009a20       ?DbgGetCaps@@YAHXZ         1001aa20 f   vJoyInterface.obj
 0002:0000a290       ?ExtractNamespace@@YA_NPBDPADPAH@Z 1001b290 f   vJoyInterface.obj
 0002:0000a430       ?FfbGetEffectState@@YAHXZ  1001b430 f   vJoyInterface.obj
 0002:0000a590       ?FfbGetEffectType@@YA?AW4FFBEType@@XZ 1001b590 f   vJoyInterface.obj
 0002:0000a630       ?GetAxisCaps@@YAHIIPAU_HIDP_VALUE_CAPS@@@Z 1001b630 f   vJoyInterface.obj
 0002:0000a990       ?GetAxisLogMax@@YAJII@Z    1001b990 f   vJoyInterface.obj
 0002:0000aa70       ?GetAxisLogMid@@YAJII@Z    1001ba70 f   vJoyInterface.obj
 0002:0000ab00       ?GetAxisLogMin@@YAJII@Z    1001bb00 f   vJoyInterface.obj
 0002:0000abe0       ?GetControls@@YAHI@Z       1001bbe0 f   vJoyInterface.obj
 0002:0000b4f0       ?GetDevInfo@@YA_NPAX0@Z    1001c4f0 f   vJoyInterface.obj
 0002:0000b8a0       ?GetDevPosition@@YAHEPAU_JOYSTICK_POSITION_V2@@@Z 1001c8a0 f   vJoyInterface.obj
 0002:0000bc00       ?GetDevStat@@YA_NEPAHPAE@Z 1001cc00 f   vJoyInterface.obj
 0002:0000bfe0       ?GetDeviceAttributes@@YAHHPAG00@Z 1001cfe0 f   vJoyInterface.obj
 0002:0000c140       ?GetDeviceIndexById@@YAHGGH@Z 1001d140 f   vJoyInterface.obj
 0002:0000c380       ?GetDeviceIndexByReportId@@YAHGGE@Z 1001d380 f   vJoyInterface.obj
 0002:0000c530       ?GetDeviceManufacturerString@@YAHHPAPA_W@Z 1001d530 f   vJoyInterface.obj
 0002:0000c6c0       ?GetDeviceNameSpace@@YAHPAPADPAHHPAK@Z 1001d6c0 f   vJoyInterface.obj
 0002:0000ccb0       ?GetDeviceProductString@@YAHHPAPA_W@Z 1001dcb0 f   vJoyInterface.obj
 0002:0000ce10       ?GetDeviceSerialNumberString@@YAHHPAPA_W@Z 1001de10 f   vJoyInterface.obj
 0002:0000cf50       ?GetDeviceVersionNumber@@YAHHPAG@Z 1001df50 f   vJoyInterface.obj
 0002:0000d090       ?GetDrvStat@@YA_NPAHPAE@Z  1001e090 f   vJoyInterface.obj
 0002:0000d420       ?GetGenControlHadle@@YAPAXXZ 1001e420 f   vJoyInterface.obj
 0002:0000d4e0       ?GetHandleByIndex@@YAPAXH@Z 1001e4e0 f   vJoyInterface.obj
 0002:0000d9f0       ?GetInitValueFromRegistry@@YAIGPAUDEVICE_INIT_VALS@@@Z 1001e9f0 f   vJoyInterface.obj
 0002:0000deb0       ?Get_PreparsedData@@YAHHPAPAU_HIDP_PREPARSED_DATA@@@Z 1001eeb0 f   vJoyInterface.obj
 0002:0000e0e0       ?Get_h@@YAPAXH@Z           1001f0e0 f   vJoyInterface.obj
 0002:0000e220       ?Get_hNotify@@YAPAXH@Z     1001f220 f   vJoyInterface.obj
 0002:0000e370       ?Get_stat@@YA?AW4VjdStat@@H@Z 1001f370 f   vJoyInterface.obj
 0002:0000e4c0       ?GetvJoyReportId@@YAHH@Z   1001f4c0 f   vJoyInterface.obj
 0002:0000e910       ?InitDll@@YAXXZ            1001f910 f   vJoyInterface.obj
 0002:0000ead0       ?InitPosition@@YAHH@Z      1001fad0 f   vJoyInterface.obj
 0002:0000f130       ?OpenDeviceInterface@@YAPAXIPAK@Z 10020130 f   vJoyInterface.obj
 0002:0000f470       ?RegisterHandleNotification@@YAPAXPAUHWND__@@PAX@Z 10020470 f   vJoyInterface.obj
 0002:0000f590       ?RegistervJoyNotification@@YAPAXPAUHWND__@@@Z 10020590 f   vJoyInterface.obj
 0002:0000f710       ?SavePosition@@YAXIPAX@Z   10020710 f   vJoyInterface.obj
 0002:0000f920       ?Set_PreparsedData@@YAHH@Z 10020920 f   vJoyInterface.obj
 0002:0000fbc0       ?Set_h@@YAXHPAX@Z          10020bc0 f   vJoyInterface.obj
 0002:0000fd50       ?Set_hNotify@@YAXHPAX@Z    10020d50 f   vJoyInterface.obj
 0002:0000fed0       ?Set_stat@@YAXHW4VjdStat@@@Z 10020ed0 f   vJoyInterface.obj
 0002:00010020       ?StartLogging@@YAXXZ       10021020 f   vJoyInterface.obj
 0002:00010320       ?Sync_Position@@YAXH@Z     10021320 f   vJoyInterface.obj
 0002:000104f0       ?Update@@YAHI@Z            100214f0 f   vJoyInterface.obj
 0002:000108c0       ?WndProc@@YGJPAUHWND__@@IIJ@Z 100218c0 f   vJoyInterface.obj
 0002:00010a70       ?_Adjust_manually_vector_aligned@std@@YAXAAPAXAAI@Z 10021a70 f i vJoyInterface.obj
 0002:00010c40       ?_Adopt@_Iterator_base0@std@@QAEXPBX@Z 10021c40 f i vJoyInterface.obj
 0002:00010c90       ?_Adopt@_Iterator_base12@std@@QAEXPBU_Container_base12@2@@Z 10021c90 f i vJoyInterface.obj
 0002:00010cf0       ?_Adopt_locked@_Iterator_base12@std@@AAEXPBU_Container_base12@2@@Z 10021cf0 f i vJoyInterface.obj
 0002:00010dc0       ?_Adopt_unlocked@_Iterator_base12@std@@AAEXPBU_Container_base12@2@@Z 10021dc0 f i vJoyInterface.obj
 0002:00010e80       ?_Alloc_sentinel_and_proxy@?$_Tree@V?$_Tmap_traits@HUDeviceStat@@U?$less@H@std@@V?$allocator@U?$pair@$$CBHUDeviceStat@@@std@@@3@$0A@@std@@@std@@IAEXXZ 10021e80 f i vJoyInterface.obj
 0002:00010fd0       ?_Alloc_sentinel_and_proxy@?$_Tree@V?$_Tmap_traits@HW4FFB_EFFECTS@@U?$less@H@std@@V?$allocator@U?$pair@$$CBHW4FFB_EFFECTS@@@std@@@3@$0A@@std@@@std@@IAEXXZ 10021fd0 f i vJoyInterface.obj
 0002:00011120       ?_Allocate@?$_Alloc_construct_ptr@V?$allocator@U?$_Tree_node@U?$pair@$$CBHUDeviceStat@@@std@@PAX@std@@@std@@@std@@QAEXXZ 10022120 f i vJoyInterface.obj
 0002:00011190       ?_Allocate@_Default_allocate_traits@std@@SAPAXI@Z 10022190 f i vJoyInterface.obj
 0002:000111f0       ?_Assign_locked@_Iterator_base12@std@@AAEXABU12@@Z 100221f0 f i vJoyInterface.obj
 0002:000112c0       ?_Assign_unlocked@_Iterator_base12@std@@AAEXABU12@@Z 100222c0 f i vJoyInterface.obj
 0002:00011350       ?_Check_grow_by_1@?$_Tree@V?$_Tmap_traits@HUDeviceStat@@U?$less@H@std@@V?$allocator@U?$pair@$$CBHUDeviceStat@@@std@@@3@$0A@@std@@@std@@IAEXXZ 10022350 f i vJoyInterface.obj
 0002:000113c0       ?_Erase@?$_Tree@V?$_Tmap_traits@HUDeviceStat@@U?$less@H@std@@V?$allocator@U?$pair@$$CBHUDeviceStat@@@std@@@3@$0A@@std@@@std@@AAEIU?$pair@PAU?$_Tree_node@U?$pair@$$CBHUDeviceStat@@@std@@PAX@std@@PAU12@@2@@Z 100223c0 f i vJoyInterface.obj
 0002:000114f0       ?_Erase_unchecked@?$_Tree@V?$_Tmap_traits@HUDeviceStat@@U?$less@H@std@@V?$allocator@U?$pair@$$CBHUDeviceStat@@@std@@@3@$0A@@std@@@std@@AAEPAU?$_Tree_node@U?$pair@$$CBHUDeviceStat@@@std@@PAX@2@V?$_Tree_unchecked_const_iterator@V?$_Tree_val@U?$_Tree_simple_types@U?$pair@$$CBHUDeviceStat@@@std@@@std@@@std@@U_Iterator_base0@2@@2@0@Z 100224f0 f i vJoyInterface.obj
 0002:00011600       ?_Erase_unchecked@?$_Tree@V?$_Tmap_traits@HUDeviceStat@@U?$less@H@std@@V?$allocator@U?$pair@$$CBHUDeviceStat@@@std@@@3@$0A@@std@@@std@@AAEPAU?$_Tree_node@U?$pair@$$CBHUDeviceStat@@@std@@PAX@2@V?$_Tree_unchecked_const_iterator@V?$_Tree_val@U?$_Tree_simple_types@U?$pair@$$CBHUDeviceStat@@@std@@@std@@@std@@U_Iterator_base0@2@@2@@Z 10022600 f i vJoyInterface.obj
 0002:000116f0       ?_Extract@?$_In_place_key_extract_map@HHUDeviceStat@@@std@@SAABHABHABUDeviceStat@@@Z 100226f0 f i vJoyInterface.obj
 0002:00011740       ?_Extract@?$_Tree_val@U?$_Tree_simple_types@U?$pair@$$CBHUDeviceStat@@@std@@@std@@@std@@QAEPAU?$_Tree_node@U?$pair@$$CBHUDeviceStat@@@std@@PAX@2@V?$_Tree_unchecked_const_iterator@V?$_Tree_val@U?$_Tree_simple_types@U?$pair@$$CBHUDeviceStat@@@std@@@std@@@std@@U_Iterator_base0@2@@2@@Z 10022740 f i vJoyInterface.obj
 0002:00011cd0       ?_Get_first@?$_Compressed_pair@U?$less@H@std@@V?$_Compressed_pair@V?$allocator@U?$_Tree_node@U?$pair@$$CBHUDeviceStat@@@std@@PAX@std@@@std@@V?$_Tree_val@U?$_Tree_simple_types@U?$pair@$$CBHUDeviceStat@@@std@@@std@@@2@$00@2@$00@std@@QBEABU?$less@H@2@XZ 10022cd0 f i vJoyInterface.obj
 0002:00011d30       ?_Get_first@?$_Compressed_pair@V?$allocator@U?$_Tree_node@U?$pair@$$CBHUDeviceStat@@@std@@PAX@std@@@std@@V?$_Tree_val@U?$_Tree_simple_types@U?$pair@$$CBHUDeviceStat@@@std@@@std@@@2@$00@std@@QAEAAV?$allocator@U?$_Tree_node@U?$pair@$$CBHUDeviceStat@@@std@@PAX@std@@@2@XZ 10022d30 f i vJoyInterface.obj
 0002:00011d90       ?_Get_first@?$_Compressed_pair@V?$allocator@U?$_Tree_node@U?$pair@$$CBHUDeviceStat@@@std@@PAX@std@@@std@@V?$_Tree_val@U?$_Tree_simple_types@U?$pair@$$CBHUDeviceStat@@@std@@@std@@@2@$00@std@@QBEABV?$allocator@U?$_Tree_node@U?$pair@$$CBHUDeviceStat@@@std@@PAX@std@@@2@XZ 10022d90 f i vJoyInterface.obj
 0002:00011df0       ?_Get_first@?$_Compressed_pair@V?$allocator@U?$_Tree_node@U?$pair@$$CBHW4FFB_EFFECTS@@@std@@PAX@std@@@std@@V?$_Tree_val@U?$_Tree_simple_types@U?$pair@$$CBHW4FFB_EFFECTS@@@std@@@std@@@2@$00@std@@QAEAAV?$allocator@U?$_Tree_node@U?$pair@$$CBHW4FFB_EFFECTS@@@std@@PAX@std@@@2@XZ 10022df0 f i vJoyInterface.obj
 0002:00011e50       ?_Get_scary@?$_Tree@V?$_Tmap_traits@HUDeviceStat@@U?$less@H@std@@V?$allocator@U?$pair@$$CBHUDeviceStat@@@std@@@3@$0A@@std@@@std@@IAEPAV?$_Tree_val@U?$_Tree_simple_types@U?$pair@$$CBHUDeviceStat@@@std@@@std@@@2@XZ 10022e50 f i vJoyInterface.obj
 0002:00011eb0       ?_Get_scary@?$_Tree@V?$_Tmap_traits@HUDeviceStat@@U?$less@H@std@@V?$allocator@U?$pair@$$CBHUDeviceStat@@@std@@@3@$0A@@std@@@std@@IBEPBV?$_Tree_val@U?$_Tree_simple_types@U?$pair@$$CBHUDeviceStat@@@std@@@std@@@2@XZ 10022eb0 f i vJoyInterface.obj
 0002:00011f10       ?_Get_scary@?$_Tree@V?$_Tmap_traits@HW4FFB_EFFECTS@@U?$less@H@std@@V?$allocator@U?$pair@$$CBHW4FFB_EFFECTS@@@std@@@3@$0A@@std@@@std@@IAEPAV?$_Tree_val@U?$_Tree_simple_types@U?$pair@$$CBHW4FFB_EFFECTS@@@std@@@std@@@2@XZ 10022f10 f i vJoyInterface.obj
 0002:00011f70       ?_Getal@?$_Tree@V?$_Tmap_traits@HUDeviceStat@@U?$less@H@std@@V?$allocator@U?$pair@$$CBHUDeviceStat@@@std@@@3@$0A@@std@@@std@@IAEAAV?$allocator@U?$_Tree_node@U?$pair@$$CBHUDeviceStat@@@std@@PAX@std@@@2@XZ 10022f70 f i vJoyInterface.obj
 0002:00011fd0       ?_Getal@?$_Tree@V?$_Tmap_traits@HUDeviceStat@@U?$less@H@std@@V?$allocator@U?$pair@$$CBHUDeviceStat@@@std@@@3@$0A@@std@@@std@@IBEABV?$allocator@U?$_Tree_node@U?$pair@$$CBHUDeviceStat@@@std@@PAX@std@@@2@XZ 10022fd0 f i vJoyInterface.obj
 0002:00012030       ?_Getal@?$_Tree@V?$_Tmap_traits@HW4FFB_EFFECTS@@U?$less@H@std@@V?$allocator@U?$pair@$$CBHW4FFB_EFFECTS@@@std@@@3@$0A@@std@@@std@@IAEAAV?$allocator@U?$_Tree_node@U?$pair@$$CBHW4FFB_EFFECTS@@@std@@PAX@std@@@2@XZ 10023030 f i vJoyInterface.obj
 0002:00012090       ?_Getcomp@?$_Tree@V?$_Tmap_traits@HUDeviceStat@@U?$less@H@std@@V?$allocator@U?$pair@$$CBHUDeviceStat@@@std@@@3@$0A@@std@@@std@@IBEABU?$less@H@2@XZ 10023090 f i vJoyInterface.obj
 0002:000120f0       ?_Getcont@_Iterator_base12@std@@QBEPBU_Container_base12@2@XZ 100230f0 f i vJoyInterface.obj
 0002:00012170       ?_Insert_node@?$_Tree_val@U?$_Tree_simple_types@U?$pair@$$CBHUDeviceStat@@@std@@@std@@@std@@QAEPAU?$_Tree_node@U?$pair@$$CBHUDeviceStat@@@std@@PAX@2@U?$_Tree_id@PAU?$_Tree_node@U?$pair@$$CBHUDeviceStat@@@std@@PAX@std@@@2@QAU32@@Z 10023170 f i vJoyInterface.obj
 0002:00012440       ?_Lrotate@?$_Tree_val@U?$_Tree_simple_types@U?$pair@$$CBHUDeviceStat@@@std@@@std@@@std@@QAEXPAU?$_Tree_node@U?$pair@$$CBHUDeviceStat@@@std@@PAX@2@@Z 10023440 f i vJoyInterface.obj
 0002:00012540       ?_Max@?$_Tree_val@U?$_Tree_simple_types@U?$pair@$$CBHUDeviceStat@@@std@@@std@@@std@@SAPAU?$_Tree_node@U?$pair@$$CBHUDeviceStat@@@std@@PAX@2@PAU32@@Z 10023540 f i vJoyInterface.obj
 0002:000125b0       ?_Min@?$_Tree_val@U?$_Tree_simple_types@U?$pair@$$CBHUDeviceStat@@@std@@@std@@@std@@SAPAU?$_Tree_node@U?$pair@$$CBHUDeviceStat@@@std@@PAX@2@PAU32@@Z 100235b0 f i vJoyInterface.obj
 0002:00012620       ?_Orphan_all@_Container_base12@std@@QAEXXZ 10023620 f i vJoyInterface.obj
 0002:00012680       ?_Orphan_all_locked_v3@_Container_base12@std@@AAEXXZ 10023680 f i vJoyInterface.obj
 0002:00012740       ?_Orphan_all_unlocked_v3@_Container_base12@std@@AAEXXZ 10023740 f i vJoyInterface.obj
 0002:000127f0       ?_Orphan_me_locked_v3@_Iterator_base12@std@@AAEXXZ 100237f0 f i vJoyInterface.obj
 0002:000128b0       ?_Orphan_me_unlocked_v3@_Iterator_base12@std@@AAEXXZ 100238b0 f i vJoyInterface.obj
 0002:000129e0       ?_Orphan_ptr@?$_Tree_val@U?$_Tree_simple_types@U?$pair@$$CBHUDeviceStat@@@std@@@std@@@std@@QAEXQAU?$_Tree_node@U?$pair@$$CBHUDeviceStat@@@std@@PAX@2@@Z 100239e0 f i vJoyInterface.obj
 0002:00012b10       ?_Orphan_ptr@?$_Tree_val@U?$_Tree_simple_types@U?$pair@$$CBHW4FFB_EFFECTS@@@std@@@std@@@std@@QAEXQAU?$_Tree_node@U?$pair@$$CBHW4FFB_EFFECTS@@@std@@PAX@2@@Z 10023b10 f i vJoyInterface.obj
 0002:00012c40       ?_Release@?$_Alloc_construct_ptr@V?$allocator@U?$_Tree_node@U?$pair@$$CBHUDeviceStat@@@std@@PAX@std@@@std@@@std@@QAEPAU?$_Tree_node@U?$pair@$$CBHUDeviceStat@@@std@@PAX@2@XZ 10023c40 f i vJoyInterface.obj
 0002:00012cc0       ?_Release@_Basic_container_proxy_ptr12@std@@QAEXXZ 10023cc0 f i vJoyInterface.obj
 0002:00012d20       ?_Rrotate@?$_Tree_val@U?$_Tree_simple_types@U?$pair@$$CBHUDeviceStat@@@std@@@std@@@std@@QAEXPAU?$_Tree_node@U?$pair@$$CBHUDeviceStat@@@std@@PAX@2@@Z 10023d20 f i vJoyInterface.obj
 0002:00012e30       ?_Throw_bad_array_new_length@std@@YAXXZ 10023e30 f i vJoyInterface.obj
 0002:00012ea0       ?_Throw_tree_length_error@std@@YAXXZ 10023ea0 f i vJoyInterface.obj
 0002:00012ef0       ?_Unchecked_begin@?$_Tree@V?$_Tmap_traits@HUDeviceStat@@U?$less@H@std@@V?$allocator@U?$pair@$$CBHUDeviceStat@@@std@@@3@$0A@@std@@@std@@QAE?AV?$_Tree_unchecked_iterator@V?$_Tree_val@U?$_Tree_simple_types@U?$pair@$$CBHUDeviceStat@@@std@@@std@@@std@@@2@XZ 10023ef0 f i vJoyInterface.obj
 0002:00012f70       ?allocate@?$allocator@U?$_Tree_node@U?$pair@$$CBHUDeviceStat@@@std@@PAX@std@@@std@@QAEPAU?$_Tree_node@U?$pair@$$CBHUDeviceStat@@@std@@PAX@2@I@Z 10023f70 f i vJoyInterface.obj
 0002:00012fe0       ?allocate@?$allocator@U?$_Tree_node@U?$pair@$$CBHW4FFB_EFFECTS@@@std@@PAX@std@@@std@@QAEPAU?$_Tree_node@U?$pair@$$CBHW4FFB_EFFECTS@@@std@@PAX@2@I@Z 10023fe0 f i vJoyInterface.obj
 0002:00013050       ?allocate@?$allocator@U_Container_proxy@std@@@std@@QAEPAU_Container_proxy@2@I@Z 10024050 f i vJoyInterface.obj
 0002:000130c0       ?clear@?$_Tree@V?$_Tmap_traits@HUDeviceStat@@U?$less@H@std@@V?$allocator@U?$pair@$$CBHUDeviceStat@@@std@@@3@$0A@@std@@@std@@QAEXXZ 100240c0 f i vJoyInterface.obj
 0002:00013180       ?clear@?$_Tree@V?$_Tmap_traits@HW4FFB_EFFECTS@@U?$less@H@std@@V?$allocator@U?$pair@$$CBHW4FFB_EFFECTS@@@std@@@3@$0A@@std@@@std@@QAEXXZ 10024180 f i vJoyInterface.obj
 0002:00013240       ?deallocate@?$_Default_allocator_traits@V?$allocator@U?$_Tree_node@U?$pair@$$CBHUDeviceStat@@@std@@PAX@std@@@std@@@std@@SAXAAV?$allocator@U?$_Tree_node@U?$pair@$$CBHUDeviceStat@@@std@@PAX@std@@@2@QAU?$_Tree_node@U?$pair@$$CBHUDeviceStat@@@std@@PAX@2@I@Z 10024240 f i vJoyInterface.obj
 0002:000132a0       ?deallocate@?$_Default_allocator_traits@V?$allocator@U?$_Tree_node@U?$pair@$$CBHW4FFB_EFFECTS@@@std@@PAX@std@@@std@@@std@@SAXAAV?$allocator@U?$_Tree_node@U?$pair@$$CBHW4FFB_EFFECTS@@@std@@PAX@std@@@2@QAU?$_Tree_node@U?$pair@$$CBHW4FFB_EFFECTS@@@std@@PAX@2@I@Z 100242a0 f i vJoyInterface.obj
 0002:00013300       ?deallocate@?$_Default_allocator_traits@V?$allocator@U_Container_proxy@std@@@std@@@std@@SAXAAV?$allocator@U_Container_proxy@std@@@2@QAU_Container_proxy@2@I@Z 10024300 f i vJoyInterface.obj
 0002:00013360       ?deallocate@?$allocator@U?$_Tree_node@U?$pair@$$CBHUDeviceStat@@@std@@PAX@std@@@std@@QAEXQAU?$_Tree_node@U?$pair@$$CBHUDeviceStat@@@std@@PAX@2@I@Z 10024360 f i vJoyInterface.obj
 0002:00013460       ?empty@?$_Tree@V?$_Tmap_traits@HUDeviceStat@@U?$less@H@std@@V?$allocator@U?$pair@$$CBHUDeviceStat@@@std@@@3@$0A@@std@@@std@@QBE_NXZ 10024460 f i vJoyInterface.obj
 0002:000134f0       ?end@?$_Tree@V?$_Tmap_traits@HUDeviceStat@@U?$less@H@std@@V?$allocator@U?$pair@$$CBHUDeviceStat@@@std@@@3@$0A@@std@@@std@@QAE?AV?$_Tree_iterator@V?$_Tree_val@U?$_Tree_simple_types@U?$pair@$$CBHUDeviceStat@@@std@@@std@@@std@@@2@XZ 100244f0 f i vJoyInterface.obj
 0002:00013570       ?erase@?$_Tree@V?$_Tmap_traits@HUDeviceStat@@U?$less@H@std@@V?$allocator@U?$pair@$$CBHUDeviceStat@@@std@@@3@$0A@@std@@@std@@QAEIABH@Z 10024570 f i vJoyInterface.obj
 0002:000135f0       ?find@?$_Tree@V?$_Tmap_traits@HUDeviceStat@@U?$less@H@std@@V?$allocator@U?$pair@$$CBHUDeviceStat@@@std@@@3@$0A@@std@@@std@@QAE?AV?$_Tree_iterator@V?$_Tree_val@U?$_Tree_simple_types@U?$pair@$$CBHUDeviceStat@@@std@@@std@@@std@@@2@ABH@Z 100245f0 f i vJoyInterface.obj
 0002:00013690       ?isRawDevice@@YA_NPBDH@Z   10024690 f   vJoyInterface.obj
 0002:00013920       ?max@?$numeric_limits@H@std@@SAHXZ 10024920 f i vJoyInterface.obj
 0002:00013970       ?max_size@?$_Default_allocator_traits@V?$allocator@U?$_Tree_node@U?$pair@$$CBHUDeviceStat@@@std@@PAX@std@@@std@@@std@@SAIABV?$allocator@U?$_Tree_node@U?$pair@$$CBHUDeviceStat@@@std@@PAX@std@@@2@@Z 10024970 f i vJoyInterface.obj
 0002:000139c0       ?max_size@?$_Tree@V?$_Tmap_traits@HUDeviceStat@@U?$less@H@std@@V?$allocator@U?$pair@$$CBHUDeviceStat@@@std@@@3@$0A@@std@@@std@@QBEIXZ 100249c0 f i vJoyInterface.obj
 0002:00013a60       ?size@?$_Tree@V?$_Tmap_traits@HUDeviceStat@@U?$less@H@std@@V?$allocator@U?$pair@$$CBHUDeviceStat@@@std@@@3@$0A@@std@@@std@@QBEIXZ 10024a60 f i vJoyInterface.obj
 0002:00013ac0       ?strstr@@YAPADQADQBD@Z     10024ac0 f i vJoyInterface.obj
 0002:00013b20       ?vJoyDeviceClear@@YAXXZ    10024b20 f   vJoyInterface.obj
 0002:00013b70       ?vJoyDeviceEntry@@YAHH@Z   10024b70 f   vJoyInterface.obj
 0002:00013db0       ?vJoyDeviceRemove@@YAHH@Z  10024db0 f   vJoyInterface.obj
 0002:00013fd0       ?what@exception@std@@UBEPBDXZ 10024fd0 f i vJoyInterface.obj
 0002:00014050       _AcquireVJD                10025050 f   vJoyInterface.obj
 0002:000141d0       _DeviceChange              100251d0 f   vJoyInterface.obj
 0002:00014440       _DriverMatch               10025440 f   vJoyInterface.obj
 0002:00014500       _FfbGetEffect              10025500 f   vJoyInterface.obj
 0002:00014560       _FfbIsStarted              10025560 f   vJoyInterface.obj
 0002:000148d0       _FfbProcessData            100258d0 f   vJoyInterface.obj
 0002:00014940       _FfbRegisterGenCB          10025940 f   vJoyInterface.obj
 0002:000149a0       _FfbSendData               100259a0 f   vJoyInterface.obj
 0002:00014aa0       _FfbStart                  10025aa0 f   vJoyInterface.obj
 0002:00014b30       _FfbStartThread            10025b30 f   vJoyInterface.obj
 0002:00014c90       _FfbStop                   10025c90 f   vJoyInterface.obj
 0002:00014ce0       _FfbWaitForData@4          10025ce0 f   vJoyInterface.obj
 0002:00015110       _Ffb_h_DevCtrl             10026110 f   vJoyInterface.obj
 0002:00015210       _Ffb_h_DevGain             10026210 f   vJoyInterface.obj
 0002:00015310       _Ffb_h_DeviceID            10026310 f   vJoyInterface.obj
 0002:000153c0       _Ffb_h_EBI                 100263c0 f   vJoyInterface.obj
 0002:000154d0       _Ffb_h_EffNew              100264d0 f   vJoyInterface.obj
 0002:000155d0       _Ffb_h_EffOp               100265d0 f   vJoyInterface.obj
 0002:00015700       _Ffb_h_Eff_Cond            10026700 f   vJoyInterface.obj
 0002:00015980       _Ffb_h_Eff_Constant        10026980 f   vJoyInterface.obj
 0002:00015ab0       _Ffb_h_Eff_Envlp           10026ab0 f   vJoyInterface.obj
 0002:00015d10       _Ffb_h_Eff_Period          10026d10 f   vJoyInterface.obj
 0002:00015f40       _Ffb_h_Eff_Ramp            10026f40 f   vJoyInterface.obj
 0002:000160b0       _Ffb_h_Eff_Report          100270b0 f   vJoyInterface.obj
 0002:00016370       _Ffb_h_Packet              10027370 f   vJoyInterface.obj
 0002:00016410       _Ffb_h_Type                10027410 f   vJoyInterface.obj
 0002:000164c0       _GetNumberExistingVJD      100274c0 f   vJoyInterface.obj
 0002:000165f0       _GetOwnerPid               100275f0 f   vJoyInterface.obj
 0002:000167f0       _GetVJDAxisExist           100277f0 f   vJoyInterface.obj
 0002:00016af0       _GetVJDAxisMax             10027af0 f   vJoyInterface.obj
 0002:00016bc0       _GetVJDAxisMin             10027bc0 f   vJoyInterface.obj
 0002:00016c90       _GetVJDButtonNumber        10027c90 f   vJoyInterface.obj
 0002:00017440       _GetVJDContPovNumber       10028440 f   vJoyInterface.obj
 0002:000177b0       _GetVJDDiscPovNumber       100287b0 f   vJoyInterface.obj
 0002:00017b30       _GetVJDStatus              10028b30 f   vJoyInterface.obj
 0002:00017e00       _GetvJoyManufacturerString 10028e00 f   vJoyInterface.obj
 0002:00017ef0       _GetvJoyMaxDevices         10028ef0 f   vJoyInterface.obj
 0002:00018020       _GetvJoyProductString      10029020 f   vJoyInterface.obj
 0002:00018110       _GetvJoySerialNumberString 10029110 f   vJoyInterface.obj
 0002:00018200       _GetvJoyVersion            10029200 f   vJoyInterface.obj
 0002:000182f0       _IsDeviceFfb               100292f0 f   vJoyInterface.obj
 0002:00018630       _IsDeviceFfbEffect         10029630 f   vJoyInterface.obj
 0002:000189e0       _RegisterRemovalCB         100299e0 f   vJoyInterface.obj
 0002:00018a40       _RelinquishVJD             10029a40 f   vJoyInterface.obj
 0002:00018af0       _ResetAll                  10029af0 f   vJoyInterface.obj
 0002:00018b40       _ResetButtons              10029b40 f   vJoyInterface.obj
 0002:00018d30       _ResetPovs                 10029d30 f   vJoyInterface.obj
 0002:000190a0       _ResetVJD                  1002a0a0 f   vJoyInterface.obj
 0002:00019380       _RtlSecureZeroMemory       1002a380 f i vJoyInterface.obj
 0002:00019400       _SetAxis                   1002a400 f   vJoyInterface.obj
 0002:000196b0       _SetBtn                    1002a6b0 f   vJoyInterface.obj
 0002:00019900       _SetContPov                1002a900 f   vJoyInterface.obj
 0002:00019b40       _SetDiscPov                1002ab40 f   vJoyInterface.obj
 0002:00019cc0       _UpdateVJD                 1002acc0 f   vJoyInterface.obj
 0002:00019d30       ___local_stdio_printf_options 1002ad30 f i vJoyInterface.obj
 0002:00019d80       ___local_stdio_scanf_options 1002ad80 f i vJoyInterface.obj
 0002:00019dd0       __vfprintf_s_l             1002add0 f i vJoyInterface.obj
 0002:00019e50       __vsprintf_s_l             1002ae50 f i vJoyInterface.obj
 0002:00019f10       __vsscanf_s_l              1002af10 f i vJoyInterface.obj
 0002:00019fa0       __vswprintf_s_l            1002afa0 f i vJoyInterface.obj
 0002:0001a060       _fprintf_s                 1002b060 f i vJoyInterface.obj
 0002:0001a0e0       _isVJDExists               1002b0e0 f   vJoyInterface.obj
 0002:0001a240       _isVJDOpen                 1002b240 f   vJoyInterface.obj
 0002:0001a310       _sprintf_s                 1002b310 f i vJoyInterface.obj
 0002:0001a390       _sscanf_s                  1002b390 f i vJoyInterface.obj
 0002:0001a410       _swprintf_s                1002b410 f i vJoyInterface.obj
 0002:0001a490       _vJoyEnabled               1002b490 f   vJoyInterface.obj
 0002:0001a560       _vJoyFfbCap                1002b560 f   vJoyInterface.obj
 0002:0001a690       _vsscanf_s                 1002b690 f i vJoyInterface.obj
 0002:0001a6ed       _SetupDiDestroyDeviceInfoList@4 1002b6ed f   setupapi:SETUPAPI.dll
 0002:0001a6f3       _SetupDiEnumDeviceInterfaces@20 1002b6f3 f   setupapi:SETUPAPI.dll
 0002:0001a6f9       _SetupDiGetDeviceInterfaceDetailA@24 1002b6f9 f   setupapi:SETUPAPI.dll
 0002:0001a6ff       _SetupDiGetClassDevsA@16   1002b6ff f   setupapi:SETUPAPI.dll
 0002:0001a705       _HidP_GetCaps@8            1002b705 f   hid:HID.DLL
 0002:0001a70b       _HidP_GetLinkCollectionNodes@12 1002b70b f   hid:HID.DLL
 0002:0001a711       _HidP_GetButtonCaps@16     1002b711 f   hid:HID.DLL
 0002:0001a717       _HidP_GetSpecificValueCaps@28 1002b717 f   hid:HID.DLL
 0002:0001a71d       _HidP_GetValueCaps@16      1002b71d f   hid:HID.DLL
 0002:0001a723       _HidP_GetUsageValue@32     1002b723 f   hid:HID.DLL
 0002:0001a729       _HidD_GetAttributes@8      1002b729 f   hid:HID.DLL
 0002:0001a72f       _HidD_GetHidGuid@4         1002b72f f   hid:HID.DLL
 0002:0001a735       _HidD_GetPreparsedData@8   1002b735 f   hid:HID.DLL
 0002:0001a73b       _HidD_FreePreparsedData@4  1002b73b f   hid:HID.DLL
 0002:0001a741       _HidD_GetManufacturerString@12 1002b741 f   hid:HID.DLL
 0002:0001a747       _HidD_GetProductString@12  1002b747 f   hid:HID.DLL
 0002:0001a74d       _HidD_GetSerialNumberString@12 1002b74d f   hid:HID.DLL
 0002:0001a753       _GetCommandLineA@0         1002b753 f   kernel32:KERNEL32.dll
 0002:0001a759       _GetEnvironmentVariableA@12 1002b759 f   kernel32:KERNEL32.dll
 0002:0001a75f       _CreateFileA@28            1002b75f f   kernel32:KERNEL32.dll
 0002:0001a765       _CloseHandle@4             1002b765 f   kernel32:KERNEL32.dll
 0002:0001a76b       _GetLastError@0            1002b76b f   kernel32:KERNEL32.dll
 0002:0001a771       _DeviceIoControl@32        1002b771 f   kernel32:KERNEL32.dll
 0002:0001a777       _GetOverlappedResult@16    1002b777 f   kernel32:KERNEL32.dll
 0002:0001a77d       _SetEvent@4                1002b77d f   kernel32:KERNEL32.dll
 0002:0001a783       _WaitForSingleObject@8     1002b783 f   kernel32:KERNEL32.dll
 0002:0001a789       _CreateEventA@16           1002b789 f   kernel32:KERNEL32.dll
 0002:0001a78f       _GetCurrentProcessId@0     1002b78f f   kernel32:KERNEL32.dll
 0002:0001a795       _CreateThread@24           1002b795 f   kernel32:KERNEL32.dll
 0002:0001a79b       _GetModuleHandleA@4        1002b79b f   kernel32:KERNEL32.dll
 0002:0001a7a1       _LocalAlloc@8              1002b7a1 f   kernel32:KERNEL32.dll
 0002:0001a7a7       _LocalFree@4               1002b7a7 f   kernel32:KERNEL32.dll
 0002:0001a7ad       _GetMessageA@16            1002b7ad f   user32:USER32.dll
 0002:0001a7b3       _TranslateMessage@4        1002b7b3 f   user32:USER32.dll
 0002:0001a7b9       _DispatchMessageA@4        1002b7b9 f   user32:USER32.dll
 0002:0001a7bf       _SendMessageA@16           1002b7bf f   user32:USER32.dll
 0002:0001a7c5       _RegisterDeviceNotificationA@12 1002b7c5 f   user32:USER32.dll
 0002:0001a7cb       _UnregisterDeviceNotification@4 1002b7cb f   user32:USER32.dll
 0002:0001a7d1       _DefWindowProcA@16         1002b7d1 f   user32:USER32.dll
 0002:0001a7d7       _PostQuitMessage@4         1002b7d7 f   user32:USER32.dll
 0002:0001a7dd       _RegisterClassExA@4        1002b7dd f   user32:USER32.dll
 0002:0001a7e3       _CreateWindowExA@48        1002b7e3 f   user32:USER32.dll
 0002:0001a7e9       _ShowWindow@8              1002b7e9 f   user32:USER32.dll
 0002:0001a7ef       _UpdateWindow@4            1002b7ef f   user32:USER32.dll
 0002:0001a7f5       _BeginPaint@8              1002b7f5 f   user32:USER32.dll
 0002:0001a7fb       _EndPaint@8                1002b7fb f   user32:USER32.dll
 0002:0001a801       _MessageBoxA@16            1002b801 f   user32:USER32.dll
 0002:0001a807       _LoadCursorA@8             1002b807 f   user32:USER32.dll
 0002:0001a80d       _LoadIconA@8               1002b80d f   user32:USER32.dll
 0002:0001a813       _RegCloseKey@4             1002b813 f   advapi32:ADVAPI32.dll
 0002:0001a819       _RegOpenKeyExW@20          1002b819 f   advapi32:ADVAPI32.dll
 0002:0001a81f       _RegGetValueW@28           1002b81f f   advapi32:ADVAPI32.dll
 0002:0001a825       ??0_Lockit@std@@QAE@H@Z    1002b825 f   msvcprtd:MSVCP140D.dll
 0002:0001a82b       ??1_Lockit@std@@QAE@XZ     1002b82b f   msvcprtd:MSVCP140D.dll
 0002:0001a831       ?_Xlength_error@std@@YAXPBD@Z 1002b831 f   msvcprtd:MSVCP140D.dll
 0002:0001a840       ??2@YAPAXI@Z               1002b840 f   MSVCRTD:new_scalar.obj
 0002:0001a8a0       ??3@YAXPAXI@Z              1002b8a0 f   MSVCRTD:delete_scalar_size.obj
 0002:0001a8c0       ??_U@YAPAXI@Z              1002b8c0 f   MSVCRTD:new_array.obj
 0002:0001a8e0       ??_V@YAXPAX@Z              1002b8e0 f   MSVCRTD:delete_array.obj
 0002:0001a900       ?configure_argv@__scrt_narrow_argv_policy@@SAHXZ 1002b900 f i MSVCRTD:utility.obj
 0002:0001a9d0       ?initialize_environment@__scrt_narrow_environment_policy@@SAHXZ 1002b9d0 f i MSVCRTD:utility.obj
 0002:0001aa70       _NtCurrentTeb              1002ba70 f i MSVCRTD:utility.obj
 0002:0001aa80       ___scrt_acquire_startup_lock 1002ba80 f   MSVCRTD:utility.obj
 0002:0001aae0       ___scrt_dllmain_after_initialize_c 1002bae0 f   MSVCRTD:utility.obj
 0002:0001ab20       ___scrt_dllmain_before_initialize_c 1002bb20 f   MSVCRTD:utility.obj
 0002:0001ab50       ___scrt_dllmain_crt_thread_attach 1002bb50 f   MSVCRTD:utility.obj
 0002:0001ab90       ___scrt_dllmain_crt_thread_detach 1002bb90 f   MSVCRTD:utility.obj
 0002:0001abb0       ___scrt_dllmain_exception_filter 1002bbb0 f   MSVCRTD:utility.obj
 0002:0001ac10       ___scrt_dllmain_uninitialize_c 1002bc10 f   MSVCRTD:utility.obj
 0002:0001ac50       ___scrt_dllmain_uninitialize_critical 1002bc50 f   MSVCRTD:utility.obj
 0002:0001ac70       ___scrt_initialize_crt     1002bc70 f   MSVCRTD:utility.obj
 0002:0001acd0       ___scrt_initialize_onexit_tables 1002bcd0 f   MSVCRTD:utility.obj
 0002:0001ade0       ___scrt_is_nonwritable_in_current_image 1002bde0 f   MSVCRTD:utility.obj
 0002:0001af60       ___scrt_release_startup_lock 1002bf60 f   MSVCRTD:utility.obj
 0002:0001af90       ___scrt_uninitialize_crt   1002bf90 f   MSVCRTD:utility.obj
 0002:0001afe0       __onexit                   1002bfe0 f   MSVCRTD:utility.obj
 0002:0001b060       _at_quick_exit             1002c060 f   MSVCRTD:utility.obj
 0002:0001b0b0       _atexit                    1002c0b0 f   MSVCRTD:utility.obj
 0002:0001b0f0       @_RTC_AllocaHelper@12      1002c0f0 f   MSVCRTD:stack.obj
 0002:0001b130       @_RTC_CheckStackVars2@12   1002c130 f   MSVCRTD:stack.obj
 0002:0001b240       @_RTC_CheckStackVars@8     1002c240 f   MSVCRTD:stack.obj
 0002:0001b2b0       __RTC_CheckEsp             1002c2b0 f   MSVCRTD:stack.obj
 0002:0001b2e0       @__CheckForDebuggerJustMyCode@4 1002c2e0 f   MSVCRTD:debugger_jmc.obj
 0002:0001b330       @__security_check_cookie@4 1002c330 f   MSVCRTD:secchk.obj
 0002:0001b350       __CRT_RTC_INIT             1002c350 f   MSVCRTD:init.obj
 0002:0001b360       __CRT_RTC_INITW            1002c360 f   MSVCRTD:init.obj
 0002:0001b370       __RTC_InitBase             1002c370 f   MSVCRTD:init.obj
 0002:0001b3b0       __RTC_Shutdown             1002c3b0 f   MSVCRTD:init.obj
 0002:0001b3d0       __alloca_probe             1002c3d0 f   MSVCRTD:chkstk.obj
 0002:0001b3d0       __chkstk                   1002c3d0 f   MSVCRTD:chkstk.obj
 0002:0001b410       ??1type_info@@UAE@XZ       1002c410 f   MSVCRTD:std_type_info_static.obj
 0002:0001b430       ??_Etype_info@@UAEPAXI@Z   1002c430 f i MSVCRTD:std_type_info_static.obj
 0002:0001b430       ??_Gtype_info@@UAEPAXI@Z   1002c430 f i MSVCRTD:std_type_info_static.obj
 0002:0001ba70       __CRT_INIT@12              1002ca70 f   MSVCRTD:dll_dllmain.obj
 0002:0001ba90       __DllMainCRTStartup@12     1002ca90 f   MSVCRTD:dll_dllmain.obj
 0002:0001bac0       ??0bad_alloc@std@@QAE@XZ   1002cac0 f i MSVCRTD:throw_bad_alloc.obj
 0002:0001baf0       ?__scrt_throw_std_bad_alloc@@YAXXZ 1002caf0 f   MSVCRTD:throw_bad_alloc.obj
 0002:0001bb20       ?__scrt_throw_std_bad_array_new_length@@YAXXZ 1002cb20 f   MSVCRTD:throw_bad_alloc.obj
 0002:0001bb50       ??3@YAXPAX@Z               1002cb50 f   MSVCRTD:delete_scalar.obj
 0002:0001bb70       ___isa_available_init      1002cb70 f   MSVCRTD:cpu_disp.obj
 0002:0001bf70       __get_startup_argv_mode    1002cf70 f   MSVCRTD:argv_mode.obj
 0002:0001bf80       ___scrt_is_ucrt_dll_in_use 1002cf80 f   MSVCRTD:ucrt_detection.obj
 0002:0001bfb0       ___scrt_fastfail           1002cfb0 f   MSVCRTD:utility_desktop.obj
 0002:0001c140       ___scrt_get_show_window_mode 1002d140 f   MSVCRTD:utility_desktop.obj
 0002:0001c190       ___scrt_initialize_mta     1002d190 f   MSVCRTD:utility_desktop.obj
 0002:0001c1a0       ___scrt_initialize_winrt   1002d1a0 f   MSVCRTD:utility_desktop.obj
 0002:0001c1b0       ___scrt_is_managed_app     1002d1b0 f   MSVCRTD:utility_desktop.obj
 0002:0001c260       ___scrt_set_unhandled_exception_filter 1002d260 f   MSVCRTD:utility_desktop.obj
 0002:0001c280       ___scrt_exe_initialize_mta 1002d280 f   MSVCRTD:utility_desktop.obj
 0002:0001c280       ___scrt_stub_for_initialize_mta 1002d280 f   MSVCRTD:utility_desktop.obj
 0002:0001c290       ___scrt_unhandled_exception_filter@4 1002d290 f   MSVCRTD:utility_desktop.obj
 0002:0001c330       __crt_debugger_hook        1002d330 f   MSVCRTD:utility_desktop.obj
 0002:0001c350       __except_handler4          1002d350 f   MSVCRTD:chandler4gs.obj
 0002:0001c3a0       @_guard_check_icall_nop@4  1002d3a0 f i MSVCRTD:guard_support.obj
 0002:0001c3b0       _ReadNoFence               1002d3b0 f i MSVCRTD:guard_support.obj
 0002:0001c3d0       _ReadPointerNoFence        1002d3d0 f i MSVCRTD:guard_support.obj
 0002:0001c3f0       ___castguard_check_failure_debugbreak 1002d3f0 f i MSVCRTD:guard_support.obj
 0002:0001c410       ___castguard_check_failure_fastfail 1002d410 f i MSVCRTD:guard_support.obj
 0002:0001c440       ___castguard_check_failure_nop 1002d440 f i MSVCRTD:guard_support.obj
 0002:0001c450       ___castguard_check_failure_os_handled 1002d450 f i MSVCRTD:guard_support.obj
 0002:0001c500       ___castguard_slow_path_check_debugbreak 1002d500 f i MSVCRTD:guard_support.obj
 0002:0001c540       ___castguard_slow_path_check_fastfail 1002d540 f i MSVCRTD:guard_support.obj
 0002:0001c590       ___castguard_slow_path_check_nop 1002d590 f i MSVCRTD:guard_support.obj
 0002:0001c5a0       ___castguard_slow_path_check_os_handled 1002d5a0 f i MSVCRTD:guard_support.obj
 0002:0001c640       __guard_icall_checks_enforced 1002d640 f i MSVCRTD:guard_support.obj
 0002:0001c730       ?_RTC_AllocaFailure@@YAXPAXPAU_RTC_ALLOCA_NODE@@H@Z 1002d730 f   MSVCRTD:error.obj
 0002:0001c850       ?_RTC_Failure@@YAXPAXH@Z   1002d850 f   MSVCRTD:error.obj
 0002:0001c8c0       ?_RTC_StackFailure@@YAXPAXPBD@Z 1002d8c0 f   MSVCRTD:error.obj
 0002:0001cd70       __RTC_UninitUse            1002dd70 f   MSVCRTD:error.obj
 0002:0001ce50       ___raise_securityfailure   1002de50 f   MSVCRTD:gs_report.obj
 0002:0001ce90       ___report_gsfailure        1002de90 f   MSVCRTD:gs_report.obj
 0002:0001cfe0       ___report_rangecheckfailure 1002dfe0 f   MSVCRTD:gs_report.obj
 0002:0001cff0       ___report_securityfailure  1002dff0 f   MSVCRTD:gs_report.obj
 0002:0001d100       ___report_securityfailureEx 1002e100 f   MSVCRTD:gs_report.obj
 0002:0001d270       ?_RTC_GetErrorFunc@@YAP6AHHPBDH00ZZPBX@Z 1002e270 f   MSVCRTD:userapi.obj
 0002:0001d280       ?_RTC_GetErrorFuncW@@YAP6AHHPB_WH00ZZPBX@Z 1002e280 f   MSVCRTD:userapi.obj
 0002:0001d290       __RTC_GetErrDesc           1002e290 f   MSVCRTD:userapi.obj
 0002:0001d2b0       __RTC_NumErrors            1002e2b0 f   MSVCRTD:userapi.obj
 0002:0001d2c0       __RTC_SetErrorFunc         1002e2c0 f   MSVCRTD:userapi.obj
 0002:0001d2f0       __RTC_SetErrorFuncW        1002e2f0 f   MSVCRTD:userapi.obj
 0002:0001d320       __RTC_SetErrorType         1002e320 f   MSVCRTD:userapi.obj
 0002:0001d3e0       ___security_init_cookie    1002e3e0 f   MSVCRTD:gs_support.obj
 0002:0001d480       _DllMain@12                1002e480 f   MSVCRTD:dll_dllmain_stub.obj
 0002:0001d4b0       ?__scrt_initialize_type_info@@YAXXZ 1002e4b0 f   MSVCRTD:tncleanup.obj
 0002:0001d4d0       ?__scrt_uninitialize_type_info@@YAXXZ 1002e4d0 f   MSVCRTD:tncleanup.obj
 0002:0001d4f0       ___scrt_initialize_default_local_stdio_options 1002e4f0 f   MSVCRTD:default_local_stdio_options.obj
 0002:0001d540       ___scrt_get_dyn_tls_init_callback 1002e540 f   MSVCRTD:dyn_tls_init.obj
 0002:0001d550       __RTC_Initialize           1002e550 f   MSVCRTD:initsect.obj
 0002:0001d590       __RTC_Terminate            1002e590 f   MSVCRTD:initsect.obj
 0002:0001db70       ?_RTC_GetSrcLine@@YAHPAEPA_WKPAH1K@Z 1002eb70 f   MSVCRTD:pdblkup.obj
 0002:0001dfd0       __except_handler4_noexcept 1002efd0 f   MSVCRTD:chandler4_noexcept.obj
 0002:0001e041       _memcpy                    1002f041 f   vcruntimed:VCRUNTIME140D.dll
 0002:0001e047       _memset                    1002f047 f   vcruntimed:VCRUNTIME140D.dll
 0002:0001e04d       _strrchr                   1002f04d f   vcruntimed:VCRUNTIME140D.dll
 0002:0001e053       _strstr                    1002f053 f   vcruntimed:VCRUNTIME140D.dll
 0002:0001e059       ___std_exception_copy      1002f059 f   vcruntimed:VCRUNTIME140D.dll
 0002:0001e05f       ___std_exception_destroy   1002f05f f   vcruntimed:VCRUNTIME140D.dll
 0002:0001e065       __CxxThrowException@8      1002f065 f   vcruntimed:VCRUNTIME140D.dll
 0002:0001e06b       ___CxxFrameHandler3        1002f06b f   vcruntimed:VCRUNTIME140D.dll
 0002:0001e071       ___current_exception       1002f071 f   vcruntimed:VCRUNTIME140D.dll
 0002:0001e077       ___current_exception_context 1002f077 f   vcruntimed:VCRUNTIME140D.dll
 0002:0001e07d       __except_handler4_common   1002f07d f   vcruntimed:VCRUNTIME140D.dll
 0002:0001e083       ___std_type_info_destroy_list 1002f083 f   vcruntimed:VCRUNTIME140D.dll
 0002:0001e089       ___vcrt_GetModuleFileNameW 1002f089 f   vcruntimed:VCRUNTIME140D.dll
 0002:0001e08f       ___vcrt_GetModuleHandleW   1002f08f f   vcruntimed:VCRUNTIME140D.dll
 0002:0001e095       ___vcrt_LoadLibraryExW     1002f095 f   vcruntimed:VCRUNTIME140D.dll
 0002:0001e09b       __invalid_parameter        1002f09b f   ucrtd:ucrtbased.dll
 0002:0001e0a1       __wcsdup                   1002f0a1 f   ucrtd:ucrtbased.dll
 0002:0001e0a7       _wcslen                    1002f0a7 f   ucrtd:ucrtbased.dll
 0002:0001e0ad       __strdup                   1002f0ad f   ucrtd:ucrtbased.dll
 0002:0001e0b3       _strlen                    1002f0b3 f   ucrtd:ucrtbased.dll
 0002:0001e0b9       __strlwr_s                 1002f0b9 f   ucrtd:ucrtbased.dll
 0002:0001e0bf       _strncpy                   1002f0bf f   ucrtd:ucrtbased.dll
 0002:0001e0c5       _calloc                    1002f0c5 f   ucrtd:ucrtbased.dll
 0002:0001e0cb       _free                      1002f0cb f   ucrtd:ucrtbased.dll
 0002:0001e0d1       _atoi                      1002f0d1 f   ucrtd:ucrtbased.dll
 0002:0001e0d7       _wcstombs                  1002f0d7 f   ucrtd:ucrtbased.dll
 0002:0001e0dd       ___stdio_common_vswprintf_s 1002f0dd f   ucrtd:ucrtbased.dll
 0002:0001e0e3       _fopen_s                   1002f0e3 f   ucrtd:ucrtbased.dll
 0002:0001e0e9       ___stdio_common_vfprintf_s 1002f0e9 f   ucrtd:ucrtbased.dll
 0002:0001e0ef       ___stdio_common_vsprintf_s 1002f0ef f   ucrtd:ucrtbased.dll
 0002:0001e0f5       ___stdio_common_vsscanf    1002f0f5 f   ucrtd:ucrtbased.dll
 0002:0001e0fb       __CrtDbgReport             1002f0fb f   ucrtd:ucrtbased.dll
 0002:0001e101       __callnewh                 1002f101 f   ucrtd:ucrtbased.dll
 0002:0001e107       _malloc                    1002f107 f   ucrtd:ucrtbased.dll
 0002:0001e10d       __seh_filter_dll           1002f10d f   ucrtd:ucrtbased.dll
 0002:0001e113       __configure_narrow_argv    1002f113 f   ucrtd:ucrtbased.dll
 0002:0001e119       __initialize_narrow_environment 1002f119 f   ucrtd:ucrtbased.dll
 0002:0001e11f       __initialize_onexit_table  1002f11f f   ucrtd:ucrtbased.dll
 0002:0001e125       __register_onexit_function 1002f125 f   ucrtd:ucrtbased.dll
 0002:0001e12b       __execute_onexit_table     1002f12b f   ucrtd:ucrtbased.dll
 0002:0001e131       __crt_atexit               1002f131 f   ucrtd:ucrtbased.dll
 0002:0001e137       __crt_at_quick_exit        1002f137 f   ucrtd:ucrtbased.dll
 0002:0001e13d       __cexit                    1002f13d f   ucrtd:ucrtbased.dll
 0002:0001e143       __CrtDbgReportW            1002f143 f   ucrtd:ucrtbased.dll
 0002:0001e149       __initterm                 1002f149 f   ucrtd:ucrtbased.dll
 0002:0001e14f       __initterm_e               1002f14f f   ucrtd:ucrtbased.dll
 0002:0001e155       __free_dbg                 1002f155 f   ucrtd:ucrtbased.dll
 0002:0001e15b       _terminate                 1002f15b f   ucrtd:ucrtbased.dll
 0002:0001e161       _strcpy_s                  1002f161 f   ucrtd:ucrtbased.dll
 0002:0001e167       _strcat_s                  1002f167 f   ucrtd:ucrtbased.dll
 0002:0001e16d       __wmakepath_s              1002f16d f   ucrtd:ucrtbased.dll
 0002:0001e173       __wsplitpath_s             1002f173 f   ucrtd:ucrtbased.dll
 0002:0001e179       _wcscpy_s                  1002f179 f   ucrtd:ucrtbased.dll
 0002:0001e17f       _GetCurrentThreadId@0      1002f17f f   kernel32:KERNEL32.dll
 0002:0001e185       _IsProcessorFeaturePresent@4 1002f185 f   kernel32:KERNEL32.dll
 0002:0001e18b       _IsDebuggerPresent@0       1002f18b f   kernel32:KERNEL32.dll
 0002:0001e191       _UnhandledExceptionFilter@4 1002f191 f   kernel32:KERNEL32.dll
 0002:0001e197       _SetUnhandledExceptionFilter@4 1002f197 f   kernel32:KERNEL32.dll
 0002:0001e19d       _GetStartupInfoW@4         1002f19d f   kernel32:KERNEL32.dll
 0002:0001e1a3       _GetModuleHandleW@4        1002f1a3 f   kernel32:KERNEL32.dll
 0002:0001e1a9       _RaiseException@16         1002f1a9 f   kernel32:KERNEL32.dll
 0002:0001e1af       _MultiByteToWideChar@24    1002f1af f   kernel32:KERNEL32.dll
 0002:0001e1b5       _WideCharToMultiByte@32    1002f1b5 f   kernel32:KERNEL32.dll
 0002:0001e1bb       _GetCurrentProcess@0       1002f1bb f   kernel32:KERNEL32.dll
 0002:0001e1c1       _TerminateProcess@8        1002f1c1 f   kernel32:KERNEL32.dll
 0002:0001e1c7       _QueryPerformanceCounter@4 1002f1c7 f   kernel32:KERNEL32.dll
 0002:0001e1cd       _GetSystemTimeAsFileTime@4 1002f1cd f   kernel32:KERNEL32.dll
 0002:0001e1d3       _DisableThreadLibraryCalls@4 1002f1d3 f   kernel32:KERNEL32.dll
 0002:0001e1d9       _InitializeSListHead@4     1002f1d9 f   kernel32:KERNEL32.dll
 0002:0001e1df       _HeapAlloc@12              1002f1df f   kernel32:KERNEL32.dll
 0002:0001e1e5       _HeapFree@12               1002f1e5 f   kernel32:KERNEL32.dll
 0002:0001e1eb       _GetProcessHeap@0          1002f1eb f   kernel32:KERNEL32.dll
 0002:0001e1f1       _VirtualQuery@12           1002f1f1 f   kernel32:KERNEL32.dll
 0002:0001e1f7       _FreeLibrary@4             1002f1f7 f   kernel32:KERNEL32.dll
 0002:0001e1fd       _GetProcAddress@8          1002f1fd f   kernel32:KERNEL32.dll
 0002:0001e210       ___acrt_initialize         1002f210 f   MSVCRTD:ucrt_stubs.obj
 0002:0001e210       ___scrt_stub_for_acrt_initialize 1002f210 f   MSVCRTD:ucrt_stubs.obj
 0002:0001e210       ___vcrt_initialize         1002f210 f   MSVCRTD:ucrt_stubs.obj
 0002:0001e220       ___acrt_thread_attach      1002f220 f   MSVCRTD:ucrt_stubs.obj
 0002:0001e220       ___scrt_stub_for_acrt_thread_attach 1002f220 f   MSVCRTD:ucrt_stubs.obj
 0002:0001e220       ___vcrt_thread_attach      1002f220 f   MSVCRTD:ucrt_stubs.obj
 0002:0001e230       ___acrt_thread_detach      1002f230 f   MSVCRTD:ucrt_stubs.obj
 0002:0001e230       ___scrt_stub_for_acrt_thread_detach 1002f230 f   MSVCRTD:ucrt_stubs.obj
 0002:0001e230       ___vcrt_thread_detach      1002f230 f   MSVCRTD:ucrt_stubs.obj
 0002:0001e240       ___acrt_uninitialize       1002f240 f   MSVCRTD:ucrt_stubs.obj
 0002:0001e240       ___scrt_stub_for_acrt_uninitialize 1002f240 f   MSVCRTD:ucrt_stubs.obj
 0002:0001e240       ___vcrt_uninitialize       1002f240 f   MSVCRTD:ucrt_stubs.obj
 0002:0001e250       ___acrt_uninitialize_critical 1002f250 f   MSVCRTD:ucrt_stubs.obj
 0002:0001e250       ___scrt_stub_for_acrt_uninitialize_critical 1002f250 f   MSVCRTD:ucrt_stubs.obj
 0002:0001e250       ___vcrt_uninitialize_critical 1002f250 f   MSVCRTD:ucrt_stubs.obj
 0002:0001e260       ___scrt_stub_for_is_c_termination_complete 1002f260 f   MSVCRTD:ucrt_stubs.obj
 0002:0001e260       __is_c_termination_complete 1002f260 f   MSVCRTD:ucrt_stubs.obj
 0002:0001e270       __filter_x86_sse2_floating_point_exception 1002f270 f   MSVCRTD:x86_exception_filter.obj
 0002:0001e270       __filter_x86_sse2_floating_point_exception_default 1002f270 f   MSVCRTD:x86_exception_filter.obj
 0003:00000000       ___xc_a                    10034000     MSVCRTD:initializers.obj
 0003:00000210       ___xc_z                    10034210     MSVCRTD:initializers.obj
 0003:00000314       ___xi_a                    10034314     MSVCRTD:initializers.obj
 0003:00000418       ___xi_z                    10034418     MSVCRTD:initializers.obj
 0003:0000051c       ___xp_a                    1003451c     MSVCRTD:initializers.obj
 0003:00000620       ___xp_z                    10034620     MSVCRTD:initializers.obj
 0003:00000724       ___xt_a                    10034724     MSVCRTD:initializers.obj
 0003:00000828       ___xt_z                    10034828     MSVCRTD:initializers.obj
 0003:00000930       _GUID_DEVINTERFACE_VJOY    10034930     stdafx.obj
 0003:00000948       ??_7exception@std@@6B@     10034948     vJoyInterface.obj
 0003:00000954       ??_C@_0BC@EOODALEL@Unknown?5exception@ 10034954     vJoyInterface.obj
 0003:00000970       ??_7bad_alloc@std@@6B@     10034970     vJoyInterface.obj
 0003:00000980       ??_7bad_array_new_length@std@@6B@ 10034980     vJoyInterface.obj
 0003:0000098c       ??_C@_0BF@KINCDENJ@bad?5array?5new?5length@ 1003498c     vJoyInterface.obj
 0003:000009a8       ??_C@_0BB@FCMFBGOM@invalid?5argument@ 100349a8     vJoyInterface.obj
 0003:000009bc       ??_C@_02DKCKIIND@?$CFs@    100349bc     vJoyInterface.obj
 0003:000009c0       ??_C@_0GC@ONGHGEHM@C?3?2Program?5Files?2Microsoft?5Visu@ 100349c0     vJoyInterface.obj
 0003:00000a38       ??_C@_1ME@DGNBIMPE@?$AAC?$AA?3?$AA?2?$AAP?$AAr?$AAo?$AAg?$AAr?$AAa?$AAm?$AA?5?$AAF?$AAi?$AAl?$AAe@ 10034a38     vJoyInterface.obj
 0003:00000b24       ??_C@_11LOCGONAA@@         10034b24     vJoyInterface.obj
 0003:00000b28       ??_C@_1CG@JNLFBNGN@?$AA?$CC?$AAi?$AAn?$AAv?$AAa?$AAl?$AAi?$AAd?$AA?5?$AAa?$AAr?$AAg?$AAu?$AAm?$AAe@ 10034b28     vJoyInterface.obj
 0003:00000b58       ??_C@_0BJ@LFDBABJJ@ITERATOR?5LIST?5CORRUPTED?$CB@ 10034b58     vJoyInterface.obj
 0003:00000b78       ??_C@_1DG@PLBPCAEM@?$AA?$CC?$AAI?$AAT?$AAE?$AAR?$AAA?$AAT?$AAO?$AAR?$AA?5?$AAL?$AAI?$AAS?$AAT?$AA?5@ 10034b78     vJoyInterface.obj
 0003:00000bb8       ??_C@_0BB@GCADKGJO@map?1set?5too?5long@ 10034bb8     vJoyInterface.obj
 0003:00000bcc       ??_C@_0BC@DJDCIKPO@vJoyInterface?5DLL@ 10034bcc     vJoyInterface.obj
 0003:00000be4       ??_C@_0CC@CIGAOLEI@Creation?5of?5Ffb?5data?9loop?5faile@ 10034be4     vJoyInterface.obj
 0003:00000c0c       ??_C@_0DI@KJIBHIIH@?6?$FL?$CF05u?$FNInfo?3?5FfbIsStarted?$CI?$CJ?5?9?5R@ 10034c0c     vJoyInterface.obj
 0003:00000c50       ??_C@_0EN@BHLHLNJM@?6?$FL?$CF05u?$FNError?3?5FfbIsStarted?$CI?$CJ?5?9?5@ 10034c50     vJoyInterface.obj
 0003:00000cac       ??_C@_0DK@FGNFEGKE@?6?$FL?$CF05u?$FNError?3?5FfbIsStarted?$CI?$CJ?5?9?5@ 10034cac     vJoyInterface.obj
 0003:00000cf8       ??_C@_0EH@PLFLBPHB@?6?$FL?$CF05u?$FNInfo?3?5FfbIsStarted?$CI?$CJ?5?9?5g@ 10034cf8     vJoyInterface.obj
 0003:00000d50       ??_C@_0EI@PGBDCIOA@?6?$FL?$CF05u?$FNInfo?3?5FfbIsStarted?$CI?$CJ?5?9?5g@ 10034d50     vJoyInterface.obj
 0003:00000da8       ??_C@_0DK@GIIAHIKB@?6?$FL?$CF05u?$FNInfo?3?5FfbWaitForData?$CI?$CJ?5?9@ 10034da8     vJoyInterface.obj
 0003:00000df0       ??_C@_0DM@IDKPOECN@?6?$FL?$CF05u?$FNError?3?5FfbWaitForData?$CI?$CJ?5@ 10034df0     vJoyInterface.obj
 0003:00000e38       ??_C@_0DM@BMIPGAAK@?6?$FL?$CF05u?$FNError?3?5FfbWaitForData?$CI?$CJ?5@ 10034e38     vJoyInterface.obj
 0003:00000e80       ??_C@_0EJ@EHPDLIOH@?6?$FL?$CF05u?$FNInfo?3?5FfbWaitForData?$CI?$CJ?5?9@ 10034e80     vJoyInterface.obj
 0003:00000ed8       ??_C@_0EK@OPMDLGDG@?6?$FL?$CF05u?$FNInfo?3?5FfbWaitForData?$CI?$CJ?5?9@ 10034ed8     vJoyInterface.obj
 0003:00000f30       ??_C@_0DF@NEAODPPN@?6?$FL?$CF05u?$FNInfo?3?5GetVJDStatus?$CI?$CFu?$CJ?5?9@ 10034f30     vJoyInterface.obj
 0003:00000f70       ??_C@_0DB@BOIMBPGK@?6?$FL?$CF05u?$FNInfo?3?5GetOwnerPid?$CI?$CFu?$CJ?5?9?5@ 10034f70     vJoyInterface.obj
 0003:00000fac       ??_C@_0DK@LCIAEING@?6?$FL?$CF05u?$FNInfo?3?5GetOwnerPid?$CI?$CFu?$CJ?5?9?5@ 10034fac     vJoyInterface.obj
 0003:00000ff8       ??_C@_0EG@PHNGBCHH@?6?$FL?$CF05u?$FNInfo?3?5GetOwnerPid?$CI?$CFu?$CJ?5?9?5@ 10034ff8     vJoyInterface.obj
 0003:0000104c       ??_C@_0DF@PEBAEFND@?6?$FL?$CF05u?$FNInfo?3?5GetVJDStatus?$CI?$CFu?$CJ?5?9@ 1003504c     vJoyInterface.obj
 0003:0000108c       ??_C@_0DF@OLMOEJ@?6?$FL?$CF05u?$FNInfo?3?5GetVJDStatus?$CI?$CFu?$CJ?5?9@ 1003508c     vJoyInterface.obj
 0003:000010cc       ??_C@_0CK@LDCNELEM@?6?$FL?$CF05u?$FNInfo?3?5GetVJDStatus?$CI?$CFu?$CJ?5?9@ 100350cc     vJoyInterface.obj
 0003:00001100       ??_C@_0DD@KAPKAMLC@?6?$FL?$CF05u?$FNInfo?3?5GetVJDButtonNumber@ 10035100     vJoyInterface.obj
 0003:00001140       ??_C@_0EK@FGGFLGJK@?6?$FL?$CF05u?$FNError?3?5GetVJDButtonNumbe@ 10035140     vJoyInterface.obj
 0003:00001198       ??_C@_0EB@FANGHBNE@?6?$FL?$CF05u?$FNError?3?5GetVJDButtonNumbe@ 10035198     vJoyInterface.obj
 0003:000011e8       ??_C@_0DJ@MIPGFEPM@?6?$FL?$CF05u?$FNInfo?3?5GetVJDButtonNumber@ 100351e8     vJoyInterface.obj
 0003:0000122c       ??_C@_0O@JLIIOHHC@?7?5Usage?$DN0x?$CFx?$DL@ 1003522c     vJoyInterface.obj
 0003:0000123c       ??_C@_0BC@CKIEAHHG@?7?5UsagePage?$DN0x?$CFx?$DL@ 1003523c     vJoyInterface.obj
 0003:00001254       ??_C@_0BM@OAIBPHPL@?7?5InputReportByteLength?$DN?$CFu?$DL@ 10035254     vJoyInterface.obj
 0003:00001278       ??_C@_0CA@BEHPBJED@?7?5NumberLinkCollectionNodes?$DN?$CFu?$DL@ 10035278     vJoyInterface.obj
 0003:000012a0       ??_C@_0BM@KGMIHPPH@?7?5NumberInputButtonCaps?$DN?$CFu?$DL@ 100352a0     vJoyInterface.obj
 0003:000012c4       ??_C@_0BL@ONMDOCNJ@?7?5NumberInputValueCaps?$DN?$CFu?$DL@ 100352c4     vJoyInterface.obj
 0003:000012e4       ??_C@_0BN@OIMOIFFL@?7?5NumberInputDataIndices?$DN?$CFu?$DL@ 100352e4     vJoyInterface.obj
 0003:00001308       ??_C@_0EH@NJPFMMFA@?6?$FL?$CF05u?$FNError?3?5GetVJDButtonNumbe@ 10035308     vJoyInterface.obj
 0003:00001360       ??_C@_0EH@MBAONGNP@?6?$FL?$CF05u?$FNError?3?5GetVJDButtonNumbe@ 10035360     vJoyInterface.obj
 0003:000013b8       ??_C@_0EA@GDNDDCLC@?6?$FL?$CF05u?$FNInfo?3?5GetVJDButtonNumber@ 100353b8     vJoyInterface.obj
 0003:00001404       ??_C@_0P@IHBDGNNC@?7?5ReportID?$DN?$CFu?$DL@ 10035404     vJoyInterface.obj
 0003:00001418       ??_C@_0P@LICDKPKK@?7?5UsageMax?$DN?$CFu?$DL@ 10035418     vJoyInterface.obj
 0003:0000142c       ??_C@_0P@FOEDAAEL@?7?5UsageMin?$DN?$CFu?$DL@ 1003542c     vJoyInterface.obj
 0003:00001440       ??_C@_0BD@NLDJCFEO@?7?5DataIndexMin?$DN?$CFu?$DL@ 10035440     vJoyInterface.obj
 0003:00001458       ??_C@_0DF@BFHCKPPP@?6?$FL?$CF05u?$FNError?3?5GetVJDButtonNumbe@ 10035458     vJoyInterface.obj
 0003:00001498       ??_C@_0DO@JCMNNNLM@?6?$FL?$CF05u?$FNInfo?3?5GetVJDButtonNumber@ 10035498     vJoyInterface.obj
 0003:000014e4       ??_C@_0DN@GKMMOCPB@?6?$FL?$CF05u?$FNInfo?3?5UpdateVJD?$CI?$CJ?5?9?5Devi@ 100354e4     vJoyInterface.obj
 0003:00001530       ??_C@_0ED@DELKEJBK@?6?$FL?$CF05u?$FNError?3?5UpdateVJD?$CI?$CJ?5?9?5Dev@ 10035530     vJoyInterface.obj
 0003:00001580       ??_C@_0DO@HGJOBJA@?6?$FL?$CF05u?$FNError?3?5UpdateVJD?$CI?$CJ?5?9?5Wai@ 10035580     vJoyInterface.obj
 0003:000015cc       ??_C@_0DG@CJNLHJGB@?6?$FL?$CF05u?$FNInfo?3?5UpdateVJD?$CI?$CJ?5?9?5Devi@ 100355cc     vJoyInterface.obj
 0003:0000160c       ??_C@_0DD@IIFFBAN@?6?$FL?$CF05u?$FNInfo?3?5GetHandleByIndex?$CIi@ 1003560c     vJoyInterface.obj
 0003:00001650       ??_C@_0EI@IBKBMHEE@?6?$FL?$CF05u?$FNError?3?5GetHandleByIndex?$CI@ 10035650     vJoyInterface.obj
 0003:000016a8       ??_C@_0GC@CGJMBGOL@?6?$FL?$CF05u?$FNWarning?3?5GetHandleByInde@ 100356a8     vJoyInterface.obj
 0003:00001720       ??_C@_0FG@LNCIOGIE@?6?$FL?$CF05u?$FNError?3?5GetHandleByIndex?$CI@ 10035720     vJoyInterface.obj
 0003:00001788       ??_C@_0FI@JJKOJABN@?6?$FL?$CF05u?$FNError?3?5GetHandleByIndex?$CI@ 10035788     vJoyInterface.obj
 0003:000017f8       ??_C@_0EE@MAENKEJ@?6?$FL?$CF05u?$FNError?3?5GetHandleByIndex?$CI@ 100357f8     vJoyInterface.obj
 0003:00001850       ??_C@_0EB@CCPPMMLE@?6?$FL?$CF05u?$FNInfo?3?5GetHandleByIndex?$CIi@ 10035850     vJoyInterface.obj
 0003:000018a0       ??_C@_0DJ@JMJDKHHE@?6?$FL?$CF05u?$FNInfo?3?5GetDeviceIndexById@ 100358a0     vJoyInterface.obj
 0003:000018e8       ??_C@_0GG@LIAAMOM@?6?$FL?$CF05u?$FNInfo?3?5GetDeviceIndexById@ 100358e8     vJoyInterface.obj
 0003:00001964       ??_C@_0DN@MDKJEAGA@?6?$FL?$CF05u?$FNInfo?3?5GetDeviceIndexById@ 10035964     vJoyInterface.obj
 0003:000019b0       ??_C@_0DF@MJJOJPJ@?6?$FL?$CF05u?$FNInfo?3?5GetDeviceIndexByRe@ 100359b0     vJoyInterface.obj
 0003:000019f0       ??_C@_0EL@MGILLLMF@?6?$FL?$CF05u?$FNInfo?3?5GetDeviceIndexByRe@ 100359f0     vJoyInterface.obj
 0003:00001a50       ??_C@_0EP@JHOMOKAP@?6?$FL?$CF05u?$FNInfo?3?5GetDeviceIndexByRe@ 10035a50     vJoyInterface.obj
 0003:00001ab0       ??_C@_0DG@OKBDGNJH@?6?$FL?$CF05u?$FNError?3?5GetDeviceIndexByR@ 10035ab0     vJoyInterface.obj
 0003:00001af0       ??_C@_0EK@LGHKGAFF@?6?$FL?$CF05u?$FNError?3?5GetDeviceNameSpac@ 10035af0     vJoyInterface.obj
 0003:00001b48       ??_C@_0GE@ELAIFKLL@?6?$FL?$CF05u?$FNError?3?5GetDeviceNameSpac@ 10035b48     vJoyInterface.obj
 0003:00001bc0       ??_C@_0FM@GGCEMBPG@?6?$FL?$CF05u?$FNError?3?5GetDeviceNameSpac@ 10035bc0     vJoyInterface.obj
 0003:00001c30       ??_C@_0DC@GAEOPMNG@?6?$FL?$CF05u?$FNInfo?3?5GetDeviceNameSpace@ 10035c30     vJoyInterface.obj
 0003:00001c70       ??_C@_0ED@HKFFFIGA@?6?$FL?$CF05u?$FNInfo?3?5GetDeviceNameSpace@ 10035c70     vJoyInterface.obj
 0003:00001cc0       ??_C@_0GE@NMJIIJJJ@?6?$FL?$CF05u?$FNInfo?3?5GetDeviceNameSpace@ 10035cc0     vJoyInterface.obj
 0003:00001d38       ??_C@_1BA@JCMDMCHI@?$AAD?$AAe?$AAv?$AAi?$AAc?$AAe?$AA_@ 10035d38     vJoyInterface.obj
 0003:00001d50       ??_C@_0EK@PCNOOKNC@?6?$FL?$CF05u?$FNError?3?5OpenDeviceInterfa@ 10035d50     vJoyInterface.obj
 0003:00001da8       ??_C@_0DM@BJLJHKNP@?6?$FL?$CF05u?$FNError?3?5OpenDeviceInterfa@ 10035da8     vJoyInterface.obj
 0003:00001df0       ??_C@_0FI@BMOHPPPH@?6?$FL?$CF05u?$FNInfo?3?5OpenDeviceInterfac@ 10035df0     vJoyInterface.obj
 0003:00001e5c       ??_C@_0CP@LKIMKJMP@?6?$FL?$CF05u?$FNInfo?3?5OpenDeviceInterfac@ 10035e5c     vJoyInterface.obj
 0003:00001e98       ??_C@_0GG@OMJAJDPH@?6?$FL?$CF05u?$FNInfo?3?5GetDevInfo?$CI?$CJ?5?9?5Ret@ 10035e98     vJoyInterface.obj
 0003:00001f14       ??_C@_0DI@FLNFFGAD@?6?$FL?$CF05u?$FNError?3?5GetDevInfo?$CI?$CJ?5?9?5Re@ 10035f14     vJoyInterface.obj
 0003:00001f58       ??_C@_0DI@MEPFNCCE@?6?$FL?$CF05u?$FNError?3?5GetDevInfo?$CI?$CJ?5?9?5er@ 10035f58     vJoyInterface.obj
 0003:00001fa0       ??_C@_0EF@GKLKBJFI@?6?$FL?$CF05u?$FNInfo?3?5GetDevInfo?$CI?$CJ?5?9?5got@ 10035fa0     vJoyInterface.obj
 0003:00001ff8       ??_C@_0EG@LEDAFBIK@?6?$FL?$CF05u?$FNInfo?3?5GetDevInfo?$CI?$CJ?5?9?5got@ 10035ff8     vJoyInterface.obj
 0003:00002050       ??_C@_0FL@OCDCLCEL@?6?$FL?$CF05u?$FNInfo?3?5GetDevStat?$CI?$CJ?5?9?5Ret@ 10036050     vJoyInterface.obj
 0003:000020c0       ??_C@_0DI@OLOAGCHJ@?6?$FL?$CF05u?$FNError?3?5GetDevStat?$CI?$CJ?5?9?5Re@ 100360c0     vJoyInterface.obj
 0003:00002104       ??_C@_0DI@HEMAOGFO@?6?$FL?$CF05u?$FNError?3?5GetDevStat?$CI?$CJ?5?9?5er@ 10036104     vJoyInterface.obj
 0003:00002148       ??_C@_0EF@EGCDMIKI@?6?$FL?$CF05u?$FNInfo?3?5GetDevStat?$CI?$CJ?5?9?5got@ 10036148     vJoyInterface.obj
 0003:000021a0       ??_C@_0EG@JKBDKEH@?6?$FL?$CF05u?$FNInfo?3?5GetDevStat?$CI?$CJ?5?9?5got@ 100361a0     vJoyInterface.obj
 0003:000021f8       ??_C@_0FD@GAKHOCIG@?6?$FL?$CF05u?$FNInfo?3?5GetDrvStat?$CI?$CJ?5?9?5Ret@ 100361f8     vJoyInterface.obj
 0003:0000225c       ??_C@_0DI@EIAKGMDI@?6?$FL?$CF05u?$FNError?3?5GetDrvStat?$CI?$CJ?5?9?5Re@ 1003625c     vJoyInterface.obj
 0003:000022a0       ??_C@_0DI@NHCKOIBP@?6?$FL?$CF05u?$FNError?3?5GetDrvStat?$CI?$CJ?5?9?5er@ 100362a0     vJoyInterface.obj
 0003:000022e8       ??_C@_0EF@KKEOOFFP@?6?$FL?$CF05u?$FNInfo?3?5GetDrvStat?$CI?$CJ?5?9?5got@ 100362e8     vJoyInterface.obj
 0003:00002340       ??_C@_0EG@CKJEDANF@?6?$FL?$CF05u?$FNInfo?3?5GetDrvStat?$CI?$CJ?5?9?5got@ 10036340     vJoyInterface.obj
 0003:00002394       ??_C@_08DNMKHOCF@?$CFs?$CFs?$CF03d@ 10036394     vJoyInterface.obj
 0003:000023a0       ??_C@_04OHGLKFFN@?$CF03d@  100363a0     vJoyInterface.obj
 0003:000023a8       ??_C@_0DI@GCJLPGON@?6?$FL?$CF05u?$FNInfo?3?5isRawDevice?$CI?$CFd?$CJ?5?9?5@ 100363a8     vJoyInterface.obj
 0003:000023ec       ??_C@_0CA@PGPJAAEK@Call?5to?5RegisterClassEx?5failed?$CB@ 100363ec     vJoyInterface.obj
 0003:00002414       ??_C@_0BG@CDOIHGNF@VJOYINTERFACELOGLEVEL@ 10036414     vJoyInterface.obj
 0003:00002430       ??_C@_0BF@FPKMOGPD@VJOYINTERFACELOGFILE@ 10036430     vJoyInterface.obj
 0003:0000244c       ??_C@_04JKHNIKCB@TEMP@     1003644c     vJoyInterface.obj
 0003:00002454       ??_C@_0BC@KPPPLGJO@vJoyInterface?4log@ 10036454     vJoyInterface.obj
 0003:0000246c       ??_C@_05BMGBEOOC@?$CFs?2?$CFs@ 1003646c     vJoyInterface.obj
 0003:00002474       ??_C@_02DPNLHKJD@a?$CL@    10036474     vJoyInterface.obj
 0003:00002478       ??_C@_0BF@PEEFBMH@?6?6?6?$FL?$CF05u?$FNProcess?3?$CFs?6@ 10036478     vJoyInterface.obj
 0003:00002494       ??_C@_0DA@IHMOFIMD@Create?5window?5process?5on?5anothe@ 10036494     vJoyInterface.obj
 0003:000024d0       ??_C@_0CB@HPGJNH@Creation?5of?5dummy?5window?5failed@ 100364d0     vJoyInterface.obj
 0003:000024f8       ??_C@_13NAACAHKO@?$AAX@    100364f8     vJoyInterface.obj
 0003:000024fc       ??_C@_13GILOGAML@?$AAY@    100364fc     vJoyInterface.obj
 0003:00002500       ??_C@_13HKALMPCF@?$AAZ@    10036500     vJoyInterface.obj
 0003:00002504       ??_C@_15BMCNAON@?$AAR?$AAX@ 10036504     vJoyInterface.obj
 0003:0000250c       ??_C@_15LJHOLHII@?$AAR?$AAY@ 1003650c     vJoyInterface.obj
 0003:00002514       ??_C@_15KLMLBIGG@?$AAR?$AAZ@ 10036514     vJoyInterface.obj
 0003:0000251c       ??_C@_17HBHJIBGA@?$AAS?$AAL?$AA1@ 1003651c     vJoyInterface.obj
 0003:00002528       ??_C@_17GDMMCOIO@?$AAS?$AAL?$AA2@ 10036528     vJoyInterface.obj
 0003:00002534       ??_C@_19MHJMLFKO@?$AAP?$AAO?$AAV?$AA1@ 10036534     vJoyInterface.obj
 0003:00002540       ??_C@_19NFCJBKEA@?$AAP?$AAO?$AAV?$AA2@ 10036540     vJoyInterface.obj
 0003:0000254c       ??_C@_19GNJFHNCF@?$AAP?$AAO?$AAV?$AA3@ 1003654c     vJoyInterface.obj
 0003:00002558       ??_C@_19PAECEFJM@?$AAP?$AAO?$AAV?$AA4@ 10036558     vJoyInterface.obj
 0003:00002568       ??_C@_1HC@DPIGBNJN@?$AAS?$AAY?$AAS?$AAT?$AAE?$AAM?$AA?2?$AAC?$AAu?$AAr?$AAr?$AAe?$AAn?$AAt?$AAC@ 10036568     vJoyInterface.obj
 0003:000025f0       ??_C@_19HABNGADD@?$AAI?$AAn?$AAi?$AAt@ 100365f0     vJoyInterface.obj
 0003:000025fc       ??_C@_1BG@NFFGKCLM@?$AA?$CF?$AAs?$AA?$CF?$AA0?$AA2?$AAu?$AA?2?$AA?$CF?$AAs?$AA?$AA@ 100365fc     vJoyInterface.obj
 0003:00002618       ??_C@_19LLLMHGHI@?$AAB?$AAT?$AAN?$AAS@ 10036618     vJoyInterface.obj
 0003:00002624       ??_C@_0DK@KMKOEHCO@?6?$FL?$CF05u?$FNInfo?3?5GetDevPosition?$CI?$CJ?5?9@ 10036624     vJoyInterface.obj
 0003:0000266c       ??_C@_0DM@POGMFEKD@?6?$FL?$CF05u?$FNError?3?5GetDevPosition?$CI?$CJ?5@ 1003666c     vJoyInterface.obj
 0003:000026b4       ??_C@_0DM@GBEMNAIE@?6?$FL?$CF05u?$FNError?3?5GetDevPosition?$CI?$CJ?5@ 100366b4     vJoyInterface.obj
 0003:00002700       ??_C@_0EJ@LKIENPKJ@?6?$FL?$CF05u?$FNInfo?3?5GetDevPosition?$CI?$CJ?5?9@ 10036700     vJoyInterface.obj
 0003:00002758       ??_C@_0EK@HOFKKNMG@?6?$FL?$CF05u?$FNInfo?3?5GetDevPosition?$CI?$CJ?5?9@ 10036758     vJoyInterface.obj
 0003:000027b0       ??_C@_0BP@OLDKBHLM@map?1set?5iterators?5incompatible@ 100367b0     vJoyInterface.obj
 0003:000027d8       ??_C@_0GA@GNHKHACC@C?3?2Program?5Files?2Microsoft?5Visu@ 100367d8     vJoyInterface.obj
 0003:00002850       ??_C@_1MA@LENEFKFL@?$AAC?$AA?3?$AA?2?$AAP?$AAr?$AAo?$AAg?$AAr?$AAa?$AAm?$AA?5?$AAF?$AAi?$AAl?$AAe@ 10036850     vJoyInterface.obj
 0003:00002938       ??_C@_1EC@JLIDLCDH@?$AA?$CC?$AAm?$AAa?$AAp?$AA?1?$AAs?$AAe?$AAt?$AA?5?$AAi?$AAt?$AAe?$AAr?$AAa?$AAt@ 10036938     vJoyInterface.obj
 0003:00002988       ??_C@_0DG@KGHKKGBC@null?5pointer?5cannot?5point?5to?5a?5@ 10036988     vJoyInterface.obj
 0003:000029c8       ??_C@_1HA@FACCKGGH@?$AA?$CC?$AAn?$AAu?$AAl?$AAl?$AA?5?$AAp?$AAo?$AAi?$AAn?$AAt?$AAe?$AAr?$AA?5?$AAc@ 100369c8     vJoyInterface.obj
 0003:00002a50       ??_C@_0BD@FEEMDEPI@invalid?5comparator@ 10036a50     vJoyInterface.obj
 0003:00002a68       ??_C@_0GD@JKKFFOCD@C?3?2Program?5Files?2Microsoft?5Visu@ 10036a68     vJoyInterface.obj
 0003:00002ae0       ??_C@_1MG@JJBOPAGB@?$AAC?$AA?3?$AA?2?$AAP?$AAr?$AAo?$AAg?$AAr?$AAa?$AAm?$AA?5?$AAF?$AAi?$AAl?$AAe@ 10036ae0     vJoyInterface.obj
 0003:00002bd0       ??_C@_1CK@NDNHPKPI@?$AA?$CC?$AAi?$AAn?$AAv?$AAa?$AAl?$AAi?$AAd?$AA?5?$AAc?$AAo?$AAm?$AAp?$AAa?$AAr@ 10036bd0     vJoyInterface.obj
 0003:00002c08       ??_7type_info@@6B@         10036c08     MSVCRTD:std_type_info_static.obj
 0003:00002c10       __pDefaultRawDllMain       10036c10     MSVCRTD:dll_dllmain.obj
 0003:00002c10       __pRawDllMain              10036c10     MSVCRTD:dll_dllmain.obj
 0003:00002c14       ??_C@_0P@GHFPNOJB@bad?5allocation@ 10036c14     MSVCRTD:throw_bad_alloc.obj
 0003:00002ce8       ??_C@_0NN@JMPELKLB@The?5value?5of?5ESP?5was?5not?5proper@ 10036ce8     MSVCRTD:error.obj
 0003:00002df8       ??_C@_0BBN@ELNNILBE@A?5cast?5to?5a?5smaller?5data?5type?5h@ 10036df8     MSVCRTD:error.obj
 0003:00002f50       ??_C@_0BN@BPOGFMJL@Stack?5memory?5was?5corrupted?$AN?6@ 10036f50     MSVCRTD:error.obj
 0003:00002f74       ??_C@_0DG@DAJCDLPN@A?5local?5variable?5was?5used?5befor@ 10036f74     MSVCRTD:error.obj
 0003:00002fb4       ??_C@_0CM@JMIDGKLA@Stack?5memory?5around?5_alloca?5was@ 10036fb4     MSVCRTD:error.obj
 0003:00002fe8       ??_C@_0BO@CHIONIOI@Unknown?5Runtime?5Check?5Error?$AN?6@ 10036fe8     MSVCRTD:error.obj
 0003:00003010       ??_C@_1GM@CNOOJIHC@?$AAR?$AAu?$AAn?$AAt?$AAi?$AAm?$AAe?$AA?5?$AAC?$AAh?$AAe?$AAc?$AAk?$AA?5?$AAE@ 10037010     MSVCRTD:error.obj
 0003:00003098       ??_C@_1EA@NFKNIFJP@?$AAR?$AAu?$AAn?$AA?9?$AAT?$AAi?$AAm?$AAe?$AA?5?$AAC?$AAh?$AAe?$AAc?$AAk?$AA?5@ 10037098     MSVCRTD:error.obj
 0003:000030e4       ??_C@_0BB@PFFGGCJP@Unknown?5Filename@ 100370e4     MSVCRTD:error.obj
 0003:000030f8       ??_C@_0BE@GNBOBNCK@Unknown?5Module?5Name@ 100370f8     MSVCRTD:error.obj
 0003:00003110       ??_C@_0CA@IODNCDPG@Run?9Time?5Check?5Failure?5?$CD?$CFd?5?9?5?$CFs@ 10037110     MSVCRTD:error.obj
 0003:00003138       ??_C@_0CG@IAFNJNEE@Stack?5corrupted?5near?5unknown?5va@ 10037138     MSVCRTD:error.obj
 0003:00003168       ??_C@_05MKKEDADM@?$CF?42X?5@ 10037168     MSVCRTD:error.obj
 0003:00003170       ??_C@_0EJ@LJKNEOLN@Stack?5area?5around?5_alloca?5memor@ 10037170     MSVCRTD:error.obj
 0003:000031c8       ??_C@_01EEMJAFIK@?6@       100371c8     MSVCRTD:error.obj
 0003:000031cc       ??_C@_02LLMPMKNF@?$DO?5@   100371cc     MSVCRTD:error.obj
 0003:000031d0       ??_C@_08OMAHNMHJ@?6Data?3?5?$DM@ 100371d0     MSVCRTD:error.obj
 0003:000031dc       ??_C@_0CK@DKGBICFE@?6Allocation?5number?5within?5this?5@ 100371dc     MSVCRTD:error.obj
 0003:00003210       ??_C@_07DFDJCKFN@?6Size?3?5@ 10037210     MSVCRTD:error.obj
 0003:0000321c       ??_C@_0N@MHFFIMFG@?6Address?3?50x@ 1003721c     MSVCRTD:error.obj
 0003:00003230       ??_C@_0EI@CLEPFNGI@Stack?5area?5around?5_alloca?5memor@ 10037230     MSVCRTD:error.obj
 0003:00003288       ??_C@_0BK@ODNDAGKB@?$CFs?$CFs?$CFp?$CFs?$CFzd?$CFs?$CFd?$CFs?$CFs?$CFs?$CFs?$CFs@ 10037288     MSVCRTD:error.obj
 0003:000032a8       ??_C@_0DE@OHJBPMBP@A?5variable?5is?5being?5used?5withou@ 100372a8     MSVCRTD:error.obj
 0003:0000330c       ??_C@_0BJ@HEGAHDFO@Stack?5pointer?5corruption@ 1003730c     MSVCRTD:userapi.obj
 0003:0000332c       ??_C@_0CK@FEGOIOPB@Cast?5to?5smaller?5type?5causing?5lo@ 1003732c     MSVCRTD:userapi.obj
 0003:00003360       ??_C@_0BI@CIGMDCBH@Stack?5memory?5corruption@ 10037360     MSVCRTD:userapi.obj
 0003:0000337c       ??_C@_0CK@CNLNOEPB@Local?5variable?5used?5before?5init@ 1003737c     MSVCRTD:userapi.obj
 0003:000033b0       ??_C@_0BP@OGBCLIBO@Stack?5around?5_alloca?5corrupted@ 100373b0     MSVCRTD:userapi.obj
 0003:00003430       ??_C@_1EI@MLPKHBGE@?$AAa?$AAp?$AAi?$AA?9?$AAm?$AAs?$AA?9?$AAw?$AAi?$AAn?$AA?9?$AAc?$AAo?$AAr?$AAe@ 10037430     MSVCRTD:pdblkup.obj
 0003:00003488       ??_C@_1BK@JHLNAEJL@?$AAa?$AAd?$AAv?$AAa?$AAp?$AAi?$AA3?$AA2?$AA?4?$AAd?$AAl?$AAl@ 10037488     MSVCRTD:pdblkup.obj
 0003:000034a8       ??_C@_0O@COHOBMLB@RegOpenKeyExW@ 100374a8     MSVCRTD:pdblkup.obj
 0003:000034b8       ??_C@_0BB@GLNAEDBD@RegQueryValueExW@ 100374b8     MSVCRTD:pdblkup.obj
 0003:000034cc       ??_C@_0M@HLOHPNFA@RegCloseKey@ 100374cc     MSVCRTD:pdblkup.obj
 0003:000034e0       ??_C@_1HE@EBEAGLFB@?$AAS?$AAO?$AAF?$AAT?$AAW?$AAA?$AAR?$AAE?$AA?2?$AAW?$AAo?$AAw?$AA6?$AA4?$AA3@ 100374e0     MSVCRTD:pdblkup.obj
 0003:0000356c       ??_C@_1BG@EABPBLLF@?$AAP?$AAr?$AAo?$AAd?$AAu?$AAc?$AAt?$AAD?$AAi?$AAr@ 1003756c     MSVCRTD:pdblkup.obj
 0003:000035ac       ??_C@_1BC@JINFINNJ@?$AAM?$AAS?$AAP?$AAD?$AAB?$AA1?$AA4?$AA0@ 100375ac     MSVCRTD:pdblkup.obj
 0003:000035c4       ??_C@_0BB@KCIACLNC@PDBOpenValidate5@ 100375c4     MSVCRTD:pdblkup.obj
 0003:000035d8       ??_C@_01KDCPPGHE@r@        100375d8     MSVCRTD:pdblkup.obj
 0003:000035e0       __load_config_used         100375e0     MSVCRTD:loadcfg.obj
 0003:000038c0       ___CastGuardVftablesStart  100378c0     MSVCRTD:guard_support.obj
 0003:00003a40       ___CastGuardVftablesEnd    10037a40     MSVCRTD:guard_support.obj
 0003:00003b8c       ??_R4exception@std@@6B@    10037b8c     vJoyInterface.obj
 0003:00003ba4       ??_R3exception@std@@8      10037ba4     vJoyInterface.obj
 0003:00003bb8       ??_R2exception@std@@8      10037bb8     vJoyInterface.obj
 0003:00003bc0       ??_R1A@?0A@EA@exception@std@@8 10037bc0     vJoyInterface.obj
 0003:00003be4       ??_R4bad_alloc@std@@6B@    10037be4     vJoyInterface.obj
 0003:00003bfc       ??_R3bad_alloc@std@@8      10037bfc     vJoyInterface.obj
 0003:00003c10       ??_R2bad_alloc@std@@8      10037c10     vJoyInterface.obj
 0003:00003c1c       ??_R1A@?0A@EA@bad_alloc@std@@8 10037c1c     vJoyInterface.obj
 0003:00003c40       ??_R4bad_array_new_length@std@@6B@ 10037c40     vJoyInterface.obj
 0003:00003c58       ??_R3bad_array_new_length@std@@8 10037c58     vJoyInterface.obj
 0003:00003c6c       ??_R2bad_array_new_length@std@@8 10037c6c     vJoyInterface.obj
 0003:00003c7c       ??_R1A@?0A@EA@bad_array_new_length@std@@8 10037c7c     vJoyInterface.obj
 0003:00003ca0       ??_R4type_info@@6B@        10037ca0     MSVCRTD:std_type_info_static.obj
 0003:00003cb8       ??_R3type_info@@8          10037cb8     MSVCRTD:std_type_info_static.obj
 0003:00003ccc       ??_R2type_info@@8          10037ccc     MSVCRTD:std_type_info_static.obj
 0003:00003cd4       ??_R1A@?0A@EA@type_info@@8 10037cd4     MSVCRTD:std_type_info_static.obj
 0003:00003f84       ___rtc_iaa                 10037f84     MSVCRTD:initsect.obj
 0003:0000418c       ___rtc_izz                 1003818c     MSVCRTD:initsect.obj
 0003:00004290       ___rtc_taa                 10038290     MSVCRTD:initsect.obj
 0003:00004498       ___rtc_tzz                 10038498     MSVCRTD:initsect.obj
 0003:00004b4c       __TI3?AVbad_array_new_length@std@@ 10038b4c     vJoyInterface.obj
 0003:00004b60       __CTA3?AVbad_array_new_length@std@@ 10038b60     vJoyInterface.obj
 0003:00004b74       __CT??_R0?AVbad_array_new_length@std@@@8??0bad_array_new_length@std@@QAE@ABV01@@Z12 10038b74     vJoyInterface.obj
 0003:00004b94       __CT??_R0?AVbad_alloc@std@@@8??0bad_alloc@std@@QAE@ABV01@@Z12 10038b94     vJoyInterface.obj
 0003:00004bb4       __CT??_R0?AVexception@std@@@8??0exception@std@@QAE@ABV01@@Z12 10038bb4     vJoyInterface.obj
 0003:00004c68       __TI2?AVbad_alloc@std@@    10038c68     MSVCRTD:throw_bad_alloc.obj
 0003:00004c7c       __CTA2?AVbad_alloc@std@@   10038c7c     MSVCRTD:throw_bad_alloc.obj
 0004:00000000       ?h0@@3PAXA                 1003a000     vJoyInterface.obj
 0004:00000050       ?__LINE__Var@?0??_Adjust_manually_vector_aligned@std@@YAXAAPAXAAI@Z@4JA 1003a050     vJoyInterface.obj
 0004:00000054       ___scrt_native_dllmain_reason 1003a054     MSVCRTD:utility.obj
 0004:00000060       ___security_cookie         1003a060     MSVCRTD:gs_cookie.obj
 0004:00000064       ___security_cookie_complement 1003a064     MSVCRTD:gs_cookie.obj
 0004:0000006c       ___isa_enabled             1003a06c     MSVCRTD:cpu_disp.obj
 0004:00000070       ?_RTC_ErrorLevels@@3PAHA   1003a070     MSVCRTD:error.obj
 0004:00000088       ___scrt_ucrt_dll_is_in_use 1003a088     MSVCRTD:ucrt_stubs.obj
 0004:00000194       ??_R0?AVbad_array_new_length@std@@@8 1003a194     vJoyInterface.obj
 0004:000001c4       ??_R0?AVbad_alloc@std@@@8  1003a1c4     vJoyInterface.obj
 0004:000001e8       ??_R0?AVexception@std@@@8  1003a1e8     vJoyInterface.obj
 0004:0000030c       ??_R0?AVtype_info@@@8      1003a30c     MSVCRTD:std_type_info_static.obj
 0004:00000428       ___@@_PchSym_@00@UfhvihUxbwUhlfixvUivklhUeqlbUzkkhUxlnnlmUeqlbrmgviuzxvUdrmDCUwvyftUhgwzucOlyq@4B2008FD98C1DD4 1003a428     stdafx.obj
 0004:0000042c       ___@@_PchSym_@00@UfhvihUxbwUhlfixvUivklhUeqlbUzkkhUxlnnlmUeqlbrmgviuzxvUdrmDCUwvyftUeqlbrmgviuzxvOlyq@4B2008FD98C1DD4 1003a42c     vJoyInterface.obj
 0004:00000430       ?Init@@3HA                 1003a430     vJoyInterface.obj
 0004:00000434       ?hInst@@3PAUHINSTANCE__@@A 1003a434     vJoyInterface.obj
 0004:00000438       ?hWnd@@3PAUHWND__@@A       1003a438     vJoyInterface.obj
 0004:0000043c       ?hDeviceNotifyInterFace@@3PAXA 1003a43c     vJoyInterface.obj
 0004:00000440       ?hDeviceNotifyHandle0@@3PAXA 1003a440     vJoyInterface.obj
 0004:00000444       ?hEvent@@3PAXA             1003a444     vJoyInterface.obj
 0004:00000448       ?ppDisable@@3PAXA          1003a448     vJoyInterface.obj
 0004:0000044c       ?ppEnable@@3PAXA           1003a44c     vJoyInterface.obj
 0004:00000450       ?LogFileName@@3PADA        1003a450     vJoyInterface.obj
 0004:00000454       ?Logging@@3HA              1003a454     vJoyInterface.obj
 0004:00000458       ?LogStream@@3PAU_iobuf@@A  1003a458     vJoyInterface.obj
 0004:0000045c       ?ProcessId@@3KA            1003a45c     vJoyInterface.obj
 0004:00000460       ?RemovalFunc@@3P6GXHHPAX@ZA 1003a460     vJoyInterface.obj
 0004:00000464       ?RemovalData@@3PAXA        1003a464     vJoyInterface.obj
 0004:00000468       ?FfbDataPacket@@3U_FFB_DATA@@A 1003a468     vJoyInterface.obj
 0004:00000474       ?FfbGebFunc@@3P6GXPAX0@ZA  1003a474     vJoyInterface.obj
 0004:00000478       ?FfbUserData@@3PAXA        1003a478     vJoyInterface.obj
 0004:0000047c       ?FfbEffectState@@3HA       1003a47c     vJoyInterface.obj
 0004:00000480       ?FfbEffectType@@3W4FFBEType@@A 1003a480     vJoyInterface.obj
 0004:00000484       ?hFfbEvent@@3PAXA          1003a484     vJoyInterface.obj
 0004:00000488       ?vJoyDevices@@3V?$map@HUDeviceStat@@U?$less@H@std@@V?$allocator@U?$pair@$$CBHUDeviceStat@@@std@@@3@@std@@A 1003a488     vJoyInterface.obj
 0004:00000494       ?mFfbEffect@@3V?$map@HW4FFB_EFFECTS@@U?$less@H@std@@V?$allocator@U?$pair@$$CBHW4FFB_EFFECTS@@@std@@@3@@std@@A 1003a494     vJoyInterface.obj
 0004:000004c8       ?_OptionsStorage@?1??__local_stdio_printf_options@@9@4_KA 1003a4c8     vJoyInterface.obj
 0004:000004d8       ?_OptionsStorage@?1??__local_stdio_scanf_options@@9@4_KA 1003a4d8     vJoyInterface.obj
 0004:000004e4       ___scrt_current_native_startup_state 1003a4e4     MSVCRTD:utility.obj
 0004:000004e8       ___scrt_native_startup_lock 1003a4e8     MSVCRTD:utility.obj
 0004:00000514       ___isa_available           1003a514     MSVCRTD:cpu_disp.obj
 0004:00000518       ___favor                   1003a518     MSVCRTD:cpu_disp.obj
 0004:00000520       ___scrt_debugger_hook_flag 1003a520     MSVCRTD:utility_desktop.obj
 0004:000008f0       ?__type_info_root_node@@3U__type_info_node@@A 1003a8f0     MSVCRTD:tncleanup.obj
 0004:00000904       ___dyn_tls_init_callback   1003a904     <common>
 0004:00000910       ___DebuggerCurrentSteppingThreadId 1003a910     <common>
 0005:00000000       __imp__RegCloseKey@4       1003b000     advapi32:ADVAPI32.dll
 0005:00000004       __imp__RegOpenKeyExW@20    1003b004     advapi32:ADVAPI32.dll
 0005:00000008       __imp__RegGetValueW@28     1003b008     advapi32:ADVAPI32.dll
 0005:0000000c       \177ADVAPI32_NULL_THUNK_DATA 1003b00c     advapi32:ADVAPI32.dll
 0005:00000038       __imp__HidD_GetSerialNumberString@12 1003b038     hid:HID.DLL
 0005:0000003c       __imp__HidP_GetCaps@8      1003b03c     hid:HID.DLL
 0005:00000040       __imp__HidP_GetLinkCollectionNodes@12 1003b040     hid:HID.DLL
 0005:00000044       __imp__HidP_GetButtonCaps@16 1003b044     hid:HID.DLL
 0005:00000048       __imp__HidP_GetSpecificValueCaps@28 1003b048     hid:HID.DLL
 0005:0000004c       __imp__HidP_GetValueCaps@16 1003b04c     hid:HID.DLL
 0005:00000050       __imp__HidP_GetUsageValue@32 1003b050     hid:HID.DLL
 0005:00000054       __imp__HidD_GetAttributes@8 1003b054     hid:HID.DLL
 0005:00000058       __imp__HidD_GetHidGuid@4   1003b058     hid:HID.DLL
 0005:0000005c       __imp__HidD_GetPreparsedData@8 1003b05c     hid:HID.DLL
 0005:00000060       __imp__HidD_FreePreparsedData@4 1003b060     hid:HID.DLL
 0005:00000064       __imp__HidD_GetManufacturerString@12 1003b064     hid:HID.DLL
 0005:00000068       __imp__HidD_GetProductString@12 1003b068     hid:HID.DLL
 0005:0000006c       \177HID_NULL_THUNK_DATA    1003b06c     hid:HID.DLL
 0005:000000a0       __imp__IsProcessorFeaturePresent@4 1003b0a0     kernel32:KERNEL32.dll
 0005:000000a4       __imp__FreeLibrary@4       1003b0a4     kernel32:KERNEL32.dll
 0005:000000a8       __imp__GetEnvironmentVariableA@12 1003b0a8     kernel32:KERNEL32.dll
 0005:000000ac       __imp__CreateFileA@28      1003b0ac     kernel32:KERNEL32.dll
 0005:000000b0       __imp__CloseHandle@4       1003b0b0     kernel32:KERNEL32.dll
 0005:000000b4       __imp__GetLastError@0      1003b0b4     kernel32:KERNEL32.dll
 0005:000000b8       __imp__DeviceIoControl@32  1003b0b8     kernel32:KERNEL32.dll
 0005:000000bc       __imp__GetOverlappedResult@16 1003b0bc     kernel32:KERNEL32.dll
 0005:000000c0       __imp__SetEvent@4          1003b0c0     kernel32:KERNEL32.dll
 0005:000000c4       __imp__WaitForSingleObject@8 1003b0c4     kernel32:KERNEL32.dll
 0005:000000c8       __imp__CreateEventA@16     1003b0c8     kernel32:KERNEL32.dll
 0005:000000cc       __imp__GetCurrentProcessId@0 1003b0cc     kernel32:KERNEL32.dll
 0005:000000d0       __imp__CreateThread@24     1003b0d0     kernel32:KERNEL32.dll
 0005:000000d4       __imp__GetModuleHandleA@4  1003b0d4     kernel32:KERNEL32.dll
 0005:000000d8       __imp__LocalAlloc@8        1003b0d8     kernel32:KERNEL32.dll
 0005:000000dc       __imp__LocalFree@4         1003b0dc     kernel32:KERNEL32.dll
 0005:000000e0       __imp__GetCommandLineA@0   1003b0e0     kernel32:KERNEL32.dll
 0005:000000e4       __imp__VirtualQuery@12     1003b0e4     kernel32:KERNEL32.dll
 0005:000000e8       __imp__GetProcessHeap@0    1003b0e8     kernel32:KERNEL32.dll
 0005:000000ec       __imp__HeapFree@12         1003b0ec     kernel32:KERNEL32.dll
 0005:000000f0       __imp__HeapAlloc@12        1003b0f0     kernel32:KERNEL32.dll
 0005:000000f4       __imp__InitializeSListHead@4 1003b0f4     kernel32:KERNEL32.dll
 0005:000000f8       __imp__DisableThreadLibraryCalls@4 1003b0f8     kernel32:KERNEL32.dll
 0005:000000fc       __imp__GetSystemTimeAsFileTime@4 1003b0fc     kernel32:KERNEL32.dll
 0005:00000100       __imp__QueryPerformanceCounter@4 1003b100     kernel32:KERNEL32.dll
 0005:00000104       __imp__TerminateProcess@8  1003b104     kernel32:KERNEL32.dll
 0005:00000108       __imp__GetCurrentProcess@0 1003b108     kernel32:KERNEL32.dll
 0005:0000010c       __imp__WideCharToMultiByte@32 1003b10c     kernel32:KERNEL32.dll
 0005:00000110       __imp__MultiByteToWideChar@24 1003b110     kernel32:KERNEL32.dll
 0005:00000114       __imp__RaiseException@16   1003b114     kernel32:KERNEL32.dll
 0005:00000118       __imp__GetModuleHandleW@4  1003b118     kernel32:KERNEL32.dll
 0005:0000011c       __imp__GetStartupInfoW@4   1003b11c     kernel32:KERNEL32.dll
 0005:00000120       __imp__SetUnhandledExceptionFilter@4 1003b120     kernel32:KERNEL32.dll
 0005:00000124       __imp__UnhandledExceptionFilter@4 1003b124     kernel32:KERNEL32.dll
 0005:00000128       __imp__IsDebuggerPresent@0 1003b128     kernel32:KERNEL32.dll
 0005:0000012c       __imp__GetProcAddress@8    1003b12c     kernel32:KERNEL32.dll
 0005:00000130       __imp__GetCurrentThreadId@0 1003b130     kernel32:KERNEL32.dll
 0005:00000134       \177KERNEL32_NULL_THUNK_DATA 1003b134     kernel32:KERNEL32.dll
 0005:0000017c       __imp_??0_Lockit@std@@QAE@H@Z 1003b17c     msvcprtd:MSVCP140D.dll
 0005:00000180       __imp_?_Xlength_error@std@@YAXPBD@Z 1003b180     msvcprtd:MSVCP140D.dll
 0005:00000184       __imp_??1_Lockit@std@@QAE@XZ 1003b184     msvcprtd:MSVCP140D.dll
 0005:00000188       \177MSVCP140D_NULL_THUNK_DATA 1003b188     msvcprtd:MSVCP140D.dll
 0005:000001b4       __imp__SetupDiEnumDeviceInterfaces@20 1003b1b4     setupapi:SETUPAPI.dll
 0005:000001b8       __imp__SetupDiGetClassDevsA@16 1003b1b8     setupapi:SETUPAPI.dll
 0005:000001bc       __imp__SetupDiGetDeviceInterfaceDetailA@24 1003b1bc     setupapi:SETUPAPI.dll
 0005:000001c0       __imp__SetupDiDestroyDeviceInfoList@4 1003b1c0     setupapi:SETUPAPI.dll
 0005:000001c4       \177SETUPAPI_NULL_THUNK_DATA 1003b1c4     setupapi:SETUPAPI.dll
 0005:000001f0       __imp__LoadIconA@8         1003b1f0     user32:USER32.dll
 0005:000001f4       __imp__LoadCursorA@8       1003b1f4     user32:USER32.dll
 0005:000001f8       __imp__MessageBoxA@16      1003b1f8     user32:USER32.dll
 0005:000001fc       __imp__EndPaint@8          1003b1fc     user32:USER32.dll
 0005:00000200       __imp__BeginPaint@8        1003b200     user32:USER32.dll
 0005:00000204       __imp__UpdateWindow@4      1003b204     user32:USER32.dll
 0005:00000208       __imp__ShowWindow@8        1003b208     user32:USER32.dll
 0005:0000020c       __imp__CreateWindowExA@48  1003b20c     user32:USER32.dll
 0005:00000210       __imp__RegisterClassExA@4  1003b210     user32:USER32.dll
 0005:00000214       __imp__PostQuitMessage@4   1003b214     user32:USER32.dll
 0005:00000218       __imp__DefWindowProcA@16   1003b218     user32:USER32.dll
 0005:0000021c       __imp__DispatchMessageA@4  1003b21c     user32:USER32.dll
 0005:00000220       __imp__GetMessageA@16      1003b220     user32:USER32.dll
 0005:00000224       __imp__TranslateMessage@4  1003b224     user32:USER32.dll
 0005:00000228       __imp__RegisterDeviceNotificationA@12 1003b228     user32:USER32.dll
 0005:0000022c       __imp__SendMessageA@16     1003b22c     user32:USER32.dll
 0005:00000230       __imp__UnregisterDeviceNotification@4 1003b230     user32:USER32.dll
 0005:00000234       \177USER32_NULL_THUNK_DATA 1003b234     user32:USER32.dll
 0005:0000026c       __imp____vcrt_LoadLibraryExW 1003b26c     vcruntimed:VCRUNTIME140D.dll
 0005:00000270       __imp____vcrt_GetModuleHandleW 1003b270     vcruntimed:VCRUNTIME140D.dll
 0005:00000274       __imp____vcrt_GetModuleFileNameW 1003b274     vcruntimed:VCRUNTIME140D.dll
 0005:00000278       __imp____std_type_info_destroy_list 1003b278     vcruntimed:VCRUNTIME140D.dll
 0005:0000027c       __imp___except_handler4_common 1003b27c     vcruntimed:VCRUNTIME140D.dll
 0005:00000280       __imp____current_exception_context 1003b280     vcruntimed:VCRUNTIME140D.dll
 0005:00000284       __imp__strrchr             1003b284     vcruntimed:VCRUNTIME140D.dll
 0005:00000288       __imp____CxxFrameHandler3  1003b288     vcruntimed:VCRUNTIME140D.dll
 0005:0000028c       __imp___CxxThrowException@8 1003b28c     vcruntimed:VCRUNTIME140D.dll
 0005:00000290       __imp____std_exception_destroy 1003b290     vcruntimed:VCRUNTIME140D.dll
 0005:00000294       __imp____std_exception_copy 1003b294     vcruntimed:VCRUNTIME140D.dll
 0005:00000298       __imp__strstr              1003b298     vcruntimed:VCRUNTIME140D.dll
 0005:0000029c       __imp__memcpy              1003b29c     vcruntimed:VCRUNTIME140D.dll
 0005:000002a0       __imp__memset              1003b2a0     vcruntimed:VCRUNTIME140D.dll
 0005:000002a4       __imp____current_exception 1003b2a4     vcruntimed:VCRUNTIME140D.dll
 0005:000002a8       \177VCRUNTIME140D_NULL_THUNK_DATA 1003b2a8     vcruntimed:VCRUNTIME140D.dll
 0005:000002e0       __imp___initialize_onexit_table 1003b2e0     ucrtd:ucrtbased.dll
 0005:000002e4       __imp___register_onexit_function 1003b2e4     ucrtd:ucrtbased.dll
 0005:000002e8       __imp___configure_narrow_argv 1003b2e8     ucrtd:ucrtbased.dll
 0005:000002ec       __imp___crt_atexit         1003b2ec     ucrtd:ucrtbased.dll
 0005:000002f0       __imp___crt_at_quick_exit  1003b2f0     ucrtd:ucrtbased.dll
 0005:000002f4       __imp___cexit              1003b2f4     ucrtd:ucrtbased.dll
 0005:000002f8       __imp___CrtDbgReportW      1003b2f8     ucrtd:ucrtbased.dll
 0005:000002fc       __imp___initterm           1003b2fc     ucrtd:ucrtbased.dll
 0005:00000300       __imp___initterm_e         1003b300     ucrtd:ucrtbased.dll
 0005:00000304       __imp___free_dbg           1003b304     ucrtd:ucrtbased.dll
 0005:00000308       __imp__terminate           1003b308     ucrtd:ucrtbased.dll
 0005:0000030c       __imp__strcpy_s            1003b30c     ucrtd:ucrtbased.dll
 0005:00000310       __imp__strcat_s            1003b310     ucrtd:ucrtbased.dll
 0005:00000314       __imp___wmakepath_s        1003b314     ucrtd:ucrtbased.dll
 0005:00000318       __imp___wsplitpath_s       1003b318     ucrtd:ucrtbased.dll
 0005:0000031c       __imp__wcscpy_s            1003b31c     ucrtd:ucrtbased.dll
 0005:00000320       __imp___initialize_narrow_environment 1003b320     ucrtd:ucrtbased.dll
 0005:00000324       __imp___seh_filter_dll     1003b324     ucrtd:ucrtbased.dll
 0005:00000328       __imp__malloc              1003b328     ucrtd:ucrtbased.dll
 0005:0000032c       __imp___callnewh           1003b32c     ucrtd:ucrtbased.dll
 0005:00000330       __imp___CrtDbgReport       1003b330     ucrtd:ucrtbased.dll
 0005:00000334       __imp____stdio_common_vsscanf 1003b334     ucrtd:ucrtbased.dll
 0005:00000338       __imp____stdio_common_vsprintf_s 1003b338     ucrtd:ucrtbased.dll
 0005:0000033c       __imp____stdio_common_vfprintf_s 1003b33c     ucrtd:ucrtbased.dll
 0005:00000340       __imp__fopen_s             1003b340     ucrtd:ucrtbased.dll
 0005:00000344       __imp____stdio_common_vswprintf_s 1003b344     ucrtd:ucrtbased.dll
 0005:00000348       __imp__wcstombs            1003b348     ucrtd:ucrtbased.dll
 0005:0000034c       __imp__atoi                1003b34c     ucrtd:ucrtbased.dll
 0005:00000350       __imp__free                1003b350     ucrtd:ucrtbased.dll
 0005:00000354       __imp__calloc              1003b354     ucrtd:ucrtbased.dll
 0005:00000358       __imp__strncpy             1003b358     ucrtd:ucrtbased.dll
 0005:0000035c       __imp___strlwr_s           1003b35c     ucrtd:ucrtbased.dll
 0005:00000360       __imp__strlen              1003b360     ucrtd:ucrtbased.dll
 0005:00000364       __imp___strdup             1003b364     ucrtd:ucrtbased.dll
 0005:00000368       __imp__wcslen              1003b368     ucrtd:ucrtbased.dll
 0005:0000036c       __imp___wcsdup             1003b36c     ucrtd:ucrtbased.dll
 0005:00000370       __imp___invalid_parameter  1003b370     ucrtd:ucrtbased.dll
 0005:00000374       __imp___execute_onexit_table 1003b374     ucrtd:ucrtbased.dll
 0005:00000378       \177ucrtbased_NULL_THUNK_DATA 1003b378     ucrtd:ucrtbased.dll
 0005:000003c0       __IMPORT_DESCRIPTOR_SETUPAPI 1003b3c0     setupapi:SETUPAPI.dll
 0005:000003d4       __IMPORT_DESCRIPTOR_HID    1003b3d4     hid:HID.DLL
 0005:000003e8       __IMPORT_DESCRIPTOR_KERNEL32 1003b3e8     kernel32:KERNEL32.dll
 0005:000003fc       __IMPORT_DESCRIPTOR_USER32 1003b3fc     user32:USER32.dll
 0005:00000410       __IMPORT_DESCRIPTOR_ADVAPI32 1003b410     advapi32:ADVAPI32.dll
 0005:00000424       __IMPORT_DESCRIPTOR_MSVCP140D 1003b424     msvcprtd:MSVCP140D.dll
 0005:00000438       __IMPORT_DESCRIPTOR_VCRUNTIME140D 1003b438     vcruntimed:VCRUNTIME140D.dll
 0005:0000044c       __IMPORT_DESCRIPTOR_ucrtbased 1003b44c     ucrtd:ucrtbased.dll
 0005:00000460       __NULL_IMPORT_DESCRIPTOR   1003b460     setupapi:SETUPAPI.dll
 0007:00000000       ___guard_check_icall_fptr  1003e000     MSVCRTD:guard_support.obj
 0007:00000004       ___guard_xfg_check_icall_fptr 1003e004     MSVCRTD:guard_support.obj
 0007:00000008       ___castguard_check_failure_os_handled_fptr 1003e008     MSVCRTD:guard_support.obj

 entry point at        0002:00000a91

 Static symbols

 0000:fffbe000       .debug$S                   10000000     vJoyInterface.exp
 0000:00000000       _volmd                     10000000     vJoyInterface.obj
 0000:00000000       _volmd                     10000000     vJoyInterface.obj
 0000:00000000       _volmd                     10000000     vJoyInterface.obj
 0000:00000000       _volmd                     10000000     vJoyInterface.obj
 0000:00000000       _volmd                     10000000     vJoyInterface.obj
 0000:00000000       _volmd                     10000000     vJoyInterface.obj
 0000:00000000       _volmd                     10000000     vJoyInterface.obj
 0000:00000000       _volmd                     10000000     vJoyInterface.obj
 0000:00000000       _volmd                     10000000     vJoyInterface.obj
 0000:00000000       _volmd                     10000000     vJoyInterface.obj
 0000:00000000       _volmd                     10000000     vJoyInterface.obj
 0000:00000000       _volmd                     10000000     vJoyInterface.obj
 0000:00000000       _volmd                     10000000     vJoyInterface.obj
 0000:00000000       _volmd                     10000000     vJoyInterface.obj
 0000:00000000       _volmd                     10000000     vJoyInterface.obj
 0000:00000000       _volmd                     10000000     vJoyInterface.obj
 0000:00000000       _volmd                     10000000     vJoyInterface.obj
 0000:00000000       _volmd                     10000000     vJoyInterface.obj
 0000:00000000       _volmd                     10000000     vJoyInterface.obj
 0000:00000000       _volmd                     10000000     vJoyInterface.obj
 0000:00000000       _volmd                     10000000     vJoyInterface.obj
 0000:00000000       _volmd                     10000000     vJoyInterface.obj
 0000:00000000       _volmd                     10000000     vJoyInterface.obj
 0000:00000000       _volmd                     10000000     vJoyInterface.obj
 0000:00000000       _volmd                     10000000     vJoyInterface.obj
 0000:00000000       _volmd                     10000000     vJoyInterface.obj
 0000:00000000       _volmd                     10000000     vJoyInterface.obj
 0000:00000000       _volmd                     10000000     vJoyInterface.obj
 0000:00000000       _volmd                     10000000     vJoyInterface.obj
 0000:00000000       _volmd                     10000000     vJoyInterface.obj
 0000:00000000       _volmd                     10000000     vJoyInterface.obj
 0000:00000000       _volmd                     10000000     vJoyInterface.obj
 0000:00000000       _volmd                     10000000     vJoyInterface.obj
 0000:00000000       _volmd                     10000000     vJoyInterface.obj
 0000:00000000       _volmd                     10000000     vJoyInterface.obj
 0000:00000000       _volmd                     10000000     vJoyInterface.obj
 0000:00000000       _volmd                     10000000     vJoyInterface.obj
 0000:00000000       _volmd                     10000000     vJoyInterface.obj
 0000:00000000       _volmd                     10000000     vJoyInterface.obj
 0000:00000000       _volmd                     10000000     vJoyInterface.obj
 0000:00000000       _volmd                     10000000     vJoyInterface.obj
 0000:00000000       _volmd                     10000000     vJoyInterface.obj
 0000:00000000       _volmd                     10000000     vJoyInterface.obj
 0000:00000000       _volmd                     10000000     vJoyInterface.obj
 0000:00000000       _volmd                     10000000     vJoyInterface.obj
 0000:00000000       _volmd                     10000000     vJoyInterface.obj
 0000:00000000       _volmd                     10000000     vJoyInterface.obj
 0000:00000000       _volmd                     10000000     vJoyInterface.obj
 0000:00000000       _volmd                     10000000     vJoyInterface.obj
 0000:00000000       _volmd                     10000000     vJoyInterface.obj
 0000:00000000       _volmd                     10000000     vJoyInterface.obj
 0000:00000000       _volmd                     10000000     vJoyInterface.obj
 0000:00000000       _volmd                     10000000     vJoyInterface.obj
 0000:00000000       _volmd                     10000000     vJoyInterface.obj
 0000:00000000       _volmd                     10000000     vJoyInterface.obj
 0000:00000000       _volmd                     10000000     vJoyInterface.obj
 0000:00000000       _volmd                     10000000     vJoyInterface.obj
 0000:00000000       _volmd                     10000000     vJoyInterface.obj
 0000:00000000       _volmd                     10000000     vJoyInterface.obj
 0000:00000000       _volmd                     10000000     vJoyInterface.obj
 0000:00000000       _volmd                     10000000     vJoyInterface.obj
 0000:00000000       _volmd                     10000000     vJoyInterface.obj
 0000:00000000       _volmd                     10000000     vJoyInterface.obj
 0000:00000000       _volmd                     10000000     vJoyInterface.obj
 0000:00000000       _volmd                     10000000     vJoyInterface.obj
 0000:00000000       _volmd                     10000000     vJoyInterface.obj
 0000:00000000       _volmd                     10000000     vJoyInterface.obj
 0000:00000000       _volmd                     10000000     vJoyInterface.obj
 0000:00000000       _volmd                     10000000     vJoyInterface.obj
 0000:00000000       _volmd                     10000000     vJoyInterface.obj
 0000:00000000       _volmd                     10000000     vJoyInterface.obj
 0000:00000000       _volmd                     10000000     vJoyInterface.obj
 0000:00000000       _volmd                     10000000     vJoyInterface.obj
 0000:00000000       _volmd                     10000000     vJoyInterface.obj
 0000:00000000       _volmd                     10000000     vJoyInterface.obj
 0000:fffbe000       .debug$S                   10000000     ucrtd:ucrtbased.dll
 0000:fffbe000       .debug$S                   10000000     ucrtd:ucrtbased.dll
 0000:fffbe000       .debug$S                   10000000     ucrtd:ucrtbased.dll
 0000:fffbe000       .debug$S                   10000000     ucrtd:ucrtbased.dll
 0000:fffbe000       .debug$S                   10000000     ucrtd:ucrtbased.dll
 0000:fffbe000       .debug$S                   10000000     ucrtd:ucrtbased.dll
 0000:fffbe000       .debug$S                   10000000     ucrtd:ucrtbased.dll
 0000:fffbe000       .debug$S                   10000000     ucrtd:ucrtbased.dll
 0000:fffbe000       .debug$S                   10000000     ucrtd:ucrtbased.dll
 0000:fffbe000       .debug$S                   10000000     ucrtd:ucrtbased.dll
 0000:fffbe000       .debug$S                   10000000     ucrtd:ucrtbased.dll
 0000:fffbe000       .debug$S                   10000000     ucrtd:ucrtbased.dll
 0000:fffbe000       .debug$S                   10000000     ucrtd:ucrtbased.dll
 0000:fffbe000       .debug$S                   10000000     ucrtd:ucrtbased.dll
 0000:fffbe000       .debug$S                   10000000     ucrtd:ucrtbased.dll
 0000:fffbe000       .debug$S                   10000000     ucrtd:ucrtbased.dll
 0000:fffbe000       .debug$S                   10000000     ucrtd:ucrtbased.dll
 0000:fffbe000       .debug$S                   10000000     ucrtd:ucrtbased.dll
 0000:fffbe000       .debug$S                   10000000     ucrtd:ucrtbased.dll
 0000:fffbe000       .debug$S                   10000000     ucrtd:ucrtbased.dll
 0000:fffbe000       .debug$S                   10000000     ucrtd:ucrtbased.dll
 0000:fffbe000       .debug$S                   10000000     ucrtd:ucrtbased.dll
 0000:fffbe000       .debug$S                   10000000     ucrtd:ucrtbased.dll
 0000:fffbe000       .debug$S                   10000000     ucrtd:ucrtbased.dll
 0000:fffbe000       .debug$S                   10000000     ucrtd:ucrtbased.dll
 0000:fffbe000       .debug$S                   10000000     ucrtd:ucrtbased.dll
 0000:fffbe000       .debug$S                   10000000     ucrtd:ucrtbased.dll
 0000:fffbe000       .debug$S                   10000000     ucrtd:ucrtbased.dll
 0000:fffbe000       .debug$S                   10000000     ucrtd:ucrtbased.dll
 0000:fffbe000       .debug$S                   10000000     ucrtd:ucrtbased.dll
 0000:fffbe000       .debug$S                   10000000     ucrtd:ucrtbased.dll
 0000:fffbe000       .debug$S                   10000000     ucrtd:ucrtbased.dll
 0000:fffbe000       .debug$S                   10000000     ucrtd:ucrtbased.dll
 0000:fffbe000       .debug$S                   10000000     ucrtd:ucrtbased.dll
 0000:fffbe000       .debug$S                   10000000     ucrtd:ucrtbased.dll
 0000:fffbe000       .debug$S                   10000000     ucrtd:ucrtbased.dll
 0000:fffbe000       .debug$S                   10000000     ucrtd:ucrtbased.dll
 0000:fffbe000       .debug$S                   10000000     ucrtd:ucrtbased.dll
 0000:fffbe000       .debug$S                   10000000     advapi32:ADVAPI32.dll
 0000:fffbe000       .debug$S                   10000000     advapi32:ADVAPI32.dll
 0000:fffbe000       .debug$S                   10000000     advapi32:ADVAPI32.dll
 0000:fffbe000       .debug$S                   10000000     hid:HID.DLL
 0000:fffbe000       .debug$S                   10000000     hid:HID.DLL
 0000:fffbe000       .debug$S                   10000000     hid:HID.DLL
 0000:fffbe000       .debug$S                   10000000     hid:HID.DLL
 0000:fffbe000       .debug$S                   10000000     hid:HID.DLL
 0000:fffbe000       .debug$S                   10000000     hid:HID.DLL
 0000:fffbe000       .debug$S                   10000000     hid:HID.DLL
 0000:fffbe000       .debug$S                   10000000     hid:HID.DLL
 0000:fffbe000       .debug$S                   10000000     hid:HID.DLL
 0000:fffbe000       .debug$S                   10000000     hid:HID.DLL
 0000:fffbe000       .debug$S                   10000000     hid:HID.DLL
 0000:fffbe000       .debug$S                   10000000     hid:HID.DLL
 0000:fffbe000       .debug$S                   10000000     hid:HID.DLL
 0000:fffbe000       .debug$S                   10000000     kernel32:KERNEL32.dll
 0000:fffbe000       .debug$S                   10000000     kernel32:KERNEL32.dll
 0000:fffbe000       .debug$S                   10000000     kernel32:KERNEL32.dll
 0000:fffbe000       .debug$S                   10000000     kernel32:KERNEL32.dll
 0000:fffbe000       .debug$S                   10000000     kernel32:KERNEL32.dll
 0000:fffbe000       .debug$S                   10000000     kernel32:KERNEL32.dll
 0000:fffbe000       .debug$S                   10000000     kernel32:KERNEL32.dll
 0000:fffbe000       .debug$S                   10000000     kernel32:KERNEL32.dll
 0000:fffbe000       .debug$S                   10000000     kernel32:KERNEL32.dll
 0000:fffbe000       .debug$S                   10000000     kernel32:KERNEL32.dll
 0000:fffbe000       .debug$S                   10000000     kernel32:KERNEL32.dll
 0000:fffbe000       .debug$S                   10000000     kernel32:KERNEL32.dll
 0000:fffbe000       .debug$S                   10000000     kernel32:KERNEL32.dll
 0000:fffbe000       .debug$S                   10000000     kernel32:KERNEL32.dll
 0000:fffbe000       .debug$S                   10000000     kernel32:KERNEL32.dll
 0000:fffbe000       .debug$S                   10000000     kernel32:KERNEL32.dll
 0000:fffbe000       .debug$S                   10000000     kernel32:KERNEL32.dll
 0000:fffbe000       .debug$S                   10000000     kernel32:KERNEL32.dll
 0000:fffbe000       .debug$S                   10000000     kernel32:KERNEL32.dll
 0000:fffbe000       .debug$S                   10000000     kernel32:KERNEL32.dll
 0000:fffbe000       .debug$S                   10000000     kernel32:KERNEL32.dll
 0000:fffbe000       .debug$S                   10000000     kernel32:KERNEL32.dll
 0000:fffbe000       .debug$S                   10000000     kernel32:KERNEL32.dll
 0000:fffbe000       .debug$S                   10000000     kernel32:KERNEL32.dll
 0000:fffbe000       .debug$S                   10000000     kernel32:KERNEL32.dll
 0000:fffbe000       .debug$S                   10000000     kernel32:KERNEL32.dll
 0000:fffbe000       .debug$S                   10000000     kernel32:KERNEL32.dll
 0000:fffbe000       .debug$S                   10000000     kernel32:KERNEL32.dll
 0000:fffbe000       .debug$S                   10000000     kernel32:KERNEL32.dll
 0000:fffbe000       .debug$S                   10000000     kernel32:KERNEL32.dll
 0000:fffbe000       .debug$S                   10000000     kernel32:KERNEL32.dll
 0000:fffbe000       .debug$S                   10000000     kernel32:KERNEL32.dll
 0000:fffbe000       .debug$S                   10000000     kernel32:KERNEL32.dll
 0000:fffbe000       .debug$S                   10000000     kernel32:KERNEL32.dll
 0000:fffbe000       .debug$S                   10000000     kernel32:KERNEL32.dll
 0000:fffbe000       .debug$S                   10000000     kernel32:KERNEL32.dll
 0000:fffbe000       .debug$S                   10000000     kernel32:KERNEL32.dll
 0000:fffbe000       .debug$S                   10000000     setupapi:SETUPAPI.dll
 0000:fffbe000       .debug$S                   10000000     setupapi:SETUPAPI.dll
 0000:fffbe000       .debug$S                   10000000     setupapi:SETUPAPI.dll
 0000:fffbe000       .debug$S                   10000000     setupapi:SETUPAPI.dll
 0000:fffbe000       .debug$S                   10000000     user32:USER32.dll
 0000:fffbe000       .debug$S                   10000000     user32:USER32.dll
 0000:fffbe000       .debug$S                   10000000     user32:USER32.dll
 0000:fffbe000       .debug$S                   10000000     user32:USER32.dll
 0000:fffbe000       .debug$S                   10000000     user32:USER32.dll
 0000:fffbe000       .debug$S                   10000000     user32:USER32.dll
 0000:fffbe000       .debug$S                   10000000     user32:USER32.dll
 0000:fffbe000       .debug$S                   10000000     user32:USER32.dll
 0000:fffbe000       .debug$S                   10000000     user32:USER32.dll
 0000:fffbe000       .debug$S                   10000000     user32:USER32.dll
 0000:fffbe000       .debug$S                   10000000     user32:USER32.dll
 0000:fffbe000       .debug$S                   10000000     user32:USER32.dll
 0000:fffbe000       .debug$S                   10000000     user32:USER32.dll
 0000:fffbe000       .debug$S                   10000000     user32:USER32.dll
 0000:fffbe000       .debug$S                   10000000     user32:USER32.dll
 0000:fffbe000       .debug$S                   10000000     user32:USER32.dll
 0000:fffbe000       .debug$S                   10000000     user32:USER32.dll
 0000:fffc3000       __guard_fids___except_handler4 10000000     MSVCRTD:chandler4gs.obj
 0000:00000000       _volmd                     10000000     MSVCRTD:cpu_disp.obj
 0000:fffc3000       __guard_fids_?dllmain_dispatch@@YAHQAUHINSTANCE__@@KQAX@Z 10000000     MSVCRTD:dll_dllmain.obj
 0000:00000000       _volmd                     10000000     MSVCRTD:gs_report.obj
 0000:fffc3000       __guard_fids__             10000000     MSVCRTD:guard_support.obj
 0000:fffc3000       __guard_fids__             10000000     MSVCRTD:guard_support.obj
 0000:fffc3000       __guard_fids___guard_icall_checks_enforced 10000000     MSVCRTD:guard_support.obj
 0000:00000000       _volmd                     10000000     MSVCRTD:guard_support.obj
 0000:00000000       _volmd                     10000000     MSVCRTD:guard_support.obj
 0000:fffc3000       __guard_fids___CRT_RTC_INIT 10000000     MSVCRTD:init.obj
 0000:fffc3000       __guard_fids___CRT_RTC_INITW 10000000     MSVCRTD:init.obj
 0000:fffc3000       __guard_fids__             10000000     MSVCRTD:std_type_info_static.obj
 0000:fffc3000       __guard_fids__             10000000     MSVCRTD:throw_bad_alloc.obj
 0000:fffc3000       __guard_fids__             10000000     MSVCRTD:throw_bad_alloc.obj
 0000:fffc3000       __guard_fids__             10000000     MSVCRTD:throw_bad_alloc.obj
 0000:fffc3000       __guard_fids__             10000000     MSVCRTD:throw_bad_alloc.obj
 0000:fffc3000       __guard_fids__             10000000     MSVCRTD:throw_bad_alloc.obj
 0000:fffc3000       __guard_fids__             10000000     MSVCRTD:throw_bad_alloc.obj
 0000:fffc3000       __guard_fids__             10000000     MSVCRTD:throw_bad_alloc.obj
 0000:fffc3000       __guard_fids__             10000000     MSVCRTD:throw_bad_alloc.obj
 0000:fffc3000       __guard_fids____scrt_set_unhandled_exception_filter 10000000     MSVCRTD:utility_desktop.obj
 0000:fffbe000       .debug$S                   10000000     msvcprtd:MSVCP140D.dll
 0000:fffbe000       .debug$S                   10000000     msvcprtd:MSVCP140D.dll
 0000:fffbe000       .debug$S                   10000000     msvcprtd:MSVCP140D.dll
 0000:fffbe000       .debug$S                   10000000     vcruntimed:VCRUNTIME140D.dll
 0000:fffbe000       .debug$S                   10000000     vcruntimed:VCRUNTIME140D.dll
 0000:fffbe000       .debug$S                   10000000     vcruntimed:VCRUNTIME140D.dll
 0000:fffbe000       .debug$S                   10000000     vcruntimed:VCRUNTIME140D.dll
 0000:fffbe000       .debug$S                   10000000     vcruntimed:VCRUNTIME140D.dll
 0000:fffbe000       .debug$S                   10000000     vcruntimed:VCRUNTIME140D.dll
 0000:fffbe000       .debug$S                   10000000     vcruntimed:VCRUNTIME140D.dll
 0000:fffbe000       .debug$S                   10000000     vcruntimed:VCRUNTIME140D.dll
 0000:fffbe000       .debug$S                   10000000     vcruntimed:VCRUNTIME140D.dll
 0000:fffbe000       .debug$S                   10000000     vcruntimed:VCRUNTIME140D.dll
 0000:fffbe000       .debug$S                   10000000     vcruntimed:VCRUNTIME140D.dll
 0000:fffbe000       .debug$S                   10000000     vcruntimed:VCRUNTIME140D.dll
 0000:fffbe000       .debug$S                   10000000     vcruntimed:VCRUNTIME140D.dll
 0000:fffbe000       .debug$S                   10000000     vcruntimed:VCRUNTIME140D.dll
 0000:fffbe000       .debug$S                   10000000     vcruntimed:VCRUNTIME140D.dll
 0002:000017e0       ??__EmFfbEffect@@YAXXZ     100127e0 f   vJoyInterface.obj
 0002:00001840       ??__EvJoyDevices@@YAXXZ    10012840 f   vJoyInterface.obj
 0002:000041f0       $LN5                       100151f0     vJoyInterface.obj
 0002:000041f8       $LN4                       100151f8     vJoyInterface.obj
 0002:00004204       $LN3                       10015204     vJoyInterface.obj
 0002:000042e0       $LN5                       100152e0     vJoyInterface.obj
 0002:000042e8       $LN4                       100152e8     vJoyInterface.obj
 0002:000042f4       $LN3                       100152f4     vJoyInterface.obj
 0002:00004a88       $LN7                       10015a88     vJoyInterface.obj
 0002:00004a90       $LN6                       10015a90     vJoyInterface.obj
 0002:00004a9c       $LN5                       10015a9c     vJoyInterface.obj
 0002:00004cd4       $LN18                      10015cd4     vJoyInterface.obj
 0002:00004cdc       $LN17                      10015cdc     vJoyInterface.obj
 0002:00004cf4       $LN15                      10015cf4     vJoyInterface.obj
 0002:00004cfc       $LN14                      10015cfc     vJoyInterface.obj
 0002:00005078       $LN6                       10016078     vJoyInterface.obj
 0002:00005080       $LN5                       10016080     vJoyInterface.obj
 0002:0000508c       $LN4                       1001608c     vJoyInterface.obj
 0002:000051bc       $LN9                       100161bc     vJoyInterface.obj
 0002:000051c4       $LN8                       100161c4     vJoyInterface.obj
 0002:000051d0       $LN7                       100161d0     vJoyInterface.obj
 0002:00005948       $LN7                       10016948     vJoyInterface.obj
 0002:00005950       $LN6                       10016950     vJoyInterface.obj
 0002:0000595c       $LN5                       1001695c     vJoyInterface.obj
 0002:00005b18       $LN7                       10016b18     vJoyInterface.obj
 0002:00005b20       $LN6                       10016b20     vJoyInterface.obj
 0002:00005b2c       $LN5                       10016b2c     vJoyInterface.obj
 0002:00006420       $LN9                       10017420     vJoyInterface.obj
 0002:00006428       $LN8                       10017428     vJoyInterface.obj
 0002:00006440       $LN7                       10017440     vJoyInterface.obj
 0002:00006447       $LN6                       10017447     vJoyInterface.obj
 0002:00006560       $LN8                       10017560     vJoyInterface.obj
 0002:00006568       $LN7                       10017568     vJoyInterface.obj
 0002:00006574       $LN6                       10017574     vJoyInterface.obj
 0002:00007084       $LN5                       10018084     vJoyInterface.obj
 0002:0000708c       $LN4                       1001808c     vJoyInterface.obj
 0002:00007098       $LN3                       10018098     vJoyInterface.obj
 0002:000081a4       $LN5                       100191a4     vJoyInterface.obj
 0002:000081ac       $LN4                       100191ac     vJoyInterface.obj
 0002:000081b8       $LN3                       100191b8     vJoyInterface.obj
 0002:00008284       $LN5                       10019284     vJoyInterface.obj
 0002:0000828c       $LN4                       1001928c     vJoyInterface.obj
 0002:00008298       $LN3                       10019298     vJoyInterface.obj
 0002:00008c6c       $LN5                       10019c6c     vJoyInterface.obj
 0002:00008c74       $LN4                       10019c74     vJoyInterface.obj
 0002:00008c80       $LN3                       10019c80     vJoyInterface.obj
 0002:00009408       $LN31                      1001a408     vJoyInterface.obj
 0002:00009410       $LN30                      1001a410     vJoyInterface.obj
 0002:00009440       $LN29                      1001a440     vJoyInterface.obj
 0002:0000944b       $LN28                      1001a44b     vJoyInterface.obj
 0002:00009456       $LN27                      1001a456     vJoyInterface.obj
 0002:00009462       $LN26                      1001a462     vJoyInterface.obj
 0002:000096c0       $LN9                       1001a6c0     vJoyInterface.obj
 0002:000096c8       $LN8                       1001a6c8     vJoyInterface.obj
 0002:000096d4       $LN7                       1001a6d4     vJoyInterface.obj
 0002:00009960       $LN10                      1001a960     vJoyInterface.obj
 0002:00009968       $LN9                       1001a968     vJoyInterface.obj
 0002:00009980       $LN8                       1001a980     vJoyInterface.obj
 0002:00009984       $LN7                       1001a984     vJoyInterface.obj
 0002:0000a018       $LN35                      1001b018     vJoyInterface.obj
 0002:0000a020       $LN34                      1001b020     vJoyInterface.obj
 0002:0000a08c       $LN33                      1001b08c     vJoyInterface.obj
 0002:0000a08f       $LN32                      1001b08f     vJoyInterface.obj
 0002:0000a092       $LN31                      1001b092     vJoyInterface.obj
 0002:0000a0a3       $LN30                      1001b0a3     vJoyInterface.obj
 0002:0000a0aa       $LN29                      1001b0aa     vJoyInterface.obj
 0002:0000a0bb       $LN28                      1001b0bb     vJoyInterface.obj
 0002:0000a0c0       $LN27                      1001b0c0     vJoyInterface.obj
 0002:0000a0c2       $LN26                      1001b0c2     vJoyInterface.obj
 0002:0000a0cf       $LN25                      1001b0cf     vJoyInterface.obj
 0002:0000a3b8       $LN11                      1001b3b8     vJoyInterface.obj
 0002:0000a3c0       $LN10                      1001b3c0     vJoyInterface.obj
 0002:0000a3cc       $LN9                       1001b3cc     vJoyInterface.obj
 0002:0000a890       $LN17                      1001b890     vJoyInterface.obj
 0002:0000a898       $LN16                      1001b898     vJoyInterface.obj
 0002:0000a8bc       $LN15                      1001b8bc     vJoyInterface.obj
 0002:0000a8be       $LN14                      1001b8be     vJoyInterface.obj
 0002:0000a8cb       $LN13                      1001b8cb     vJoyInterface.obj
 0002:0000aa20       $LN8                       1001ba20     vJoyInterface.obj
 0002:0000aa28       $LN7                       1001ba28     vJoyInterface.obj
 0002:0000aa34       $LN6                       1001ba34     vJoyInterface.obj
 0002:0000ab90       $LN8                       1001bb90     vJoyInterface.obj
 0002:0000ab98       $LN7                       1001bb98     vJoyInterface.obj
 0002:0000aba4       $LN6                       1001bba4     vJoyInterface.obj
 0002:0000b2a4       $LN34                      1001c2a4     vJoyInterface.obj
 0002:0000b2ac       $LN33                      1001c2ac     vJoyInterface.obj
 0002:0000b2d0       $LN32                      1001c2d0     vJoyInterface.obj
 0002:0000b2d2       $LN31                      1001c2d2     vJoyInterface.obj
 0002:0000b2df       $LN30                      1001c2df     vJoyInterface.obj
 0002:0000b2f0       $LN29                      1001c2f0     vJoyInterface.obj
 0002:0000b790       $LN20                      1001c790     vJoyInterface.obj
 0002:0000b798       $LN19                      1001c798     vJoyInterface.obj
 0002:0000b7bc       $LN18                      1001c7bc     vJoyInterface.obj
 0002:0000b7c9       $LN17                      1001c7c9     vJoyInterface.obj
 0002:0000b7d4       $LN16                      1001c7d4     vJoyInterface.obj
 0002:0000bb00       $LN19                      1001cb00     vJoyInterface.obj
 0002:0000bb08       $LN18                      1001cb08     vJoyInterface.obj
 0002:0000bb2c       $LN17                      1001cb2c     vJoyInterface.obj
 0002:0000bb39       $LN16                      1001cb39     vJoyInterface.obj
 0002:0000bb44       $LN15                      1001cb44     vJoyInterface.obj
 0002:0000bec4       $LN21                      1001cec4     vJoyInterface.obj
 0002:0000becc       $LN20                      1001cecc     vJoyInterface.obj
 0002:0000bef0       $LN19                      1001cef0     vJoyInterface.obj
 0002:0000befd       $LN18                      1001cefd     vJoyInterface.obj
 0002:0000bf08       $LN17                      1001cf08     vJoyInterface.obj
 0002:0000c0d0       $LN8                       1001d0d0     vJoyInterface.obj
 0002:0000c0d8       $LN7                       1001d0d8     vJoyInterface.obj
 0002:0000c0e4       $LN6                       1001d0e4     vJoyInterface.obj
 0002:0000c2e8       $LN14                      1001d2e8     vJoyInterface.obj
 0002:0000c2f0       $LN13                      1001d2f0     vJoyInterface.obj
 0002:0000c2fc       $LN12                      1001d2fc     vJoyInterface.obj
 0002:0000c654       $LN9                       1001d654     vJoyInterface.obj
 0002:0000c65c       $LN8                       1001d65c     vJoyInterface.obj
 0002:0000c668       $LN7                       1001d668     vJoyInterface.obj
 0002:0000cb24       $LN31                      1001db24     vJoyInterface.obj
 0002:0000cb2c       $LN30                      1001db2c     vJoyInterface.obj
 0002:0000cb50       $LN29                      1001db50     vJoyInterface.obj
 0002:0000cb59       $LN28                      1001db59     vJoyInterface.obj
 0002:0000cb68       $LN27                      1001db68     vJoyInterface.obj
 0002:0000d02c       $LN8                       1001e02c     vJoyInterface.obj
 0002:0000d034       $LN7                       1001e034     vJoyInterface.obj
 0002:0000d040       $LN6                       1001e040     vJoyInterface.obj
 0002:0000d320       $LN19                      1001e320     vJoyInterface.obj
 0002:0000d328       $LN18                      1001e328     vJoyInterface.obj
 0002:0000d34c       $LN17                      1001e34c     vJoyInterface.obj
 0002:0000d359       $LN16                      1001e359     vJoyInterface.obj
 0002:0000d364       $LN15                      1001e364     vJoyInterface.obj
 0002:0000d898       $LN22                      1001e898     vJoyInterface.obj
 0002:0000d8a0       $LN21                      1001e8a0     vJoyInterface.obj
 0002:0000d8c4       $LN20                      1001e8c4     vJoyInterface.obj
 0002:0000d8d3       $LN19                      1001e8d3     vJoyInterface.obj
 0002:0000d8e2       $LN18                      1001e8e2     vJoyInterface.obj
 0002:0000dd68       $LN21                      1001ed68     vJoyInterface.obj
 0002:0000dd70       $LN20                      1001ed70     vJoyInterface.obj
 0002:0000dda0       $LN19                      1001eda0     vJoyInterface.obj
 0002:0000dda8       $LN18                      1001eda8     vJoyInterface.obj
 0002:0000ddb0       $LN17                      1001edb0     vJoyInterface.obj
 0002:0000ddb5       $LN16                      1001edb5     vJoyInterface.obj
 0002:0000e04c       $LN13                      1001f04c     vJoyInterface.obj
 0002:0000e054       $LN12                      1001f054     vJoyInterface.obj
 0002:0000e060       $LN10                      1001f060     vJoyInterface.obj
 0002:0000e7d4       $LN15                      1001f7d4     vJoyInterface.obj
 0002:0000e7dc       $LN14                      1001f7dc     vJoyInterface.obj
 0002:0000e80c       $LN13                      1001f80c     vJoyInterface.obj
 0002:0000e80e       $LN12                      1001f80e     vJoyInterface.obj
 0002:0000e813       $LN11                      1001f813     vJoyInterface.obj
 0002:0000e820       $LN10                      1001f820     vJoyInterface.obj
 0002:0000ea50       $LN9                       1001fa50     vJoyInterface.obj
 0002:0000ea58       $LN8                       1001fa58     vJoyInterface.obj
 0002:0000ea64       $LN7                       1001fa64     vJoyInterface.obj
 0002:0000efc4       $LN15                      1001ffc4     vJoyInterface.obj
 0002:0000efcc       $LN14                      1001ffcc     vJoyInterface.obj
 0002:0000efd8       $LN13                      1001ffd8     vJoyInterface.obj
 0002:0000f380       $LN18                      10020380     vJoyInterface.obj
 0002:0000f388       $LN17                      10020388     vJoyInterface.obj
 0002:0000f3ac       $LN16                      100203ac     vJoyInterface.obj
 0002:0000f3b1       $LN15                      100203b1     vJoyInterface.obj
 0002:0000f3bb       $LN14                      100203bb     vJoyInterface.obj
 0002:0000f528       $LN7                       10020528     vJoyInterface.obj
 0002:0000f530       $LN6                       10020530     vJoyInterface.obj
 0002:0000f53c       $LN5                       1002053c     vJoyInterface.obj
 0002:0000f678       $LN7                       10020678     vJoyInterface.obj
 0002:0000f680       $LN6                       10020680     vJoyInterface.obj
 0002:0000f698       $LN5                       10020698     vJoyInterface.obj
 0002:0000f6ab       $LN4                       100206ab     vJoyInterface.obj
 0002:0000fb10       $LN14                      10020b10     vJoyInterface.obj
 0002:0000fb18       $LN13                      10020b18     vJoyInterface.obj
 0002:0000fb24       $LN11                      10020b24     vJoyInterface.obj
 0002:00010234       $LN15                      10021234     vJoyInterface.obj
 0002:0001023c       $LN14                      1002123c     vJoyInterface.obj
 0002:00010260       $LN13                      10021260     vJoyInterface.obj
 0002:00010269       $LN12                      10021269     vJoyInterface.obj
 0002:00010272       $LN11                      10021272     vJoyInterface.obj
 0002:00010474       $LN11                      10021474     vJoyInterface.obj
 0002:0001047c       $LN10                      1002147c     vJoyInterface.obj
 0002:00010488       $LN8                       10021488     vJoyInterface.obj
 0002:000107cc       $LN21                      100217cc     vJoyInterface.obj
 0002:000107d4       $LN20                      100217d4     vJoyInterface.obj
 0002:000107ec       $LN18                      100217ec     vJoyInterface.obj
 0002:000107f7       $LN17                      100217f7     vJoyInterface.obj
 0002:000109f8       $LN13                      100219f8     vJoyInterface.obj
 0002:00010a00       $LN12                      10021a00     vJoyInterface.obj
 0002:00010a0c       $LN11                      10021a0c     vJoyInterface.obj
 0002:00010d74       $LN5                       10021d74     vJoyInterface.obj
 0002:00010d7c       $LN4                       10021d7c     vJoyInterface.obj
 0002:00010d88       $LN3                       10021d88     vJoyInterface.obj
 0002:00010f60       $LN8                       10021f60     vJoyInterface.obj
 0002:00010f68       $LN7                       10021f68     vJoyInterface.obj
 0002:00010f80       $LN5                       10021f80     vJoyInterface.obj
 0002:00010f87       $LN4                       10021f87     vJoyInterface.obj
 0002:000110b0       $LN8                       100220b0     vJoyInterface.obj
 0002:000110b8       $LN7                       100220b8     vJoyInterface.obj
 0002:000110d0       $LN5                       100220d0     vJoyInterface.obj
 0002:000110d7       $LN4                       100220d7     vJoyInterface.obj
 0002:00011274       $LN5                       10022274     vJoyInterface.obj
 0002:0001127c       $LN4                       1002227c     vJoyInterface.obj
 0002:00011288       $LN3                       10022288     vJoyInterface.obj
 0002:00011480       $LN7                       10022480     vJoyInterface.obj
 0002:00011488       $LN6                       10022488     vJoyInterface.obj
 0002:000114a0       $LN4                       100224a0     vJoyInterface.obj
 0002:000114a6       $LN3                       100224a6     vJoyInterface.obj
 0002:000115ac       $LN8                       100225ac     vJoyInterface.obj
 0002:000115b4       $LN7                       100225b4     vJoyInterface.obj
 0002:000115c0       $LN6                       100225c0     vJoyInterface.obj
 0002:000116a0       $LN5                       100226a0     vJoyInterface.obj
 0002:000116a8       $LN4                       100226a8     vJoyInterface.obj
 0002:000116b4       $LN3                       100226b4     vJoyInterface.obj
 0002:00012700       $LN5                       10023700     vJoyInterface.obj
 0002:00012708       $LN4                       10023708     vJoyInterface.obj
 0002:00012714       $LN3                       10023714     vJoyInterface.obj
 0002:00012870       $LN5                       10023870     vJoyInterface.obj
 0002:00012878       $LN4                       10023878     vJoyInterface.obj
 0002:00012884       $LN3                       10023884     vJoyInterface.obj
 0002:00012ab8       $LN10                      10023ab8     vJoyInterface.obj
 0002:00012ac0       $LN9                       10023ac0     vJoyInterface.obj
 0002:00012acc       $LN8                       10023acc     vJoyInterface.obj
 0002:00012be8       $LN10                      10023be8     vJoyInterface.obj
 0002:00012bf0       $LN9                       10023bf0     vJoyInterface.obj
 0002:00012bfc       $LN8                       10023bfc     vJoyInterface.obj
 0002:00013864       $LN11                      10024864     vJoyInterface.obj
 0002:0001386c       $LN10                      1002486c     vJoyInterface.obj
 0002:00013884       $LN9                       10024884     vJoyInterface.obj
 0002:00013886       $LN8                       10024886     vJoyInterface.obj
 0002:00013d24       $LN11                      10024d24     vJoyInterface.obj
 0002:00013d2c       $LN10                      10024d2c     vJoyInterface.obj
 0002:00013d38       $LN8                       10024d38     vJoyInterface.obj
 0002:00014164       $LN11                      10025164     vJoyInterface.obj
 0002:0001416c       $LN10                      1002516c     vJoyInterface.obj
 0002:00014178       $LN9                       10025178     vJoyInterface.obj
 0002:000147bc       $LN20                      100257bc     vJoyInterface.obj
 0002:000147c4       $LN19                      100257c4     vJoyInterface.obj
 0002:000147f4       $LN18                      100257f4     vJoyInterface.obj
 0002:00014801       $LN17                      10025801     vJoyInterface.obj
 0002:0001480c       $LN16                      1002580c     vJoyInterface.obj
 0002:00014811       $LN15                      10025811     vJoyInterface.obj
 0002:00014c1c       $LN9                       10025c1c     vJoyInterface.obj
 0002:00014c24       $LN8                       10025c24     vJoyInterface.obj
 0002:00014c30       $LN7                       10025c30     vJoyInterface.obj
 0002:00014fd8       $LN23                      10025fd8     vJoyInterface.obj
 0002:00014fe0       $LN22                      10025fe0     vJoyInterface.obj
 0002:00015010       $LN21                      10026010     vJoyInterface.obj
 0002:0001501e       $LN20                      1002601e     vJoyInterface.obj
 0002:0001502b       $LN19                      1002602b     vJoyInterface.obj
 0002:00015033       $LN18                      10026033     vJoyInterface.obj
 0002:000151b8       $LN9                       100261b8     vJoyInterface.obj
 0002:000151c0       $LN8                       100261c0     vJoyInterface.obj
 0002:000151cc       $LN7                       100261cc     vJoyInterface.obj
 0002:000152b8       $LN9                       100262b8     vJoyInterface.obj
 0002:000152c0       $LN8                       100262c0     vJoyInterface.obj
 0002:000152cc       $LN7                       100262cc     vJoyInterface.obj
 0002:00015480       $LN10                      10026480     vJoyInterface.obj
 0002:00015488       $LN9                       10026488     vJoyInterface.obj
 0002:00015494       $LN8                       10026494     vJoyInterface.obj
 0002:00015578       $LN9                       10026578     vJoyInterface.obj
 0002:00015580       $LN8                       10026580     vJoyInterface.obj
 0002:0001558c       $LN7                       1002658c     vJoyInterface.obj
 0002:000156a4       $LN9                       100266a4     vJoyInterface.obj
 0002:000156ac       $LN8                       100266ac     vJoyInterface.obj
 0002:000156b8       $LN7                       100266b8     vJoyInterface.obj
 0002:000158e4       $LN9                       100268e4     vJoyInterface.obj
 0002:000158ec       $LN8                       100268ec     vJoyInterface.obj
 0002:000158f8       $LN7                       100268f8     vJoyInterface.obj
 0002:00015a54       $LN9                       10026a54     vJoyInterface.obj
 0002:00015a5c       $LN8                       10026a5c     vJoyInterface.obj
 0002:00015a68       $LN7                       10026a68     vJoyInterface.obj
 0002:00015c7c       $LN9                       10026c7c     vJoyInterface.obj
 0002:00015c84       $LN8                       10026c84     vJoyInterface.obj
 0002:00015c90       $LN7                       10026c90     vJoyInterface.obj
 0002:00015eac       $LN9                       10026eac     vJoyInterface.obj
 0002:00015eb4       $LN8                       10026eb4     vJoyInterface.obj
 0002:00015ec0       $LN7                       10026ec0     vJoyInterface.obj
 0002:0001604c       $LN9                       1002704c     vJoyInterface.obj
 0002:00016054       $LN8                       10027054     vJoyInterface.obj
 0002:00016060       $LN7                       10027060     vJoyInterface.obj
 0002:000162c0       $LN13                      100272c0     vJoyInterface.obj
 0002:000162c8       $LN12                      100272c8     vJoyInterface.obj
 0002:000162d4       $LN11                      100272d4     vJoyInterface.obj
 0002:0001657c       $LN9                       1002757c     vJoyInterface.obj
 0002:00016584       $LN8                       10027584     vJoyInterface.obj
 0002:0001659c       $LN7                       1002759c     vJoyInterface.obj
 0002:000165a3       $LN6                       100275a3     vJoyInterface.obj
 0002:00016750       $LN12                      10027750     vJoyInterface.obj
 0002:00016758       $LN11                      10027758     vJoyInterface.obj
 0002:00016770       $LN10                      10027770     vJoyInterface.obj
 0002:00016777       $LN9                       10027777     vJoyInterface.obj
 0002:00016a10       $LN18                      10027a10     vJoyInterface.obj
 0002:00016a18       $LN17                      10027a18     vJoyInterface.obj
 0002:00016a24       $LN16                      10027a24     vJoyInterface.obj
 0002:00016a30       $LN15                      10027a30     vJoyInterface.obj
 0002:00016b78       $LN6                       10027b78     vJoyInterface.obj
 0002:00016b80       $LN5                       10027b80     vJoyInterface.obj
 0002:00016b8c       $LN4                       10027b8c     vJoyInterface.obj
 0002:00016c48       $LN6                       10027c48     vJoyInterface.obj
 0002:00016c50       $LN5                       10027c50     vJoyInterface.obj
 0002:00016c5c       $LN4                       10027c5c     vJoyInterface.obj
 0002:00017264       $LN24                      10028264     vJoyInterface.obj
 0002:0001726c       $LN23                      1002826c     vJoyInterface.obj
 0002:00017290       $LN22                      10028290     vJoyInterface.obj
 0002:00017292       $LN21                      10028292     vJoyInterface.obj
 0002:0001729f       $LN20                      1002829f     vJoyInterface.obj
 0002:000176ac       $LN16                      100286ac     vJoyInterface.obj
 0002:000176b4       $LN15                      100286b4     vJoyInterface.obj
 0002:000176d8       $LN14                      100286d8     vJoyInterface.obj
 0002:000176da       $LN13                      100286da     vJoyInterface.obj
 0002:000176e7       $LN12                      100286e7     vJoyInterface.obj
 0002:00017a2c       $LN16                      10028a2c     vJoyInterface.obj
 0002:00017a34       $LN15                      10028a34     vJoyInterface.obj
 0002:00017a58       $LN14                      10028a58     vJoyInterface.obj
 0002:00017a5a       $LN13                      10028a5a     vJoyInterface.obj
 0002:00017a67       $LN12                      10028a67     vJoyInterface.obj
 0002:00017d3c       $LN15                      10028d3c     vJoyInterface.obj
 0002:00017d44       $LN14                      10028d44     vJoyInterface.obj
 0002:00017d5c       $LN13                      10028d5c     vJoyInterface.obj
 0002:00017d63       $LN12                      10028d63     vJoyInterface.obj
 0002:00017e94       $LN7                       10028e94     vJoyInterface.obj
 0002:00017e9c       $LN6                       10028e9c     vJoyInterface.obj
 0002:00017ea8       $LN5                       10028ea8     vJoyInterface.obj
 0002:00017fb0       $LN9                       10028fb0     vJoyInterface.obj
 0002:00017fb8       $LN8                       10028fb8     vJoyInterface.obj
 0002:00017fd0       $LN7                       10028fd0     vJoyInterface.obj
 0002:00017fd7       $LN6                       10028fd7     vJoyInterface.obj
 0002:000180b4       $LN7                       100290b4     vJoyInterface.obj
 0002:000180bc       $LN6                       100290bc     vJoyInterface.obj
 0002:000180c8       $LN5                       100290c8     vJoyInterface.obj
 0002:000181a4       $LN7                       100291a4     vJoyInterface.obj
 0002:000181ac       $LN6                       100291ac     vJoyInterface.obj
 0002:000181b8       $LN5                       100291b8     vJoyInterface.obj
 0002:0001829c       $LN7                       1002929c     vJoyInterface.obj
 0002:000182a4       $LN6                       100292a4     vJoyInterface.obj
 0002:000182b0       $LN5                       100292b0     vJoyInterface.obj
 0002:00018530       $LN16                      10029530     vJoyInterface.obj
 0002:00018538       $LN15                      10029538     vJoyInterface.obj
 0002:00018568       $LN14                      10029568     vJoyInterface.obj
 0002:0001856d       $LN13                      1002956d     vJoyInterface.obj
 0002:0001856f       $LN12                      1002956f     vJoyInterface.obj
 0002:0001857c       $LN11                      1002957c     vJoyInterface.obj
 0002:000188d4       $LN19                      100298d4     vJoyInterface.obj
 0002:000188dc       $LN18                      100298dc     vJoyInterface.obj
 0002:00018900       $LN17                      10029900     vJoyInterface.obj
 0002:00018903       $LN16                      10029903     vJoyInterface.obj
 0002:00018910       $LN15                      10029910     vJoyInterface.obj
 0002:00018cac       $LN7                       10029cac     vJoyInterface.obj
 0002:00018cb4       $LN6                       10029cb4     vJoyInterface.obj
 0002:00018cc0       $LN5                       10029cc0     vJoyInterface.obj
 0002:00018fcc       $LN15                      10029fcc     vJoyInterface.obj
 0002:00018fd4       $LN14                      10029fd4     vJoyInterface.obj
 0002:00018fe0       $LN13                      10029fe0     vJoyInterface.obj
 0002:000192b0       $LN16                      1002a2b0     vJoyInterface.obj
 0002:000192b8       $LN15                      1002a2b8     vJoyInterface.obj
 0002:000192d0       $LN14                      1002a2d0     vJoyInterface.obj
 0002:000192d6       $LN13                      1002a2d6     vJoyInterface.obj
 0002:000195fc       $LN17                      1002a5fc     vJoyInterface.obj
 0002:00019874       $LN14                      1002a874     vJoyInterface.obj
 0002:00019ab8       $LN12                      1002aab8     vJoyInterface.obj
 0002:0001a1c4       $LN10                      1002b1c4     vJoyInterface.obj
 0002:0001a1cc       $LN9                       1002b1cc     vJoyInterface.obj
 0002:0001a1e4       $LN8                       1002b1e4     vJoyInterface.obj
 0002:0001a1eb       $LN7                       1002b1eb     vJoyInterface.obj
 0002:0001a2c8       $LN7                       1002b2c8     vJoyInterface.obj
 0002:0001a2d0       $LN6                       1002b2d0     vJoyInterface.obj
 0002:0001a2dc       $LN5                       1002b2dc     vJoyInterface.obj
 0002:0001a504       $LN7                       1002b504     vJoyInterface.obj
 0002:0001a50c       $LN6                       1002b50c     vJoyInterface.obj
 0002:0001a524       $LN5                       1002b524     vJoyInterface.obj
 0002:0001a529       $LN4                       1002b529     vJoyInterface.obj
 0002:0001a61c       $LN8                       1002b61c     vJoyInterface.obj
 0002:0001a624       $LN7                       1002b624     vJoyInterface.obj
 0002:0001a63c       $LN6                       1002b63c     vJoyInterface.obj
 0002:0001a643       $LN5                       1002b643     vJoyInterface.obj
 0002:0001a920       ?find_pe_section@@YAPAU_IMAGE_SECTION_HEADER@@QAEI@Z 1002b920 f   MSVCRTD:utility.obj
 0002:0001a9e0       ?is_potentially_valid_image_base@@YA_NQAX@Z 1002b9e0 f   MSVCRTD:utility.obj
 0002:0001b3d0       $$000000                   1002c3d0     MSVCRTD:chkstk.obj
 0002:0001b3e4       cs10                       1002c3e4     MSVCRTD:chkstk.obj
 0002:0001b3f2       cs20                       1002c3f2     MSVCRTD:chkstk.obj
 0002:0001b470       ?dllmain_crt_dispatch@@YGHQAUHINSTANCE__@@KQAX@Z 1002c470 f   MSVCRTD:dll_dllmain.obj
 0002:0001b4dc       $LN11                      1002c4dc     MSVCRTD:dll_dllmain.obj
 0002:0001b510       ?dllmain_crt_process_attach@@YAHQAUHINSTANCE__@@QAX@Z 1002c510 f   MSVCRTD:dll_dllmain.obj
 0002:0001b6e0       ?dllmain_crt_process_detach@@YAH_N@Z 1002c6e0 f   MSVCRTD:dll_dllmain.obj
 0002:0001b820       ?dllmain_dispatch@@YAHQAUHINSTANCE__@@KQAX@Z 1002c820 f   MSVCRTD:dll_dllmain.obj
 0002:0001ba10       ?dllmain_raw@@YGHQAUHINSTANCE__@@KQAX@Z 1002ca10 f   MSVCRTD:dll_dllmain.obj
 0002:0001c480       ___castguard_check_failure_os_handled_wrapper 1002d480 f   MSVCRTD:guard_support.obj
 0002:0001c4b0       ___castguard_compat_check  1002d4b0 f   MSVCRTD:guard_support.obj
 0002:0001c5f0       ___castguard_slow_path_compat_check 1002d5f0 f   MSVCRTD:guard_support.obj
 0002:0001c680       ?DebuggerProbe@@YA_NK@Z    1002d680 f   MSVCRTD:error.obj
 0002:0001c6d0       ?DebuggerRuntime@@YA_NKHPAXPB_W@Z 1002d6d0 f   MSVCRTD:error.obj
 0002:0001c9a0       ?_getMemBlockDataString@@YAXPAD0PBDI@Z 1002d9a0 f   MSVCRTD:error.obj
 0002:0001ca30       ?_strlen_priv@@YAIPBD@Z    1002da30 f   MSVCRTD:error.obj
 0002:0001ca50       ?failwithmessage@@YAXPAXHHPBD@Z 1002da50 f   MSVCRTD:error.obj
 0002:0001ccd0       ?notify_debugger@@YAXABUtagEXCEPTION_VISUALCPP_DEBUG_INFO@@@Z 1002dcd0 f   MSVCRTD:error.obj
 0002:0001d350       ___get_entropy             1002e350 f   MSVCRTD:gs_support.obj
 0002:0001d5d0       ?GetPdbDll@@YAPAUHINSTANCE__@@XZ 1002e5d0 f   MSVCRTD:pdblkup.obj
 0002:0001d770       ?GetPdbDllFromInstallPath@@YAPAUHINSTANCE__@@XZ 1002e770 f   MSVCRTD:pdblkup.obj
 0002:0001da60       ?GetPdbDllPathFromFilePath@@YAHPB_WPA_WI@Z 1002ea60 f   MSVCRTD:pdblkup.obj
 0002:0001f950       __unwindfunclet$??$?0AAHUDeviceStat@@@?$_Tree_temp_node@V?$allocator@U?$_Tree_node@U?$pair@$$CBHUDeviceStat@@@std@@PAX@std@@@std@@@std@@QAE@AAV?$allocator@U?$_Tree_node@U?$pair@$$CBHUDeviceStat@@@std@@PAX@std@@@1@PAU?$_Tree_node@U?$pair@$$CBHUDeviceStat@@@std@@PAX@1@AAH$$QAUDeviceStat@@@Z$0 10030950 f   vJoyInterface.obj
 0002:0001f95d       __ehhandler$??$?0AAHUDeviceStat@@@?$_Tree_temp_node@V?$allocator@U?$_Tree_node@U?$pair@$$CBHUDeviceStat@@@std@@PAX@std@@@std@@@std@@QAE@AAV?$allocator@U?$_Tree_node@U?$pair@$$CBHUDeviceStat@@@std@@PAX@std@@@1@PAU?$_Tree_node@U?$pair@$$CBHUDeviceStat@@@std@@PAX@1@AAH$$QAUDeviceStat@@@Z 1003095d f   vJoyInterface.obj
 0002:0001f990       __ehhandler$??$?0ABH$0A@@?$tuple@ABH@std@@QAE@ABH@Z 10030990 f   vJoyInterface.obj
 0002:0001f9c0       __unwindfunclet$??$?0ABUpiecewise_construct_t@std@@V?$tuple@$$QAH@1@V?$tuple@$$V@1@@?$_Tree_temp_node@V?$allocator@U?$_Tree_node@U?$pair@$$CBHUDeviceStat@@@std@@PAX@std@@@std@@@std@@QAE@AAV?$allocator@U?$_Tree_node@U?$pair@$$CBHUDeviceStat@@@std@@PAX@std@@@1@PAU?$_Tree_node@U?$pair@$$CBHUDeviceStat@@@std@@PAX@1@ABUpiecewise_construct_t@1@$$QAV?$tuple@$$QAH@1@$$QAV?$tuple@$$V@1@@Z$0 100309c0 f   vJoyInterface.obj
 0002:0001f9cd       __ehhandler$??$?0ABUpiecewise_construct_t@std@@V?$tuple@$$QAH@1@V?$tuple@$$V@1@@?$_Tree_temp_node@V?$allocator@U?$_Tree_node@U?$pair@$$CBHUDeviceStat@@@std@@PAX@std@@@std@@@std@@QAE@AAV?$allocator@U?$_Tree_node@U?$pair@$$CBHUDeviceStat@@@std@@PAX@std@@@1@PAU?$_Tree_node@U?$pair@$$CBHUDeviceStat@@@std@@PAX@1@ABUpiecewise_construct_t@1@$$QAV?$tuple@$$QAH@1@$$QAV?$tuple@$$V@1@@Z 100309cd f   vJoyInterface.obj
 0002:0001fa00       __unwindfunclet$??$?0ABUpiecewise_construct_t@std@@V?$tuple@ABH@1@V?$tuple@$$V@1@@?$_Tree_temp_node@V?$allocator@U?$_Tree_node@U?$pair@$$CBHUDeviceStat@@@std@@PAX@std@@@std@@@std@@QAE@AAV?$allocator@U?$_Tree_node@U?$pair@$$CBHUDeviceStat@@@std@@PAX@std@@@1@PAU?$_Tree_node@U?$pair@$$CBHUDeviceStat@@@std@@PAX@1@ABUpiecewise_construct_t@1@$$QAV?$tuple@ABH@1@$$QAV?$tuple@$$V@1@@Z$0 10030a00 f   vJoyInterface.obj
 0002:0001fa0d       __ehhandler$??$?0ABUpiecewise_construct_t@std@@V?$tuple@ABH@1@V?$tuple@$$V@1@@?$_Tree_temp_node@V?$allocator@U?$_Tree_node@U?$pair@$$CBHUDeviceStat@@@std@@PAX@std@@@std@@@std@@QAE@AAV?$allocator@U?$_Tree_node@U?$pair@$$CBHUDeviceStat@@@std@@PAX@std@@@1@PAU?$_Tree_node@U?$pair@$$CBHUDeviceStat@@@std@@PAX@1@ABUpiecewise_construct_t@1@$$QAV?$tuple@ABH@1@$$QAV?$tuple@$$V@1@@Z 10030a0d f   vJoyInterface.obj
 0002:0001fa40       __ehhandler$??$?0H$$V$0A@@?$tuple@$$QAH@std@@QAE@$$QAH@Z 10030a40 f   vJoyInterface.obj
 0002:0001fa70       __ehhandler$??$_Deallocate@$07$0A@@std@@YAXPAXI@Z 10030a70 f   vJoyInterface.obj
 0002:0001faa0       __ehhandler$??$_Deallocate_plain@V?$allocator@U_Container_proxy@std@@@std@@@std@@YAXAAV?$allocator@U_Container_proxy@std@@@0@QAU_Container_proxy@0@@Z 10030aa0 f   vJoyInterface.obj
 0002:0001fad0       __ehhandler$??$_Eqrange@H@?$_Tree@V?$_Tmap_traits@HUDeviceStat@@U?$less@H@std@@V?$allocator@U?$pair@$$CBHUDeviceStat@@@std@@@3@$0A@@std@@@std@@IBE?AU?$pair@PAU?$_Tree_node@U?$pair@$$CBHUDeviceStat@@@std@@PAX@std@@PAU12@@1@ABH@Z 10030ad0 f   vJoyInterface.obj
 0002:0001fb00       __ehhandler$??$_Freenode0@V?$allocator@U?$_Tree_node@U?$pair@$$CBHUDeviceStat@@@std@@PAX@std@@@std@@@?$_Tree_node@U?$pair@$$CBHUDeviceStat@@@std@@PAX@std@@SAXAAV?$allocator@U?$_Tree_node@U?$pair@$$CBHUDeviceStat@@@std@@PAX@std@@@1@PAU01@@Z 10030b00 f   vJoyInterface.obj
 0002:0001fb30       __ehhandler$??$_Freenode0@V?$allocator@U?$_Tree_node@U?$pair@$$CBHW4FFB_EFFECTS@@@std@@PAX@std@@@std@@@?$_Tree_node@U?$pair@$$CBHW4FFB_EFFECTS@@@std@@PAX@std@@SAXAAV?$allocator@U?$_Tree_node@U?$pair@$$CBHW4FFB_EFFECTS@@@std@@PAX@std@@@1@PAU01@@Z 10030b30 f   vJoyInterface.obj
 0002:0001fb60       __ehhandler$??$_Freenode@V?$allocator@U?$_Tree_node@U?$pair@$$CBHUDeviceStat@@@std@@PAX@std@@@std@@@?$_Tree_node@U?$pair@$$CBHUDeviceStat@@@std@@PAX@std@@SAXAAV?$allocator@U?$_Tree_node@U?$pair@$$CBHUDeviceStat@@@std@@PAX@std@@@1@PAU01@@Z 10030b60 f   vJoyInterface.obj
 0002:0001fb90       __ehhandler$??$_Freenode@V?$allocator@U?$_Tree_node@U?$pair@$$CBHW4FFB_EFFECTS@@@std@@PAX@std@@@std@@@?$_Tree_node@U?$pair@$$CBHW4FFB_EFFECTS@@@std@@PAX@std@@SAXAAV?$allocator@U?$_Tree_node@U?$pair@$$CBHW4FFB_EFFECTS@@@std@@PAX@std@@@1@PAU01@@Z 10030b90 f   vJoyInterface.obj
 0002:0001fbc0       __unwindfunclet$??0?$_Tree_temp_node_alloc@V?$allocator@U?$_Tree_node@U?$pair@$$CBHUDeviceStat@@@std@@PAX@std@@@std@@@std@@QAE@AAV?$allocator@U?$_Tree_node@U?$pair@$$CBHUDeviceStat@@@std@@PAX@std@@@1@@Z$0 10030bc0 f   vJoyInterface.obj
 0002:0001fbcd       __ehhandler$??0?$_Tree_temp_node_alloc@V?$allocator@U?$_Tree_node@U?$pair@$$CBHUDeviceStat@@@std@@PAX@std@@@std@@@std@@QAE@AAV?$allocator@U?$_Tree_node@U?$pair@$$CBHUDeviceStat@@@std@@PAX@std@@@1@@Z 10030bcd f   vJoyInterface.obj
 0002:0001fc00       __ehhandler$??1?$_Alloc_construct_ptr@V?$allocator@U?$_Tree_node@U?$pair@$$CBHUDeviceStat@@@std@@PAX@std@@@std@@@std@@QAE@XZ 10030c00 f   vJoyInterface.obj
 0002:0001fc30       __ehhandler$??1?$_Tree_temp_node@V?$allocator@U?$_Tree_node@U?$pair@$$CBHUDeviceStat@@@std@@PAX@std@@@std@@@std@@QAE@XZ 10030c30 f   vJoyInterface.obj
 0002:0001fc60       __unwindfunclet$?AreControlsInit@@YAHI@Z$0 10030c60 f   vJoyInterface.obj
 0002:0001fc87       __ehhandler$?AreControlsInit@@YAHI@Z 10030c87 f   vJoyInterface.obj
 0002:0001fcc0       __unwindfunclet$?Get_PreparsedData@@YAHHPAPAU_HIDP_PREPARSED_DATA@@@Z$0 10030cc0 f   vJoyInterface.obj
 0002:0001fcd0       __ehhandler$?Get_PreparsedData@@YAHHPAPAU_HIDP_PREPARSED_DATA@@@Z 10030cd0 f   vJoyInterface.obj
 0002:0001fd10       __unwindfunclet$?Get_h@@YAPAXH@Z$0 10030d10 f   vJoyInterface.obj
 0002:0001fd20       __ehhandler$?Get_h@@YAPAXH@Z 10030d20 f   vJoyInterface.obj
 0002:0001fd50       __unwindfunclet$?Get_hNotify@@YAPAXH@Z$0 10030d50 f   vJoyInterface.obj
 0002:0001fd60       __ehhandler$?Get_hNotify@@YAPAXH@Z 10030d60 f   vJoyInterface.obj
 0002:0001fd90       __unwindfunclet$?Get_stat@@YA?AW4VjdStat@@H@Z$0 10030d90 f   vJoyInterface.obj
 0002:0001fda0       __ehhandler$?Get_stat@@YA?AW4VjdStat@@H@Z 10030da0 f   vJoyInterface.obj
 0002:0001fdd0       __unwindfunclet$?SavePosition@@YAXIPAX@Z$0 10030dd0 f   vJoyInterface.obj
 0002:0001fdf7       __ehhandler$?SavePosition@@YAXIPAX@Z 10030df7 f   vJoyInterface.obj
 0002:0001fe30       __unwindfunclet$?Set_PreparsedData@@YAHH@Z$0 10030e30 f   vJoyInterface.obj
 0002:0001fe40       __ehhandler$?Set_PreparsedData@@YAHH@Z 10030e40 f   vJoyInterface.obj
 0002:0001fe70       __unwindfunclet$?Set_h@@YAXHPAX@Z$0 10030e70 f   vJoyInterface.obj
 0002:0001fe80       __ehhandler$?Set_h@@YAXHPAX@Z 10030e80 f   vJoyInterface.obj
 0002:0001feb0       __unwindfunclet$?Set_hNotify@@YAXHPAX@Z$0 10030eb0 f   vJoyInterface.obj
 0002:0001fec0       __ehhandler$?Set_hNotify@@YAXHPAX@Z 10030ec0 f   vJoyInterface.obj
 0002:0001fef0       __unwindfunclet$?Set_stat@@YAXHW4VjdStat@@@Z$0 10030ef0 f   vJoyInterface.obj
 0002:0001ff00       __ehhandler$?Set_stat@@YAXHW4VjdStat@@@Z 10030f00 f   vJoyInterface.obj
 0002:0001ff30       __unwindfunclet$?Sync_Position@@YAXH@Z$0 10030f30 f   vJoyInterface.obj
 0002:0001ff40       __ehhandler$?Sync_Position@@YAXH@Z 10030f40 f   vJoyInterface.obj
 0002:0001ff80       __unwindfunclet$?Update@@YAHI@Z$0 10030f80 f   vJoyInterface.obj
 0002:0001ffa2       __unwindfunclet$?Update@@YAHI@Z$1 10030fa2 f   vJoyInterface.obj
 0002:0001ffc9       __ehhandler$?Update@@YAHI@Z 10030fc9 f   vJoyInterface.obj
 0002:00020010       __unwindfunclet$?_Alloc_sentinel_and_proxy@?$_Tree@V?$_Tmap_traits@HUDeviceStat@@U?$less@H@std@@V?$allocator@U?$pair@$$CBHUDeviceStat@@@std@@@3@$0A@@std@@@std@@IAEXXZ$0 10031010 f   vJoyInterface.obj
 0002:0002001d       __ehhandler$?_Alloc_sentinel_and_proxy@?$_Tree@V?$_Tmap_traits@HUDeviceStat@@U?$less@H@std@@V?$allocator@U?$pair@$$CBHUDeviceStat@@@std@@@3@$0A@@std@@@std@@IAEXXZ 1003101d f   vJoyInterface.obj
 0002:00020050       __unwindfunclet$?_Alloc_sentinel_and_proxy@?$_Tree@V?$_Tmap_traits@HW4FFB_EFFECTS@@U?$less@H@std@@V?$allocator@U?$pair@$$CBHW4FFB_EFFECTS@@@std@@@3@$0A@@std@@@std@@IAEXXZ$0 10031050 f   vJoyInterface.obj
 0002:0002005d       __ehhandler$?_Alloc_sentinel_and_proxy@?$_Tree@V?$_Tmap_traits@HW4FFB_EFFECTS@@U?$less@H@std@@V?$allocator@U?$pair@$$CBHW4FFB_EFFECTS@@@std@@@3@$0A@@std@@@std@@IAEXXZ 1003105d f   vJoyInterface.obj
 0002:00020090       __ehhandler$?_Erase@?$_Tree@V?$_Tmap_traits@HUDeviceStat@@U?$less@H@std@@V?$allocator@U?$pair@$$CBHUDeviceStat@@@std@@@3@$0A@@std@@@std@@AAEIU?$pair@PAU?$_Tree_node@U?$pair@$$CBHUDeviceStat@@@std@@PAX@std@@PAU12@@2@@Z 10031090 f   vJoyInterface.obj
 0002:000200c0       __unwindfunclet$?vJoyDeviceEntry@@YAHH@Z$0 100310c0 f   vJoyInterface.obj
 0002:000200d0       __ehhandler$?vJoyDeviceEntry@@YAHH@Z 100310d0 f   vJoyInterface.obj
 0002:00020110       __unwindfunclet$?vJoyDeviceRemove@@YAHH@Z$0 10031110 f   vJoyInterface.obj
 0002:00020120       __ehhandler$?vJoyDeviceRemove@@YAHH@Z 10031120 f   vJoyInterface.obj
 0002:00021190       ??__FmFfbEffect@@YAXXZ     10032190 f   vJoyInterface.obj
 0002:000211e0       ??__FvJoyDevices@@YAXXZ    100321e0 f   vJoyInterface.obj
 0003:00000104       ?vJoyDevices$initializer$@@3P6AXXZA 10034104     vJoyInterface.obj
 0003:00000108       ?mFfbEffect$initializer$@@3P6AXXZA 10034108     vJoyInterface.obj
 0003:00000943       ?piecewise_construct@std@@3Upiecewise_construct_t@1@B 10034943     vJoyInterface.obj
 0003:00002c28       ?_RTC_ErrorMessages@@3QBQBDB 10036c28     MSVCRTD:error.obj
 0003:00002c40       ?_RTC_NoFalsePositives@@3QBHB 10036c40     MSVCRTD:error.obj
 0003:00002c58       ?stack_premsg@@3QBDB       10036c58     MSVCRTD:error.obj
 0003:00002c74       ?stack_postmsg@@3QBDB      10036c74     MSVCRTD:error.obj
 0003:00002c88       ?uninit_premsg@@3QBDB      10036c88     MSVCRTD:error.obj
 0003:00002c98       ?uninit_postmsg@@3QBDB     10036c98     MSVCRTD:error.obj
 0003:000032e8       _GS_ExceptionPointers      100372e8     MSVCRTD:gs_report.obj
 0003:000032f4       ?_RTC_errlist@@3QBQBDB     100372f4     MSVCRTD:userapi.obj
 0003:000033d8       ?mspdbName@@3QB_WB         100373d8     MSVCRTD:pdblkup.obj
 0003:000033fc       ?debugCrtFileName@@3QB_WB  100373fc     MSVCRTD:pdblkup.obj
 0003:00003588       ?dllExt@?1??GetPdbDllPathFromFilePath@@YAHPB_WPA_WI@Z@4QB_WB 10037588     MSVCRTD:pdblkup.obj
 0003:00003594       ?mspdbFilename@?1??GetPdbDllPathFromFilePath@@YAHPB_WPA_WI@Z@4QB_WB 10037594     MSVCRTD:pdblkup.obj
 0003:00004088       __RTC_InitBase.rtc$IMZ     10038088     vJoyInterface.obj
 0003:00004394       __RTC_Shutdown.rtc$TMZ     10038394     vJoyInterface.obj
 0003:000045a0       __unwindtable$?SavePosition@@YAXIPAX@Z 100385a0     vJoyInterface.obj
 0003:000045a8       __ehfuncinfo$?SavePosition@@YAXIPAX@Z 100385a8     vJoyInterface.obj
 0003:000045d0       __unwindtable$?Update@@YAHI@Z 100385d0     vJoyInterface.obj
 0003:000045e0       __ehfuncinfo$?Update@@YAHI@Z 100385e0     vJoyInterface.obj
 0003:0000460c       __unwindtable$?AreControlsInit@@YAHI@Z 1003860c     vJoyInterface.obj
 0003:00004614       __ehfuncinfo$?AreControlsInit@@YAHI@Z 10038614     vJoyInterface.obj
 0003:0000463c       __unwindtable$?vJoyDeviceEntry@@YAHH@Z 1003863c     vJoyInterface.obj
 0003:00004644       __ehfuncinfo$?vJoyDeviceEntry@@YAHH@Z 10038644     vJoyInterface.obj
 0003:0000466c       __unwindtable$?vJoyDeviceRemove@@YAHH@Z 1003866c     vJoyInterface.obj
 0003:00004674       __ehfuncinfo$?vJoyDeviceRemove@@YAHH@Z 10038674     vJoyInterface.obj
 0003:0000469c       __unwindtable$?Set_PreparsedData@@YAHH@Z 1003869c     vJoyInterface.obj
 0003:000046a4       __ehfuncinfo$?Set_PreparsedData@@YAHH@Z 100386a4     vJoyInterface.obj
 0003:000046cc       __unwindtable$?Get_PreparsedData@@YAHHPAPAU_HIDP_PREPARSED_DATA@@@Z 100386cc     vJoyInterface.obj
 0003:000046d4       __ehfuncinfo$?Get_PreparsedData@@YAHHPAPAU_HIDP_PREPARSED_DATA@@@Z 100386d4     vJoyInterface.obj
 0003:000046fc       __unwindtable$?Set_h@@YAXHPAX@Z 100386fc     vJoyInterface.obj
 0003:00004704       __ehfuncinfo$?Set_h@@YAXHPAX@Z 10038704     vJoyInterface.obj
 0003:0000472c       __unwindtable$?Sync_Position@@YAXH@Z 1003872c     vJoyInterface.obj
 0003:00004734       __ehfuncinfo$?Sync_Position@@YAXH@Z 10038734     vJoyInterface.obj
 0003:0000475c       __unwindtable$?Get_h@@YAPAXH@Z 1003875c     vJoyInterface.obj
 0003:00004764       __ehfuncinfo$?Get_h@@YAPAXH@Z 10038764     vJoyInterface.obj
 0003:0000478c       __unwindtable$?Set_stat@@YAXHW4VjdStat@@@Z 1003878c     vJoyInterface.obj
 0003:00004794       __ehfuncinfo$?Set_stat@@YAXHW4VjdStat@@@Z 10038794     vJoyInterface.obj
 0003:000047bc       __unwindtable$?Get_stat@@YA?AW4VjdStat@@H@Z 100387bc     vJoyInterface.obj
 0003:000047c4       __ehfuncinfo$?Get_stat@@YA?AW4VjdStat@@H@Z 100387c4     vJoyInterface.obj
 0003:000047ec       __unwindtable$?Set_hNotify@@YAXHPAX@Z 100387ec     vJoyInterface.obj
 0003:000047f4       __ehfuncinfo$?Set_hNotify@@YAXHPAX@Z 100387f4     vJoyInterface.obj
 0003:0000481c       __unwindtable$?Get_hNotify@@YAPAXH@Z 1003881c     vJoyInterface.obj
 0003:00004824       __ehfuncinfo$?Get_hNotify@@YAPAXH@Z 10038824     vJoyInterface.obj
 0003:0000484c       __ehfuncinfo$?_Erase@?$_Tree@V?$_Tmap_traits@HUDeviceStat@@U?$less@H@std@@V?$allocator@U?$pair@$$CBHUDeviceStat@@@std@@@3@$0A@@std@@@std@@AAEIU?$pair@PAU?$_Tree_node@U?$pair@$$CBHUDeviceStat@@@std@@PAX@std@@PAU12@@2@@Z 1003884c     vJoyInterface.obj
 0003:00004874       __unwindtable$?_Alloc_sentinel_and_proxy@?$_Tree@V?$_Tmap_traits@HUDeviceStat@@U?$less@H@std@@V?$allocator@U?$pair@$$CBHUDeviceStat@@@std@@@3@$0A@@std@@@std@@IAEXXZ 10038874     vJoyInterface.obj
 0003:0000487c       __ehfuncinfo$?_Alloc_sentinel_and_proxy@?$_Tree@V?$_Tmap_traits@HUDeviceStat@@U?$less@H@std@@V?$allocator@U?$pair@$$CBHUDeviceStat@@@std@@@3@$0A@@std@@@std@@IAEXXZ 1003887c     vJoyInterface.obj
 0003:000048a4       __unwindtable$?_Alloc_sentinel_and_proxy@?$_Tree@V?$_Tmap_traits@HW4FFB_EFFECTS@@U?$less@H@std@@V?$allocator@U?$pair@$$CBHW4FFB_EFFECTS@@@std@@@3@$0A@@std@@@std@@IAEXXZ 100388a4     vJoyInterface.obj
 0003:000048ac       __ehfuncinfo$?_Alloc_sentinel_and_proxy@?$_Tree@V?$_Tmap_traits@HW4FFB_EFFECTS@@U?$less@H@std@@V?$allocator@U?$pair@$$CBHW4FFB_EFFECTS@@@std@@@3@$0A@@std@@@std@@IAEXXZ 100388ac     vJoyInterface.obj
 0003:000048d4       __ehfuncinfo$??$_Eqrange@H@?$_Tree@V?$_Tmap_traits@HUDeviceStat@@U?$less@H@std@@V?$allocator@U?$pair@$$CBHUDeviceStat@@@std@@@3@$0A@@std@@@std@@IBE?AU?$pair@PAU?$_Tree_node@U?$pair@$$CBHUDeviceStat@@@std@@PAX@std@@PAU12@@1@ABH@Z 100388d4     vJoyInterface.obj
 0003:000048fc       __ehfuncinfo$??$_Freenode@V?$allocator@U?$_Tree_node@U?$pair@$$CBHUDeviceStat@@@std@@PAX@std@@@std@@@?$_Tree_node@U?$pair@$$CBHUDeviceStat@@@std@@PAX@std@@SAXAAV?$allocator@U?$_Tree_node@U?$pair@$$CBHUDeviceStat@@@std@@PAX@std@@@1@PAU01@@Z 100388fc     vJoyInterface.obj
 0003:00004924       __ehfuncinfo$??$_Freenode@V?$allocator@U?$_Tree_node@U?$pair@$$CBHW4FFB_EFFECTS@@@std@@PAX@std@@@std@@@?$_Tree_node@U?$pair@$$CBHW4FFB_EFFECTS@@@std@@PAX@std@@SAXAAV?$allocator@U?$_Tree_node@U?$pair@$$CBHW4FFB_EFFECTS@@@std@@PAX@std@@@1@PAU01@@Z 10038924     vJoyInterface.obj
 0003:0000494c       __ehfuncinfo$??$_Freenode0@V?$allocator@U?$_Tree_node@U?$pair@$$CBHW4FFB_EFFECTS@@@std@@PAX@std@@@std@@@?$_Tree_node@U?$pair@$$CBHW4FFB_EFFECTS@@@std@@PAX@std@@SAXAAV?$allocator@U?$_Tree_node@U?$pair@$$CBHW4FFB_EFFECTS@@@std@@PAX@std@@@1@PAU01@@Z 1003894c     vJoyInterface.obj
 0003:00004974       __ehfuncinfo$??$_Deallocate_plain@V?$allocator@U_Container_proxy@std@@@std@@@std@@YAXAAV?$allocator@U_Container_proxy@std@@@0@QAU_Container_proxy@0@@Z 10038974     vJoyInterface.obj
 0003:0000499c       __ehfuncinfo$??1?$_Alloc_construct_ptr@V?$allocator@U?$_Tree_node@U?$pair@$$CBHUDeviceStat@@@std@@PAX@std@@@std@@@std@@QAE@XZ 1003899c     vJoyInterface.obj
 0003:000049c4       __unwindtable$??0?$_Tree_temp_node_alloc@V?$allocator@U?$_Tree_node@U?$pair@$$CBHUDeviceStat@@@std@@PAX@std@@@std@@@std@@QAE@AAV?$allocator@U?$_Tree_node@U?$pair@$$CBHUDeviceStat@@@std@@PAX@std@@@1@@Z 100389c4     vJoyInterface.obj
 0003:000049cc       __ehfuncinfo$??0?$_Tree_temp_node_alloc@V?$allocator@U?$_Tree_node@U?$pair@$$CBHUDeviceStat@@@std@@PAX@std@@@std@@@std@@QAE@AAV?$allocator@U?$_Tree_node@U?$pair@$$CBHUDeviceStat@@@std@@PAX@std@@@1@@Z 100389cc     vJoyInterface.obj
 0003:000049f4       __ehfuncinfo$??1?$_Tree_temp_node@V?$allocator@U?$_Tree_node@U?$pair@$$CBHUDeviceStat@@@std@@PAX@std@@@std@@@std@@QAE@XZ 100389f4     vJoyInterface.obj
 0003:00004a1c       __unwindtable$??$?0ABUpiecewise_construct_t@std@@V?$tuple@ABH@1@V?$tuple@$$V@1@@?$_Tree_temp_node@V?$allocator@U?$_Tree_node@U?$pair@$$CBHUDeviceStat@@@std@@PAX@std@@@std@@@std@@QAE@AAV?$allocator@U?$_Tree_node@U?$pair@$$CBHUDeviceStat@@@std@@PAX@std@@@1@PAU?$_Tree_node@U?$pair@$$CBHUDeviceStat@@@std@@PAX@1@ABUpiecewise_construct_t@1@$$QAV?$tuple@ABH@1@$$QAV?$tuple@$$V@1@@Z 10038a1c     vJoyInterface.obj
 0003:00004a24       __ehfuncinfo$??$?0ABUpiecewise_construct_t@std@@V?$tuple@ABH@1@V?$tuple@$$V@1@@?$_Tree_temp_node@V?$allocator@U?$_Tree_node@U?$pair@$$CBHUDeviceStat@@@std@@PAX@std@@@std@@@std@@QAE@AAV?$allocator@U?$_Tree_node@U?$pair@$$CBHUDeviceStat@@@std@@PAX@std@@@1@PAU?$_Tree_node@U?$pair@$$CBHUDeviceStat@@@std@@PAX@1@ABUpiecewise_construct_t@1@$$QAV?$tuple@ABH@1@$$QAV?$tuple@$$V@1@@Z 10038a24     vJoyInterface.obj
 0003:00004a4c       __unwindtable$??$?0ABUpiecewise_construct_t@std@@V?$tuple@$$QAH@1@V?$tuple@$$V@1@@?$_Tree_temp_node@V?$allocator@U?$_Tree_node@U?$pair@$$CBHUDeviceStat@@@std@@PAX@std@@@std@@@std@@QAE@AAV?$allocator@U?$_Tree_node@U?$pair@$$CBHUDeviceStat@@@std@@PAX@std@@@1@PAU?$_Tree_node@U?$pair@$$CBHUDeviceStat@@@std@@PAX@1@ABUpiecewise_construct_t@1@$$QAV?$tuple@$$QAH@1@$$QAV?$tuple@$$V@1@@Z 10038a4c     vJoyInterface.obj
 0003:00004a54       __ehfuncinfo$??$?0ABUpiecewise_construct_t@std@@V?$tuple@$$QAH@1@V?$tuple@$$V@1@@?$_Tree_temp_node@V?$allocator@U?$_Tree_node@U?$pair@$$CBHUDeviceStat@@@std@@PAX@std@@@std@@@std@@QAE@AAV?$allocator@U?$_Tree_node@U?$pair@$$CBHUDeviceStat@@@std@@PAX@std@@@1@PAU?$_Tree_node@U?$pair@$$CBHUDeviceStat@@@std@@PAX@1@ABUpiecewise_construct_t@1@$$QAV?$tuple@$$QAH@1@$$QAV?$tuple@$$V@1@@Z 10038a54     vJoyInterface.obj
 0003:00004a7c       __ehfuncinfo$??$_Freenode0@V?$allocator@U?$_Tree_node@U?$pair@$$CBHUDeviceStat@@@std@@PAX@std@@@std@@@?$_Tree_node@U?$pair@$$CBHUDeviceStat@@@std@@PAX@std@@SAXAAV?$allocator@U?$_Tree_node@U?$pair@$$CBHUDeviceStat@@@std@@PAX@std@@@1@PAU01@@Z 10038a7c     vJoyInterface.obj
 0003:00004aa4       __ehfuncinfo$??$_Deallocate@$07$0A@@std@@YAXPAXI@Z 10038aa4     vJoyInterface.obj
 0003:00004acc       __unwindtable$??$?0AAHUDeviceStat@@@?$_Tree_temp_node@V?$allocator@U?$_Tree_node@U?$pair@$$CBHUDeviceStat@@@std@@PAX@std@@@std@@@std@@QAE@AAV?$allocator@U?$_Tree_node@U?$pair@$$CBHUDeviceStat@@@std@@PAX@std@@@1@PAU?$_Tree_node@U?$pair@$$CBHUDeviceStat@@@std@@PAX@1@AAH$$QAUDeviceStat@@@Z 10038acc     vJoyInterface.obj
 0003:00004ad4       __ehfuncinfo$??$?0AAHUDeviceStat@@@?$_Tree_temp_node@V?$allocator@U?$_Tree_node@U?$pair@$$CBHUDeviceStat@@@std@@PAX@std@@@std@@@std@@QAE@AAV?$allocator@U?$_Tree_node@U?$pair@$$CBHUDeviceStat@@@std@@PAX@std@@@1@PAU?$_Tree_node@U?$pair@$$CBHUDeviceStat@@@std@@PAX@1@AAH$$QAUDeviceStat@@@Z 10038ad4     vJoyInterface.obj
 0003:00004afc       __ehfuncinfo$??$?0ABH$0A@@?$tuple@ABH@std@@QAE@ABH@Z 10038afc     vJoyInterface.obj
 0003:00004b24       __ehfuncinfo$??$?0H$$V$0A@@?$tuple@$$QAH@std@@QAE@$$QAH@Z 10038b24     vJoyInterface.obj
 0003:00004bd8       __sehtable$___scrt_is_nonwritable_in_current_image 10038bd8     MSVCRTD:utility.obj
 0003:00004bf8       __sehtable$?dllmain_crt_process_attach@@YAHQAUHINSTANCE__@@QAX@Z 10038bf8     MSVCRTD:dll_dllmain.obj
 0003:00004c18       __sehtable$?dllmain_crt_process_detach@@YAH_N@Z 10038c18     MSVCRTD:dll_dllmain.obj
 0003:00004c48       __sehtable$?dllmain_dispatch@@YAHQAUHINSTANCE__@@KQAX@Z 10038c48     MSVCRTD:dll_dllmain.obj
 0003:00004c90       __sehtable$?notify_debugger@@YAXABUtagEXCEPTION_VISUALCPP_DEBUG_INFO@@@Z 10038c90     MSVCRTD:error.obj
 0003:00004e70       .edata                     10038e70     vJoyInterface.exp
 0003:00004e98       rgpv                       10038e98     vJoyInterface.exp
 0003:00004f64       rgszName                   10038f64     vJoyInterface.exp
 0003:00005030       rgwOrd                     10039030     vJoyInterface.exp
 0003:00005096       szName                     10039096     vJoyInterface.exp
 0003:000050a8       $N00001                    100390a8     vJoyInterface.exp
 0003:000050b3       $N00002                    100390b3     vJoyInterface.exp
 0003:000050bf       $N00003                    100390bf     vJoyInterface.exp
 0003:000050cc       $N00004                    100390cc     vJoyInterface.exp
 0003:000050dd       $N00005                    100390dd     vJoyInterface.exp
 0003:000050e6       $N00006                    100390e6     vJoyInterface.exp
 0003:000050ee       $N00007                    100390ee     vJoyInterface.exp
 0003:000050fc       $N00008                    100390fc     vJoyInterface.exp
 0003:0000510a       $N00009                    1003910a     vJoyInterface.exp
 0003:00005119       $N00010                    10039119     vJoyInterface.exp
 0003:00005123       $N00011                    10039123     vJoyInterface.exp
 0003:00005130       $N00012                    10039130     vJoyInterface.exp
 0003:0000513c       $N00013                    1003913c     vJoyInterface.exp
 0003:0000514b       $N00014                    1003914b     vJoyInterface.exp
 0003:0000515e       $N00015                    1003915e     vJoyInterface.exp
 0003:0000516e       $N00016                    1003916e     vJoyInterface.exp
 0003:0000517f       $N00017                    1003917f     vJoyInterface.exp
 0003:0000518e       $N00018                    1003918e     vJoyInterface.exp
 0003:0000519f       $N00019                    1003919f     vJoyInterface.exp
 0003:000051ac       $N00020                    100391ac     vJoyInterface.exp
 0003:000051b7       $N00021                    100391b7     vJoyInterface.exp
 0003:000051cc       $N00022                    100391cc     vJoyInterface.exp
 0003:000051d8       $N00023                    100391d8     vJoyInterface.exp
 0003:000051e8       $N00024                    100391e8     vJoyInterface.exp
 0003:000051f6       $N00025                    100391f6     vJoyInterface.exp
 0003:00005204       $N00026                    10039204     vJoyInterface.exp
 0003:00005217       $N00027                    10039217     vJoyInterface.exp
 0003:0000522b       $N00028                    1003922b     vJoyInterface.exp
 0003:0000523f       $N00029                    1003923f     vJoyInterface.exp
 0003:0000524c       $N00030                    1003924c     vJoyInterface.exp
 0003:00005266       $N00031                    10039266     vJoyInterface.exp
 0003:00005278       $N00032                    10039278     vJoyInterface.exp
 0003:0000528d       $N00033                    1003928d     vJoyInterface.exp
 0003:000052a7       $N00034                    100392a7     vJoyInterface.exp
 0003:000052b6       $N00035                    100392b6     vJoyInterface.exp
 0003:000052c2       $N00036                    100392c2     vJoyInterface.exp
 0003:000052d4       $N00037                    100392d4     vJoyInterface.exp
 0003:000052e6       $N00038                    100392e6     vJoyInterface.exp
 0003:000052f4       $N00039                    100392f4     vJoyInterface.exp
 0003:000052fd       $N00040                    100392fd     vJoyInterface.exp
 0003:0000530a       $N00041                    1003930a     vJoyInterface.exp
 0003:00005314       $N00042                    10039314     vJoyInterface.exp
 0003:0000531d       $N00043                    1003931d     vJoyInterface.exp
 0003:00005325       $N00044                    10039325     vJoyInterface.exp
 0003:0000532c       $N00045                    1003932c     vJoyInterface.exp
 0003:00005337       $N00046                    10039337     vJoyInterface.exp
 0003:00005342       $N00047                    10039342     vJoyInterface.exp
 0003:0000534c       $N00048                    1003934c     vJoyInterface.exp
 0003:00005358       $N00049                    10039358     vJoyInterface.exp
 0003:00005362       $N00050                    10039362     vJoyInterface.exp
 0003:0000536e       $N00051                    1003936e     vJoyInterface.exp
 0004:00000004       ?szWindowClass@@3PADA      1003a004     vJoyInterface.obj
 0004:00000020       ?szTitle@@3PADA            1003a020     vJoyInterface.obj
 0004:000004a0       ?cnt_complete@?1??DeviceChange@@9@4HA 1003a4a0     vJoyInterface.obj
 0004:000004a4       ?cnt_arrive@?1??DeviceChange@@9@4HA 1003a4a4     vJoyInterface.obj
 0004:000004a8       ?StatNS@?1??GetDeviceNameSpace@@YAHPAPADPAHHPAK@Z@4PADA 1003a4a8     vJoyInterface.obj
 0004:000004ec       ?is_initialized_as_dll@@3_NA 1003a4ec     MSVCRTD:utility.obj
 0004:000004ed       ?module_local_atexit_table_initialized@@3_NA 1003a4ed     MSVCRTD:utility.obj
 0004:000004f0       ?module_local_atexit_table@@3U_onexit_table_t@@A 1003a4f0     MSVCRTD:utility.obj
 0004:000004fc       ?module_local_at_quick_exit_table@@3U_onexit_table_t@@A 1003a4fc     MSVCRTD:utility.obj
 0004:0000050f       ?init@?1??_RTC_InitBase@@9@4_NA 1003a50f     MSVCRTD:init.obj
 0004:00000510       ?__proc_attached@@3HA      1003a510     MSVCRTD:dll_dllmain.obj
 0004:00000528       _GS_ExceptionRecord        1003a528     MSVCRTD:gs_report.obj
 0004:00000578       _GS_ContextRecord          1003a578     MSVCRTD:gs_report.obj
 0004:000008e4       ?_RTC_ErrorReportFunc@@3P6AHHPBDH00ZZA 1003a8e4     MSVCRTD:userapi.obj
 0004:000008e8       ?_RTC_ErrorReportFuncW@@3P6AHHPB_WH00ZZA 1003a8e8     MSVCRTD:userapi.obj
 0004:000008fc       ?mspdb@@3PAUHINSTANCE__@@A 1003a8fc     MSVCRTD:pdblkup.obj
 0004:00000900       ?alreadyTried@?1??GetPdbDll@@YAPAUHINSTANCE__@@XZ@4_NA 1003a900     MSVCRTD:pdblkup.obj
 0004:00000901       ?PDBOK@?1??_RTC_GetSrcLine@@YAHPAEPA_WKPAH1K@Z@4_NA 1003a901     MSVCRTD:pdblkup.obj
 0005:000008ae       .idata$6                   1003b8ae     setupapi:SETUPAPI.dll
 0005:000009f4       .idata$6                   1003b9f4     hid:HID.DLL
 0005:00000b02       .idata$6                   1003bb02     kernel32:KERNEL32.dll
 0005:00000c3e       .idata$6                   1003bc3e     user32:USER32.dll
 0005:00000c78       .idata$6                   1003bc78     advapi32:ADVAPI32.dll
 0005:00000cda       .idata$6                   1003bcda     msvcprtd:MSVCP140D.dll
 0005:00000e2a       .idata$6                   1003be2a     vcruntimed:VCRUNTIME140D.dll
 0005:000010aa       .idata$6                   1003c0aa     ucrtd:ucrtbased.dll
 0006:00000000       __E1218CD7_targetver@h     1003d000     stdafx.obj
 0006:00000001       __3347223C_winpackagefamily@h 1003d001     stdafx.obj
 0006:00000002       __F5B671E4_winapifamily@h  1003d002     stdafx.obj
 0006:00000003       __6866F092_sdkddkver@h     1003d003     stdafx.obj
 0006:00000004       __CD417A16_concurrencysal@h 1003d004     stdafx.obj
 0006:00000005       __18C11F8D_sal@h           1003d005     stdafx.obj
 0006:00000006       __BD42D05E_vadefs@h        1003d006     stdafx.obj
 0006:00000007       __2DC9DF70_vcruntime@h     1003d007     stdafx.obj
 0006:00000008       __D7225C87_excpt@h         1003d008     stdafx.obj
 0006:00000009       __F19000F7_stdarg@h        1003d009     stdafx.obj
 0006:0000000a       __4114BAD5_specstrings_undef@h 1003d00a     stdafx.obj
 0006:0000000b       __50F9AEDC_specstrings_strict@h 1003d00b     stdafx.obj
 0006:0000000c       __BEFC0098_sdv_driverspecs@h 1003d00c     stdafx.obj
 0006:0000000d       __39A39701_driverspecs@h   1003d00d     stdafx.obj
 0006:0000000e       __B4D8BDAA_specstrings@h   1003d00e     stdafx.obj
 0006:0000000f       __04C75F1C_corecrt@h       1003d00f     stdafx.obj
 0006:00000010       __78D0C915_corecrt_wctype@h 1003d010     stdafx.obj
 0006:00000011       __6AECDA3E_ctype@h         1003d011     stdafx.obj
 0006:00000012       __B6CCE7CD_kernelspecs@h   1003d012     stdafx.obj
 0006:00000013       __201B1099_basetsd@h       1003d013     stdafx.obj
 0006:00000014       __15E49872_errno@h         1003d014     stdafx.obj
 0006:00000015       __6BB4896E_vcruntime_string@h 1003d015     stdafx.obj
 0006:00000016       __184F7456_corecrt_memcpy_s@h 1003d016     stdafx.obj
 0006:00000017       __82377222_corecrt_memory@h 1003d017     stdafx.obj
 0006:00000018       __5B29309E_corecrt_wstring@h 1003d018     stdafx.obj
 0006:00000019       __F787F5CD_string@h        1003d019     stdafx.obj
 0006:0000001a       __8C99318D_guiddef@h       1003d01a     stdafx.obj
 0006:0000001b       __A3CAA675_pshpack4@h      1003d01b     stdafx.obj
 0006:0000001c       __2611E9B9_poppack@h       1003d01c     stdafx.obj
 0006:0000001d       __A747DAC7_pshpack2@h      1003d01d     stdafx.obj
 0006:0000001e       __AAD05F11_pshpack8@h      1003d01e     stdafx.obj
 0006:0000001f       __A501649E_pshpack1@h      1003d01f     stdafx.obj
 0006:00000020       __0E9D9C0E_apiset@h        1003d020     stdafx.obj
 0006:00000021       __F9851A06_ktmtypes@h      1003d021     stdafx.obj
 0006:00000022       __9DA2B69E_winnt@h         1003d022     stdafx.obj
 0006:00000023       __E9AED855_minwindef@h     1003d023     stdafx.obj
 0006:00000024       __9668718B_windef@h        1003d024     stdafx.obj
 0006:00000025       __B47C9622_apisetcconv@h   1003d025     stdafx.obj
 0006:00000026       __77F4CE3E_minwinbase@h    1003d026     stdafx.obj
 0006:00000027       __42CF8FD5_apiquery2@h     1003d027     stdafx.obj
 0006:00000028       __A6C51434_processenv@h    1003d028     stdafx.obj
 0006:00000029       __415D7145_fileapi@h       1003d029     stdafx.obj
 0006:0000002a       __A7316A9B_fileapifromapp@h 1003d02a     stdafx.obj
 0006:0000002b       __A0359A2D_debugapi@h      1003d02b     stdafx.obj
 0006:0000002c       __28BE1226_utilapiset@h    1003d02c     stdafx.obj
 0006:0000002d       __6933B394_handleapi@h     1003d02d     stdafx.obj
 0006:0000002e       __57F09DF9_errhandlingapi@h 1003d02e     stdafx.obj
 0006:0000002f       __E0622DF9_fibersapi@h     1003d02f     stdafx.obj
 0006:00000030       __D531F6AB_namedpipeapi@h  1003d030     stdafx.obj
 0006:00000031       __ADD82BB4_profileapi@h    1003d031     stdafx.obj
 0006:00000032       __ECFC4D70_heapapi@h       1003d032     stdafx.obj
 0006:00000033       __4F41815B_ioapiset@h      1003d033     stdafx.obj
 0006:00000034       __8D44BFB7_synchapi@h      1003d034     stdafx.obj
 0006:00000035       __8CAEC090_interlockedapi@h 1003d035     stdafx.obj
 0006:00000036       __8ABF54F4_processthreadsapi@h 1003d036     stdafx.obj
 0006:00000037       __1462A586_sysinfoapi@h    1003d037     stdafx.obj
 0006:00000038       __369DBA4C_memoryapi@h     1003d038     stdafx.obj
 0006:00000039       __02D65571_enclaveapi@h    1003d039     stdafx.obj
 0006:0000003a       __50387E19_threadpoollegacyapiset@h 1003d03a     stdafx.obj
 0006:0000003b       __C40195AA_threadpoolapiset@h 1003d03b     stdafx.obj
 0006:0000003c       __792B5764_jobapi@h        1003d03c     stdafx.obj
 0006:0000003d       __BAD0D5EB_jobapi2@h       1003d03d     stdafx.obj
 0006:0000003e       __C6FE0B21_wow64apiset@h   1003d03e     stdafx.obj
 0006:0000003f       __94EE79C1_libloaderapi@h  1003d03f     stdafx.obj
 0006:00000040       __E203BDE6_securitybaseapi@h 1003d040     stdafx.obj
 0006:00000041       __9590F1DC_namespaceapi@h  1003d041     stdafx.obj
 0006:00000042       __0F4602F6_systemtopologyapi@h 1003d042     stdafx.obj
 0006:00000043       __B1B3B677_processtopologyapi@h 1003d043     stdafx.obj
 0006:00000044       __7DD200C2_securityappcontainer@h 1003d044     stdafx.obj
 0006:00000045       __130664A2_realtimeapiset@h 1003d045     stdafx.obj
 0006:00000046       __A8C6672F_winerror@h      1003d046     stdafx.obj
 0006:00000047       __A093DD28_timezoneapi@h   1003d047     stdafx.obj
 0006:00000048       __6BD3506C_winbase@h       1003d048     stdafx.obj
 0006:00000049       __DABCB3B7_wingdi@h        1003d049     stdafx.obj
 0006:0000004a       __CD8F5E54_tvout@h         1003d04a     stdafx.obj
 0006:0000004b       __033B1B1B_winuser@h       1003d04b     stdafx.obj
 0006:0000004c       __F8663FCA_datetimeapi@h   1003d04c     stdafx.obj
 0006:0000004d       __03A9DF8F_winnls@h        1003d04d     stdafx.obj
 0006:0000004e       __CB7A78CC_stringapiset@h  1003d04e     stdafx.obj
 0006:0000004f       __3F149E59_wincontypes@h   1003d04f     stdafx.obj
 0006:00000050       __7CC6F8F3_consoleapi@h    1003d050     stdafx.obj
 0006:00000051       __D4BE3EA3_consoleapi2@h   1003d051     stdafx.obj
 0006:00000052       __D57C5494_consoleapi3@h   1003d052     stdafx.obj
 0006:00000053       __FD7284F3_wincon@h        1003d053     stdafx.obj
 0006:00000054       __2EBE7A74_verrsrc@h       1003d054     stdafx.obj
 0006:00000055       __2FF32671_winver@h        1003d055     stdafx.obj
 0006:00000056       __E384C5B4_reason@h        1003d056     stdafx.obj
 0006:00000057       __C09EE12A_winreg@h        1003d057     stdafx.obj
 0006:00000058       __F1A080AC_wnnc@h          1003d058     stdafx.obj
 0006:00000059       __C375DB87_winnetwk@h      1003d059     stdafx.obj
 0006:0000005a       __F202032E_cderr@h         1003d05a     stdafx.obj
 0006:0000005b       __96C2AB0F_dde@h           1003d05b     stdafx.obj
 0006:0000005c       __005A4F24_ddeml@h         1003d05c     stdafx.obj
 0006:0000005d       __8B7EE07A_dlgs@h          1003d05d     stdafx.obj
 0006:0000005e       __0D44BE7C_lzexpand@h      1003d05e     stdafx.obj
 0006:0000005f       __7DBDB4C6_mmsyscom@h      1003d05f     stdafx.obj
 0006:00000060       __DE89C4CA_mciapi@h        1003d060     stdafx.obj
 0006:00000061       __42D37885_mmiscapi@h      1003d061     stdafx.obj
 0006:00000062       __6DE6FF2A_mmiscapi2@h     1003d062     stdafx.obj
 0006:00000063       __FF70E3D7_playsoundapi@h  1003d063     stdafx.obj
 0006:00000064       __F9747FEC_mmeapi@h        1003d064     stdafx.obj
 0006:00000065       __651C1006_timeapi@h       1003d065     stdafx.obj
 0006:00000066       __60A046E1_joystickapi@h   1003d066     stdafx.obj
 0006:00000067       __C0C01F30_mmsystem@h      1003d067     stdafx.obj
 0006:00000068       __A366D611_nb30@h          1003d068     stdafx.obj
 0006:00000069       __2CD5644B_rpcdcep@h       1003d069     stdafx.obj
 0006:0000006a       __B77D54A9_rpcdce@h        1003d06a     stdafx.obj
 0006:0000006b       __1C5A7A47_rpcnsi@h        1003d06b     stdafx.obj
 0006:0000006c       __71643EA7_rpcnterr@h      1003d06c     stdafx.obj
 0006:0000006d       __38122515_rpcasync@h      1003d06d     stdafx.obj
 0006:0000006e       __DEF407DB_rpc@h           1003d06e     stdafx.obj
 0006:0000006f       __064CC72C_shellapi@h      1003d06f     stdafx.obj
 0006:00000070       __6AB78C00_winperf@h       1003d070     stdafx.obj
 0006:00000071       __683BB200_inaddr@h        1003d071     stdafx.obj
 0006:00000072       __46EE45A6_winsock@h       1003d072     stdafx.obj
 0006:00000073       __924250EA_bcrypt@h        1003d073     stdafx.obj
 0006:00000074       __7D79DD11_ncrypt@h        1003d074     stdafx.obj
 0006:00000075       __C925E4C0_dpapi@h         1003d075     stdafx.obj
 0006:00000076       __CE4C9021_wincrypt@h      1003d076     stdafx.obj
 0006:00000077       __1BC40EFA_winefs@h        1003d077     stdafx.obj
 0006:00000078       __6BCC8C1A_rpcnsip@h       1003d078     stdafx.obj
 0006:00000079       __C065EC3F_rpcsal@h        1003d079     stdafx.obj
 0006:0000007a       __7973C144_rpcndr@h        1003d07a     stdafx.obj
 0006:0000007b       __B58B1953_wtypesbase@h    1003d07b     stdafx.obj
 0006:0000007c       __013FEE7F_wtypes@h        1003d07c     stdafx.obj
 0006:0000007d       __62733496_winioctl@h      1003d07d     stdafx.obj
 0006:0000007e       __B9109027_winsmcrd@h      1003d07e     stdafx.obj
 0006:0000007f       __87A76A69_winscard@h      1003d07f     stdafx.obj
 0006:00000080       __8C0F76A7_prsht@h         1003d080     stdafx.obj
 0006:00000081       __11B57AC7_winspool@h      1003d081     stdafx.obj
 0006:00000082       __494656A0_corecrt_malloc@h 1003d082     stdafx.obj
 0006:00000083       __0C5B3DCC_stddef@h        1003d083     stdafx.obj
 0006:00000084       __F1F53BCE_corecrt_search@h 1003d084     stdafx.obj
 0006:00000085       __DD5AA43A_corecrt_wstdlib@h 1003d085     stdafx.obj
 0006:00000086       __7B399007_limits@h        1003d086     stdafx.obj
 0006:00000087       __71F46169_stdlib@h        1003d087     stdafx.obj
 0006:00000088       __DBA05CC8_unknwnbase@h    1003d088     stdafx.obj
 0006:00000089       __D99DEA84_objidlbase@h    1003d089     stdafx.obj
 0006:0000008a       __A2F85269_cguid@h         1003d08a     stdafx.obj
 0006:0000008b       __A856EBD7_combaseapi@h    1003d08b     stdafx.obj
 0006:0000008c       __47009772_unknwn@h        1003d08c     stdafx.obj
 0006:0000008d       __558FF34F_objidl@h        1003d08d     stdafx.obj
 0006:0000008e       __EA6828E6_oaidl@h         1003d08e     stdafx.obj
 0006:0000008f       __DD5918D8_propidlbase@h   1003d08f     stdafx.obj
 0006:00000090       __A0E2593F_coml2api@h      1003d090     stdafx.obj
 0006:00000091       __F4E63AC7_oleidl@h        1003d091     stdafx.obj
 0006:00000092       __0E8757FF_servprov@h      1003d092     stdafx.obj
 0006:00000093       __13616BE7_msxml@h         1003d093     stdafx.obj
 0006:00000094       __287654D0_urlmon@h        1003d094     stdafx.obj
 0006:00000095       __3465A794_propidl@h       1003d095     stdafx.obj
 0006:00000096       __D5EE8840_objbase@h       1003d096     stdafx.obj
 0006:00000097       __B5981418_oleauto@h       1003d097     stdafx.obj
 0006:00000098       __3AE83FC5_ole2@h          1003d098     stdafx.obj
 0006:00000099       __5F30FE09_commdlg@h       1003d099     stdafx.obj
 0006:0000009a       __DD9DD587_stralign@h      1003d09a     stdafx.obj
 0006:0000009b       __B85B9837_winsvc@h        1003d09b     stdafx.obj
 0006:0000009c       __12FBC1E4_mcx@h           1003d09c     stdafx.obj
 0006:0000009d       __BC6D10F5_ime_cmodes@h    1003d09d     stdafx.obj
 0006:0000009e       __1D49718C_imm@h           1003d09e     stdafx.obj
 0006:0000009f       __95734585_windows@h       1003d09f     stdafx.obj
 0006:000000a0       __C9149A6D_xkeycheck@h     1003d0a0     stdafx.obj
 0006:000000a1       __94F3B4AE_yvals_core@h    1003d0a1     stdafx.obj
 0006:000000a2       __C54FBE38_stdint@h        1003d0a2     stdafx.obj
 0006:000000a3       __2308314D_cstdint         1003d0a3     stdafx.obj
 0006:000000a4       __05E338F6_xtr1common      1003d0a4     stdafx.obj
 0006:000000a5       __3B9D0A9D_cstddef         1003d0a5     stdafx.obj
 0006:000000a6       __92857972_corecrt_math@h  1003d0a6     stdafx.obj
 0006:000000a7       __A29DED85_math@h          1003d0a7     stdafx.obj
 0006:000000a8       __9E56D030_cstdlib         1003d0a8     stdafx.obj
 0006:000000a9       __D7870C25_initializer_list 1003d0a9     stdafx.obj
 0006:000000aa       __5E44C2A9_xstddef         1003d0aa     stdafx.obj
 0006:000000ab       __87BD5CA6_type_traits     1003d0ab     stdafx.obj
 0006:000000ac       __A95B55BB_utility         1003d0ac     stdafx.obj
 0006:000000ad       __EE76B579___msvc_iter_core@hpp 1003d0ad     stdafx.obj
 0006:000000ae       __DC58087B_tuple           1003d0ae     stdafx.obj
 0006:000000af       __CDB0EEF0_float@h         1003d0af     stdafx.obj
 0006:000000b0       __D5150992_cfloat          1003d0b0     stdafx.obj
 0006:000000b1       __1AB9F2C2_climits         1003d0b1     stdafx.obj
 0006:000000b2       __C44F8F6B_corecrt_stdio_config@h 1003d0b2     stdafx.obj
 0006:000000b3       __A7F89B2B_corecrt_wstdio@h 1003d0b3     stdafx.obj
 0006:000000b4       __B5C48800_stdio@h         1003d0b4     stdafx.obj
 0006:000000b5       __A651C215_cstdio          1003d0b5     stdafx.obj
 0006:000000b6       __E387ED1C_corecrt_wconio@h 1003d0b6     stdafx.obj
 0006:000000b7       __02A4DD57_corecrt_wdirect@h 1003d0b7     stdafx.obj
 0006:000000b8       __A056EFF3_corecrt_share@h 1003d0b8     stdafx.obj
 0006:000000b9       __91FC0EDF_corecrt_wio@h   1003d0b9     stdafx.obj
 0006:000000ba       __6619318A_corecrt_wprocess@h 1003d0ba     stdafx.obj
 0006:000000bb       __18070508_corecrt_wtime@h 1003d0bb     stdafx.obj
 0006:000000bc       __3D2AFB26_types@h         1003d0bc     stdafx.obj
 0006:000000bd       __72103B05_stat@h          1003d0bd     stdafx.obj
 0006:000000be       __4BE26BFD_wchar@h         1003d0be     stdafx.obj
 0006:000000bf       __3CDA1446_cwchar          1003d0bf     stdafx.obj
 0006:000000c0       __99FA516B_intrin0@inl@h   1003d0c0     stdafx.obj
 0006:000000c1       __8CEB98C2_intrin0@h       1003d0c1     stdafx.obj
 0006:000000c2       __B83F831D_isa_availability@h 1003d0c2     stdafx.obj
 0006:000000c3       __B3F344F6_limits          1003d0c3     stdafx.obj
 0006:000000c4       __E81B5085_vcruntime_new@h 1003d0c4     stdafx.obj
 0006:000000c5       __130137D5_vcruntime_new_debug@h 1003d0c5     stdafx.obj
 0006:000000c6       __8CF369C8_crtdbg@h        1003d0c6     stdafx.obj
 0006:000000c7       __95C621C9_crtdefs@h       1003d0c7     stdafx.obj
 0006:000000c8       __FEED0ABF_use_ansi@h      1003d0c8     stdafx.obj
 0006:000000c9       __2816668F_yvals@h         1003d0c9     stdafx.obj
 0006:000000ca       __E5D9469F_malloc@h        1003d0ca     stdafx.obj
 0006:000000cb       __C78E68C1_corecrt_terminate@h 1003d0cb     stdafx.obj
 0006:000000cc       __510B0051_eh@h            1003d0cc     stdafx.obj
 0006:000000cd       __1BEF3287_vcruntime_exception@h 1003d0cd     stdafx.obj
 0006:000000ce       __5D994F5F_exception       1003d0ce     stdafx.obj
 0006:000000cf       __7E4C13A5_new             1003d0cf     stdafx.obj
 0006:000000d0       __5795C389_xatomic@h       1003d0d0     stdafx.obj
 0006:000000d1       __D2C478D0_cstring         1003d0d1     stdafx.obj
 0006:000000d2       __A997C6C5_xutility        1003d0d2     stdafx.obj
 0006:000000d3       __C3CE3678_xmemory         1003d0d3     stdafx.obj
 0006:000000d4       __7352ED38_xtree           1003d0d4     stdafx.obj
 0006:000000d5       __8602FD5B_map             1003d0d5     stdafx.obj
 0006:000000d6       __7C4CD365_INITGUID@H      1003d0d6     stdafx.obj
 0006:000000d7       __D33F56CB_public@h        1003d0d7     stdafx.obj
 0006:000000d8       __701FEF85_stdafx@h        1003d0d8     stdafx.obj
 0006:000000d9       __5DDD8A17_vJoyInterface@pch 1003d0d9     stdafx.obj
 0006:000000da       __8D78C31F_stdafx@cpp      1003d0da     stdafx.obj
 0006:00000106       __E1218CD7_targetver@h     1003d106     vJoyInterface.obj
 0006:00000107       __3347223C_winpackagefamily@h 1003d107     vJoyInterface.obj
 0006:00000108       __F5B671E4_winapifamily@h  1003d108     vJoyInterface.obj
 0006:00000109       __6866F092_sdkddkver@h     1003d109     vJoyInterface.obj
 0006:0000010a       __CD417A16_concurrencysal@h 1003d10a     vJoyInterface.obj
 0006:0000010b       __18C11F8D_sal@h           1003d10b     vJoyInterface.obj
 0006:0000010c       __BD42D05E_vadefs@h        1003d10c     vJoyInterface.obj
 0006:0000010d       __2DC9DF70_vcruntime@h     1003d10d     vJoyInterface.obj
 0006:0000010e       __D7225C87_excpt@h         1003d10e     vJoyInterface.obj
 0006:0000010f       __F19000F7_stdarg@h        1003d10f     vJoyInterface.obj
 0006:00000110       __4114BAD5_specstrings_undef@h 1003d110     vJoyInterface.obj
 0006:00000111       __50F9AEDC_specstrings_strict@h 1003d111     vJoyInterface.obj
 0006:00000112       __BEFC0098_sdv_driverspecs@h 1003d112     vJoyInterface.obj
 0006:00000113       __39A39701_driverspecs@h   1003d113     vJoyInterface.obj
 0006:00000114       __B4D8BDAA_specstrings@h   1003d114     vJoyInterface.obj
 0006:00000115       __04C75F1C_corecrt@h       1003d115     vJoyInterface.obj
 0006:00000116       __78D0C915_corecrt_wctype@h 1003d116     vJoyInterface.obj
 0006:00000117       __6AECDA3E_ctype@h         1003d117     vJoyInterface.obj
 0006:00000118       __B6CCE7CD_kernelspecs@h   1003d118     vJoyInterface.obj
 0006:00000119       __201B1099_basetsd@h       1003d119     vJoyInterface.obj
 0006:0000011a       __15E49872_errno@h         1003d11a     vJoyInterface.obj
 0006:0000011b       __6BB4896E_vcruntime_string@h 1003d11b     vJoyInterface.obj
 0006:0000011c       __184F7456_corecrt_memcpy_s@h 1003d11c     vJoyInterface.obj
 0006:0000011d       __82377222_corecrt_memory@h 1003d11d     vJoyInterface.obj
 0006:0000011e       __5B29309E_corecrt_wstring@h 1003d11e     vJoyInterface.obj
 0006:0000011f       __F787F5CD_string@h        1003d11f     vJoyInterface.obj
 0006:00000120       __8C99318D_guiddef@h       1003d120     vJoyInterface.obj
 0006:00000121       __A3CAA675_pshpack4@h      1003d121     vJoyInterface.obj
 0006:00000122       __2611E9B9_poppack@h       1003d122     vJoyInterface.obj
 0006:00000123       __A747DAC7_pshpack2@h      1003d123     vJoyInterface.obj
 0006:00000124       __AAD05F11_pshpack8@h      1003d124     vJoyInterface.obj
 0006:00000125       __A501649E_pshpack1@h      1003d125     vJoyInterface.obj
 0006:00000126       __0E9D9C0E_apiset@h        1003d126     vJoyInterface.obj
 0006:00000127       __F9851A06_ktmtypes@h      1003d127     vJoyInterface.obj
 0006:00000128       __9DA2B69E_winnt@h         1003d128     vJoyInterface.obj
 0006:00000129       __E9AED855_minwindef@h     1003d129     vJoyInterface.obj
 0006:0000012a       __9668718B_windef@h        1003d12a     vJoyInterface.obj
 0006:0000012b       __B47C9622_apisetcconv@h   1003d12b     vJoyInterface.obj
 0006:0000012c       __77F4CE3E_minwinbase@h    1003d12c     vJoyInterface.obj
 0006:0000012d       __42CF8FD5_apiquery2@h     1003d12d     vJoyInterface.obj
 0006:0000012e       __A6C51434_processenv@h    1003d12e     vJoyInterface.obj
 0006:0000012f       __415D7145_fileapi@h       1003d12f     vJoyInterface.obj
 0006:00000130       __A7316A9B_fileapifromapp@h 1003d130     vJoyInterface.obj
 0006:00000131       __A0359A2D_debugapi@h      1003d131     vJoyInterface.obj
 0006:00000132       __28BE1226_utilapiset@h    1003d132     vJoyInterface.obj
 0006:00000133       __6933B394_handleapi@h     1003d133     vJoyInterface.obj
 0006:00000134       __57F09DF9_errhandlingapi@h 1003d134     vJoyInterface.obj
 0006:00000135       __E0622DF9_fibersapi@h     1003d135     vJoyInterface.obj
 0006:00000136       __D531F6AB_namedpipeapi@h  1003d136     vJoyInterface.obj
 0006:00000137       __ADD82BB4_profileapi@h    1003d137     vJoyInterface.obj
 0006:00000138       __ECFC4D70_heapapi@h       1003d138     vJoyInterface.obj
 0006:00000139       __4F41815B_ioapiset@h      1003d139     vJoyInterface.obj
 0006:0000013a       __8D44BFB7_synchapi@h      1003d13a     vJoyInterface.obj
 0006:0000013b       __8CAEC090_interlockedapi@h 1003d13b     vJoyInterface.obj
 0006:0000013c       __8ABF54F4_processthreadsapi@h 1003d13c     vJoyInterface.obj
 0006:0000013d       __1462A586_sysinfoapi@h    1003d13d     vJoyInterface.obj
 0006:0000013e       __369DBA4C_memoryapi@h     1003d13e     vJoyInterface.obj
 0006:0000013f       __02D65571_enclaveapi@h    1003d13f     vJoyInterface.obj
 0006:00000140       __50387E19_threadpoollegacyapiset@h 1003d140     vJoyInterface.obj
 0006:00000141       __C40195AA_threadpoolapiset@h 1003d141     vJoyInterface.obj
 0006:00000142       __792B5764_jobapi@h        1003d142     vJoyInterface.obj
 0006:00000143       __BAD0D5EB_jobapi2@h       1003d143     vJoyInterface.obj
 0006:00000144       __C6FE0B21_wow64apiset@h   1003d144     vJoyInterface.obj
 0006:00000145       __94EE79C1_libloaderapi@h  1003d145     vJoyInterface.obj
 0006:00000146       __E203BDE6_securitybaseapi@h 1003d146     vJoyInterface.obj
 0006:00000147       __9590F1DC_namespaceapi@h  1003d147     vJoyInterface.obj
 0006:00000148       __0F4602F6_systemtopologyapi@h 1003d148     vJoyInterface.obj
 0006:00000149       __B1B3B677_processtopologyapi@h 1003d149     vJoyInterface.obj
 0006:0000014a       __7DD200C2_securityappcontainer@h 1003d14a     vJoyInterface.obj
 0006:0000014b       __130664A2_realtimeapiset@h 1003d14b     vJoyInterface.obj
 0006:0000014c       __A8C6672F_winerror@h      1003d14c     vJoyInterface.obj
 0006:0000014d       __A093DD28_timezoneapi@h   1003d14d     vJoyInterface.obj
 0006:0000014e       __6BD3506C_winbase@h       1003d14e     vJoyInterface.obj
 0006:0000014f       __DABCB3B7_wingdi@h        1003d14f     vJoyInterface.obj
 0006:00000150       __CD8F5E54_tvout@h         1003d150     vJoyInterface.obj
 0006:00000151       __033B1B1B_winuser@h       1003d151     vJoyInterface.obj
 0006:00000152       __F8663FCA_datetimeapi@h   1003d152     vJoyInterface.obj
 0006:00000153       __03A9DF8F_winnls@h        1003d153     vJoyInterface.obj
 0006:00000154       __CB7A78CC_stringapiset@h  1003d154     vJoyInterface.obj
 0006:00000155       __3F149E59_wincontypes@h   1003d155     vJoyInterface.obj
 0006:00000156       __7CC6F8F3_consoleapi@h    1003d156     vJoyInterface.obj
 0006:00000157       __D4BE3EA3_consoleapi2@h   1003d157     vJoyInterface.obj
 0006:00000158       __D57C5494_consoleapi3@h   1003d158     vJoyInterface.obj
 0006:00000159       __FD7284F3_wincon@h        1003d159     vJoyInterface.obj
 0006:0000015a       __2EBE7A74_verrsrc@h       1003d15a     vJoyInterface.obj
 0006:0000015b       __2FF32671_winver@h        1003d15b     vJoyInterface.obj
 0006:0000015c       __E384C5B4_reason@h        1003d15c     vJoyInterface.obj
 0006:0000015d       __C09EE12A_winreg@h        1003d15d     vJoyInterface.obj
 0006:0000015e       __F1A080AC_wnnc@h          1003d15e     vJoyInterface.obj
 0006:0000015f       __C375DB87_winnetwk@h      1003d15f     vJoyInterface.obj
 0006:00000160       __F202032E_cderr@h         1003d160     vJoyInterface.obj
 0006:00000161       __96C2AB0F_dde@h           1003d161     vJoyInterface.obj
 0006:00000162       __005A4F24_ddeml@h         1003d162     vJoyInterface.obj
 0006:00000163       __8B7EE07A_dlgs@h          1003d163     vJoyInterface.obj
 0006:00000164       __0D44BE7C_lzexpand@h      1003d164     vJoyInterface.obj
 0006:00000165       __7DBDB4C6_mmsyscom@h      1003d165     vJoyInterface.obj
 0006:00000166       __DE89C4CA_mciapi@h        1003d166     vJoyInterface.obj
 0006:00000167       __42D37885_mmiscapi@h      1003d167     vJoyInterface.obj
 0006:00000168       __6DE6FF2A_mmiscapi2@h     1003d168     vJoyInterface.obj
 0006:00000169       __FF70E3D7_playsoundapi@h  1003d169     vJoyInterface.obj
 0006:0000016a       __F9747FEC_mmeapi@h        1003d16a     vJoyInterface.obj
 0006:0000016b       __651C1006_timeapi@h       1003d16b     vJoyInterface.obj
 0006:0000016c       __60A046E1_joystickapi@h   1003d16c     vJoyInterface.obj
 0006:0000016d       __C0C01F30_mmsystem@h      1003d16d     vJoyInterface.obj
 0006:0000016e       __A366D611_nb30@h          1003d16e     vJoyInterface.obj
 0006:0000016f       __2CD5644B_rpcdcep@h       1003d16f     vJoyInterface.obj
 0006:00000170       __B77D54A9_rpcdce@h        1003d170     vJoyInterface.obj
 0006:00000171       __1C5A7A47_rpcnsi@h        1003d171     vJoyInterface.obj
 0006:00000172       __71643EA7_rpcnterr@h      1003d172     vJoyInterface.obj
 0006:00000173       __38122515_rpcasync@h      1003d173     vJoyInterface.obj
 0006:00000174       __DEF407DB_rpc@h           1003d174     vJoyInterface.obj
 0006:00000175       __064CC72C_shellapi@h      1003d175     vJoyInterface.obj
 0006:00000176       __6AB78C00_winperf@h       1003d176     vJoyInterface.obj
 0006:00000177       __683BB200_inaddr@h        1003d177     vJoyInterface.obj
 0006:00000178       __46EE45A6_winsock@h       1003d178     vJoyInterface.obj
 0006:00000179       __924250EA_bcrypt@h        1003d179     vJoyInterface.obj
 0006:0000017a       __7D79DD11_ncrypt@h        1003d17a     vJoyInterface.obj
 0006:0000017b       __C925E4C0_dpapi@h         1003d17b     vJoyInterface.obj
 0006:0000017c       __CE4C9021_wincrypt@h      1003d17c     vJoyInterface.obj
 0006:0000017d       __1BC40EFA_winefs@h        1003d17d     vJoyInterface.obj
 0006:0000017e       __6BCC8C1A_rpcnsip@h       1003d17e     vJoyInterface.obj
 0006:0000017f       __C065EC3F_rpcsal@h        1003d17f     vJoyInterface.obj
 0006:00000180       __7973C144_rpcndr@h        1003d180     vJoyInterface.obj
 0006:00000181       __B58B1953_wtypesbase@h    1003d181     vJoyInterface.obj
 0006:00000182       __013FEE7F_wtypes@h        1003d182     vJoyInterface.obj
 0006:00000183       __62733496_winioctl@h      1003d183     vJoyInterface.obj
 0006:00000184       __B9109027_winsmcrd@h      1003d184     vJoyInterface.obj
 0006:00000185       __87A76A69_winscard@h      1003d185     vJoyInterface.obj
 0006:00000186       __8C0F76A7_prsht@h         1003d186     vJoyInterface.obj
 0006:00000187       __11B57AC7_winspool@h      1003d187     vJoyInterface.obj
 0006:00000188       __494656A0_corecrt_malloc@h 1003d188     vJoyInterface.obj
 0006:00000189       __0C5B3DCC_stddef@h        1003d189     vJoyInterface.obj
 0006:0000018a       __F1F53BCE_corecrt_search@h 1003d18a     vJoyInterface.obj
 0006:0000018b       __DD5AA43A_corecrt_wstdlib@h 1003d18b     vJoyInterface.obj
 0006:0000018c       __7B399007_limits@h        1003d18c     vJoyInterface.obj
 0006:0000018d       __71F46169_stdlib@h        1003d18d     vJoyInterface.obj
 0006:0000018e       __DBA05CC8_unknwnbase@h    1003d18e     vJoyInterface.obj
 0006:0000018f       __D99DEA84_objidlbase@h    1003d18f     vJoyInterface.obj
 0006:00000190       __A2F85269_cguid@h         1003d190     vJoyInterface.obj
 0006:00000191       __A856EBD7_combaseapi@h    1003d191     vJoyInterface.obj
 0006:00000192       __47009772_unknwn@h        1003d192     vJoyInterface.obj
 0006:00000193       __558FF34F_objidl@h        1003d193     vJoyInterface.obj
 0006:00000194       __EA6828E6_oaidl@h         1003d194     vJoyInterface.obj
 0006:00000195       __DD5918D8_propidlbase@h   1003d195     vJoyInterface.obj
 0006:00000196       __A0E2593F_coml2api@h      1003d196     vJoyInterface.obj
 0006:00000197       __F4E63AC7_oleidl@h        1003d197     vJoyInterface.obj
 0006:00000198       __0E8757FF_servprov@h      1003d198     vJoyInterface.obj
 0006:00000199       __13616BE7_msxml@h         1003d199     vJoyInterface.obj
 0006:0000019a       __287654D0_urlmon@h        1003d19a     vJoyInterface.obj
 0006:0000019b       __3465A794_propidl@h       1003d19b     vJoyInterface.obj
 0006:0000019c       __D5EE8840_objbase@h       1003d19c     vJoyInterface.obj
 0006:0000019d       __B5981418_oleauto@h       1003d19d     vJoyInterface.obj
 0006:0000019e       __3AE83FC5_ole2@h          1003d19e     vJoyInterface.obj
 0006:0000019f       __5F30FE09_commdlg@h       1003d19f     vJoyInterface.obj
 0006:000001a0       __DD9DD587_stralign@h      1003d1a0     vJoyInterface.obj
 0006:000001a1       __B85B9837_winsvc@h        1003d1a1     vJoyInterface.obj
 0006:000001a2       __12FBC1E4_mcx@h           1003d1a2     vJoyInterface.obj
 0006:000001a3       __BC6D10F5_ime_cmodes@h    1003d1a3     vJoyInterface.obj
 0006:000001a4       __1D49718C_imm@h           1003d1a4     vJoyInterface.obj
 0006:000001a5       __95734585_windows@h       1003d1a5     vJoyInterface.obj
 0006:000001a6       __C9149A6D_xkeycheck@h     1003d1a6     vJoyInterface.obj
 0006:000001a7       __94F3B4AE_yvals_core@h    1003d1a7     vJoyInterface.obj
 0006:000001a8       __C54FBE38_stdint@h        1003d1a8     vJoyInterface.obj
 0006:000001a9       __2308314D_cstdint         1003d1a9     vJoyInterface.obj
 0006:000001aa       __05E338F6_xtr1common      1003d1aa     vJoyInterface.obj
 0006:000001ab       __3B9D0A9D_cstddef         1003d1ab     vJoyInterface.obj
 0006:000001ac       __92857972_corecrt_math@h  1003d1ac     vJoyInterface.obj
 0006:000001ad       __A29DED85_math@h          1003d1ad     vJoyInterface.obj
 0006:000001ae       __9E56D030_cstdlib         1003d1ae     vJoyInterface.obj
 0006:000001af       __D7870C25_initializer_list 1003d1af     vJoyInterface.obj
 0006:000001b0       __5E44C2A9_xstddef         1003d1b0     vJoyInterface.obj
 0006:000001b1       __87BD5CA6_type_traits     1003d1b1     vJoyInterface.obj
 0006:000001b2       __A95B55BB_utility         1003d1b2     vJoyInterface.obj
 0006:000001b3       __EE76B579___msvc_iter_core@hpp 1003d1b3     vJoyInterface.obj
 0006:000001b4       __DC58087B_tuple           1003d1b4     vJoyInterface.obj
 0006:000001b5       __CDB0EEF0_float@h         1003d1b5     vJoyInterface.obj
 0006:000001b6       __D5150992_cfloat          1003d1b6     vJoyInterface.obj
 0006:000001b7       __1AB9F2C2_climits         1003d1b7     vJoyInterface.obj
 0006:000001b8       __C44F8F6B_corecrt_stdio_config@h 1003d1b8     vJoyInterface.obj
 0006:000001b9       __A7F89B2B_corecrt_wstdio@h 1003d1b9     vJoyInterface.obj
 0006:000001ba       __B5C48800_stdio@h         1003d1ba     vJoyInterface.obj
 0006:000001bb       __A651C215_cstdio          1003d1bb     vJoyInterface.obj
 0006:000001bc       __E387ED1C_corecrt_wconio@h 1003d1bc     vJoyInterface.obj
 0006:000001bd       __02A4DD57_corecrt_wdirect@h 1003d1bd     vJoyInterface.obj
 0006:000001be       __A056EFF3_corecrt_share@h 1003d1be     vJoyInterface.obj
 0006:000001bf       __91FC0EDF_corecrt_wio@h   1003d1bf     vJoyInterface.obj
 0006:000001c0       __6619318A_corecrt_wprocess@h 1003d1c0     vJoyInterface.obj
 0006:000001c1       __18070508_corecrt_wtime@h 1003d1c1     vJoyInterface.obj
 0006:000001c2       __3D2AFB26_types@h         1003d1c2     vJoyInterface.obj
 0006:000001c3       __72103B05_stat@h          1003d1c3     vJoyInterface.obj
 0006:000001c4       __4BE26BFD_wchar@h         1003d1c4     vJoyInterface.obj
 0006:000001c5       __3CDA1446_cwchar          1003d1c5     vJoyInterface.obj
 0006:000001c6       __99FA516B_intrin0@inl@h   1003d1c6     vJoyInterface.obj
 0006:000001c7       __8CEB98C2_intrin0@h       1003d1c7     vJoyInterface.obj
 0006:000001c8       __B83F831D_isa_availability@h 1003d1c8     vJoyInterface.obj
 0006:000001c9       __B3F344F6_limits          1003d1c9     vJoyInterface.obj
 0006:000001ca       __E81B5085_vcruntime_new@h 1003d1ca     vJoyInterface.obj
 0006:000001cb       __130137D5_vcruntime_new_debug@h 1003d1cb     vJoyInterface.obj
 0006:000001cc       __8CF369C8_crtdbg@h        1003d1cc     vJoyInterface.obj
 0006:000001cd       __95C621C9_crtdefs@h       1003d1cd     vJoyInterface.obj
 0006:000001ce       __FEED0ABF_use_ansi@h      1003d1ce     vJoyInterface.obj
 0006:000001cf       __2816668F_yvals@h         1003d1cf     vJoyInterface.obj
 0006:000001d0       __E5D9469F_malloc@h        1003d1d0     vJoyInterface.obj
 0006:000001d1       __C78E68C1_corecrt_terminate@h 1003d1d1     vJoyInterface.obj
 0006:000001d2       __510B0051_eh@h            1003d1d2     vJoyInterface.obj
 0006:000001d3       __1BEF3287_vcruntime_exception@h 1003d1d3     vJoyInterface.obj
 0006:000001d4       __5D994F5F_exception       1003d1d4     vJoyInterface.obj
 0006:000001d5       __7E4C13A5_new             1003d1d5     vJoyInterface.obj
 0006:000001d6       __5795C389_xatomic@h       1003d1d6     vJoyInterface.obj
 0006:000001d7       __D2C478D0_cstring         1003d1d7     vJoyInterface.obj
 0006:000001d8       __A997C6C5_xutility        1003d1d8     vJoyInterface.obj
 0006:000001d9       __C3CE3678_xmemory         1003d1d9     vJoyInterface.obj
 0006:000001da       __7352ED38_xtree           1003d1da     vJoyInterface.obj
 0006:000001db       __8602FD5B_map             1003d1db     vJoyInterface.obj
 0006:000001dc       __7C4CD365_INITGUID@H      1003d1dc     vJoyInterface.obj
 0006:000001dd       __D33F56CB_public@h        1003d1dd     vJoyInterface.obj
 0006:000001de       __701FEF85_stdafx@h        1003d1de     vJoyInterface.obj
 0006:000001df       __5DDD8A17_vJoyInterface@pch 1003d1df     vJoyInterface.obj
 0006:000001e0       __06BD36BF_assert@h        1003d1e0     vJoyInterface.obj
 0006:000001e1       __C1D62156_spapidef@h      1003d1e1     vJoyInterface.obj
 0006:000001e2       __1C2F47EE_dpa_dsa@h       1003d1e2     vJoyInterface.obj
 0006:000001e3       __C5859B4B_commctrl@h      1003d1e3     vJoyInterface.obj
 0006:000001e4       __77B432AB_devpropdef@h    1003d1e4     vJoyInterface.obj
 0006:000001e5       __C1400A33_setupapi@h      1003d1e5     vJoyInterface.obj
 0006:000001e6       __B8BC9EA1_hidusage@h      1003d1e6     vJoyInterface.obj
 0006:000001e7       __CB81E9A0_hidpi@h         1003d1e7     vJoyInterface.obj
 0006:000001e8       __0A3E78F6_Hidsdi@h        1003d1e8     vJoyInterface.obj
 0006:000001e9       __6F8C1290_Dbt@h           1003d1e9     vJoyInterface.obj
 0006:000001ea       __7A0A7160_tchar@h         1003d1ea     vJoyInterface.obj
 0006:000001eb       __67E0D18C_vJoyInterface@h 1003d1eb     vJoyInterface.obj
 0006:000001ec       __8D63CA82_vJoyInterface@cpp 1003d1ec     vJoyInterface.obj
 0008:00000270       $R000000                   1003f270     version.res
 0008:00000280       $R000010                   1003f280     version.res
 0008:00000288       $R000018                   1003f288     version.res
 0008:00000608       $R000398                   1003f608     version.res
